:020000021000EC
:10F00000F0FF002039F5010061F5010063F5010012
:10F0100065F5010067F5010069F5010000000000D9
:10F020000000000000000000000000006BF501007F
:10F030006DF50100000000006FF50100FD98030070
:10F04000C54D020073F50100B94F0200254E0200C4
:10F05000714E020073F501006951020073F5010061
:10F0600073F501004199030073F5010073F5010088
:10F0700073F50100915A020073F5010073F5010068
:10F080003D9903008D29020073F5010073F501001D
:10F09000952A020091BD0300111B020073F50100C7
:10F0A00073F5010073F5010073F5010073F50100BC
:10F0B00073F5010073F5010000000000000000007E
:10F0C00073F5010073F5010073F5010073F501009C
:10F0D00073F501005D5C020073F5010000000000A3
:10F0E0000000000000000000000000000000000020
:10F0F0000000000000000000000000000000000010
:10F1000000000000000000000000000000000000FF
:10F1100000000000000000000000000000000000EF
:10F4000010B5054C237833B9044B13B10448AFF35E
:10F4100000800123237010BD382D00200000000063
:10F42000B0B7050008B5034B1BB103490348AFF360
:10F43000008008BD000000003C2D0020B0B7050092
:10F44000154B002B08BF134B9D46A3F5803A0021B6
:10F450008B460F461348144A121A00F063F80F4BFC
:10F46000002B00D098470E4B002B00D0984700206F
:10F47000002104000D000D48002802D00C48AFF315
:10F48000008000F02BF8200029001EF027FD00F07E
:10F4900011F800BF00000800F0FF0020000000008D
:10F4A00000000000382D0020A4B300200000000060
:10F4B0000000000008B5074B044613B10021AFF36C
:10F4C0000080054B1868836A03B19847204600F016
:10F4D00031F800BF00000000E83A050070B50D4D9E
:10F4E0000D4C641BA4100026A64209D10B4D0C4CF8
:10F4F00034F0EEFA641BA4100026A64205D170BDBC
:10F5000055F8043B98470136EEE755F8043B984719
:10F510000136F2E7202D0020202D0020202D002094
:10F52000242D002002440346934200D1704703F883
:10F53000011BF9E7FEE700BF0649074A074B9B1A84
:10F5400003DD043BC858D050FBDC06F075FCFFF728
:10F5500077FF0000BCB70500402C0020382D0020AC
:10F56000FEE7FEE7FEE7FEE7FEE7FEE7FEE7FEE773
:10F57000FEE7FEE71FB501238DF80030054B8DF83F
:10F58000080001916846D3E90012904705B05DF884
:10F5900004FB00BF80A0002061DF704748DF704798
:10F5A00010B50388012B11D8094A02EB03124388D6
:10F5B0005189CC1A032C09D4C3F57F43FD330B4486
:10F5C0005381002303804380184610BD0420FCE7CC
:10F5D00054A4002010B5124A0B6802EB00104268D8
:10F5E00073B15888033003EB800302F580524FF665
:10F5F000FF749A4202D91868013004D1002009E052
:10F6000002F10803F1E79888A04204D0188810B1ED
:10F610000B60012010BD5888033003EB8003E8E73E
:10F6200054A4002073B5436804460D4613B31E4A24
:10F6300011688B421ED3526893421BD813F003000B
:10F6400018D11A4A21891289914213D121689A68E6
:10F6500091420FD1164A5268934201D80A2004E021
:10F6600002F580529342F9D22880B0FA80F0400926
:10F6700002B070BD00232B801E46019601A9288888
:10F68000FFF7A8FF30B92B8801339BB22B80002BEA
:10F69000F3D0EDE7019B226899689142EED1636057
:10F6A000024B1B892381E3E7282D00203CA2002088
:10F6B00054A40020033083B240F2FD32934230B5AF
:10F6C0000ED909200BE0228965892A441A4492B296
:10F6D000B2F5806F08D2088062891344638130BD1F
:10F6E000024C20780028EED00720F8E754A4002030
:10F6F00010B50A494A788C78531CDBB29C4208BF8B
:10F7000000230C789C421FBF0370486802EB420242
:10F7100000EBC20008BF002010BD00BFD0A3002036
:10F72000AADF7047A9DF7047A7DF704785DF704702
:10F730007FDF70477EDF7047084A30B500230C2416
:10F7400004FB03F18D5A854202D10A44508830BD32
:10F750000133082BF4D14FF6FF70F8E7A6A1002083
:10F760006EDF7047012804D0043804288CBF0020C5
:10F77000012070478378013B072B07D8DFE803F0AF
:10F7800007060606060704091423038070470123B1
:10F79000FBE743689B8809339B08F6E770B5054D86
:10F7A0000646002455F8043B304601349847052CA2
:10F7B000F8D170BDA43C0500114BF0B50022142611
:10F7C0001D4606FB02F4E75A874212D12344142651
:10F7D00000249A788A420AD001342246072A0BD89C
:10F7E00006FB02F3EF5A874208D1EB18F1D1184615
:10F7F000F0BD0132082AE4D10023F8E70132EDE739
:10F80000E8A50020F8B5074D074E074600243378D9
:10F81000A34200DCF8BD55F8043B38469847013454
:10F82000F5E700BF18A20020C9A300207DDF7047C4
:10F8300079DF70476DDF704758B1CB0801F00701E1
:10F84000C25C012303FA01F10A4214BF18460020EA
:10F85000704701207047000070B50A4E34680546B5
:10F8600054B1706860B1FF2D08D02946FFF7E4FF5E
:10F8700030B1F36803FB0544204670BD0024FBE76C
:10F880000446F9E7D8A5002030B5072185B0FFF779
:10F8900093FF044600283AD04568002D39D1007CFA
:10F8A000FFF7DAFF0721CDE902558DF80A1040B3C2
:10F8B000E368039003EB83031B019BB29B0802A840
:10F8C000ADF80830FFF756FF9DF80A00FFF74AFF32
:10F8D000D8B1114B1B789B0715D5BDF808500DF119
:10F8E00006012846FFF7E6FE48B9BDF80630A380BA
:10F8F000E5800A4B185C092803D005B030BD092803
:10F90000F7D90320F9E70220F3E70846F5E70520D9
:10F91000F3E70020F1E700BF38A20020043B050018
:10F9200038B54FF6FF73984218BF01300D4614BF2B
:10F9300084B20024FF2C03D94FF6FF74204638BD53
:10F9400021462846FFF778FF0028F7D10134A4B2FA
:10F95000F0E7000038B5074C051E04F1080318BF96
:10F960001C4623682BB11A6822605B6828469847BA
:10F97000F7E738BD58A100200023435082B0435818
:10F980000193019B02B070472DE9F0470D789DF877
:10F9900020609DF824A004460F469946002D60D1B2
:10F9A000D0F8243192F800809BB14FF49271FFF7A8
:10F9B000E3FF012363613B70B04550D1D4F80431BB
:10F9C000002B4CD04FF482712046FFF7D5FF002565
:10F9D0001DE0D0F81C31FBB14FF48E71FFF7CCFF66
:10F9E000D0F824311BB14FF492712046DFE7137831
:10F9F0009E4207D919F80330C0F81C35137801333B
:10FA00001370D9E70123BAF1000F03D0C361284670
:10FA1000BDE8F0874361CFE7D0F80831002BCBD0A9
:10FA20004FF48471FFF7A8FFD0F82431002BDAD10E
:10FA300013789E42C0D9D0F8181509F8031013782E
:10FA40000133DBB21370721E934205D10223C0F85A
:10FA5000003201232362AFE79E42FAD1ACE70125D1
:10FA6000D5E74FF49271FFF787FF4FF48E71FFF7E0
:10FA700083FF4FF48471FFF77FFF9FE72DE9F34782
:10FA80000C4605464FF4827120461F469046FFF70C
:10FA900073FF4FF49271FFF76FFF4FF48E71FFF712
:10FAA0006BFF4FF48471FFF767FF0023012F85F888
:10FAB000263085F8233008BF02224FF001030CBF27
:10FAC000C4F80022C4F80032236223602E6846BBCB
:10FAD00005F1260A05F12309CDE900764346524691
:10FAE00049462046FFF750FF0028F5D195F823300E
:10FAF000EBB1D4F8C434C4F8C434C3B113F0010F6B
:10FB000014BF4FF40240032048F2012213F0020F09
:10FB100018BF104613F0040F48F2022318BF18460E
:10FB200006E040F28623AB60AB68C4F804330020E3
:10FB300002B0BDE8F0872DE9F3470C4605464FF4C7
:10FB4000827120461F4616469DF82880FFF714FF55
:10FB50004FF49271FFF710FF4FF48E71FFF70CFF17
:10FB60004FF48471FFF708FF0023C4F8003285F8D2
:10FB7000263085F8233001232362A36095F82620E0
:10FB8000974232D9B35CC4F81C3595F8263001335E
:10FB900085F826302B687BBB05F1260A05F1230981
:10FBA000CDE900783346524649462046FFF7ECFE41
:10FBB0000028F5D195F8233023B3D4F8C434C4F821
:10FBC000C434FBB113F0010F14BF4FF40240032003
:10FBD00048F2012213F0020F18BF104613F0040F71
:10FBE00048F2022318BF18460DE0B8F1000F01D00B
:10FBF000E361CFE76361CDE740F28623AB60AB689A
:10FC0000C4F80433002002B0BDE8F087002343505D
:10FC100082B043580193019B02B0704708B5024679
:10FC20004FF492710068FFF7F1FF4FF48471106890
:10FC3000FFF7ECFF136801221A6008BD10B5CB7DF9
:10FC40000A464FF4847123B9FFF7E0FFD0F8183566
:10FC500010BDFFF7DBFF537ED168D0F81805C854FC
:10FC6000537E0133DBB25376F2E70A4610B54FF408
:10FC70008E71FFF7CBFF938A91689BB2C95C938A20
:10FC800001339BB29382C0F81C1510BD2DE9F047DB
:10FC900093F9005090B00024013D6E46AD00274618
:10FCA000A446A0465FF0000E03E05FEA080EBEEB3C
:10FCB000050EB8EB0E0952F809A051F80E90A9FBF9
:10FCC0000A9A14EB090457EB0A075CF1000C1EF1C9
:10FCD000040EAE4501DCC645EBDD46F808403C4667
:10FCE00067465FF0000C18F10408A845DADDB8EBB0
:10FCF000450FDADD46F80840D3F8B0303146984772
:10FD000010B0BDE8F08713460A46FFF7BFBFF0B555
:10FD1000154689B01C4607460E461A4629466846CF
:10FD2000FFF7F1FF23466A4639463846FFF7AEFF34
:10FD300023462A4669466846FFF7A8FF23466A46D7
:10FD400031463046FFF7A2FF09B0F0BD00EB81015C
:10FD50000023884200D3704751F8042D43EA520330
:10FD60000B60D307F5E710B5013A52B2130601D57F
:10FD7000002010BD50F8224051F822309C4205D896
:10FD800002F1FF32F2D24FF0FF30F2E70120F0E74C
:10FD900010B500235CB2A24200DC10BD51F8234034
:10FDA00040F823400133F5E7013910B549B2041D8D
:10FDB0000A06CBB204D4013954F82120002AF7D026
:10FDC00001335BB273B103F18042013A50F8222053
:10FDD000002022B9013B00EB431318B210BD5208BA
:10FDE0000130F6E71846F9E7002310B51C465AB271
:10FDF000914200DC10BD40F823400133F7E70000DA
:10FE0000C3F10803DB0070B50133002403A500BF74
:10FE10005B1920C940CAAD1B20C0184720C940CA81
:10FE2000B54120C020C940CAB54120C020C940CA40
:10FE3000B54120C020C940CAB54120C020C940CA30
:10FE4000B54120C020C940CAB54120C020C940CA20
:10FE5000B54120C06441B4FA84F0400970BD00BFD0
:10FE6000C3F10803DB0070B50133002403A500BF14
:10FE70005B1920C940CAAD1920C0184720C940CA23
:10FE8000754120C020C940CA754120C020C940CA60
:10FE9000754120C020C940CA754120C020C940CA50
:10FEA000754120C020C940CA754120C020C940CA40
:10FEB000754120C06441204670BD00BFF0B50822E6
:10FEC00089B00C460646FFF763FFCB6A03930B6BC2
:10FED00004934B6B05938B6B0693CB6B07930027B7
:10FEE00008236A4669466846CDE901770097FFF71F
:10FEF000B7FF082305466A4631463046FFF7B0FF94
:10FF0000236B0393636B0493A36B0593E36B05442B
:10FF1000CDE906376A46082369466846FFF7A0FF21
:10FF2000082305446A4631463046FFF799FF236AA5
:10FF30000093636A0193A36A0293A36B0693E36B36
:10FF40000793054408236A4631463046CDE90477D5
:10FF50000397FFF785FF636A0093A36AA26B01937F
:10FF6000E36A02930492636BE26B0393CDE905238A
:10FF7000236A0793054408236A4631463046FFF753
:10FF80006FFFE36A0093236B0193636B0293236A11
:10FF90000693A36A0793054408236A463146304610
:10FFA000CDE904770397FFF72BFF236B0093636B77
:10FFB0000193A36B0293E36B0393636A0693E36A73
:10FFC00007932D1A08236A4631463046CDE9047757
:10FFD000FFF716FF636B0093A36B0193E36B029330
:10FFE000236A0393636A0493A36ACDE90537236BFD
:10FFF00007932D1A08236A4631463046FFF700FF63
:020000022000DC
:10000000A36B0093E36BCDE90137636A0393A36AA3
:100010000493E36ACDE90537636B07932D1A082330
:100020006A4631463046FFF7EBFE2D1A0D4C0FD4D1
:1000300035B9082231462046FFF795FE01280FD03A
:100040000823224631463046FFF7DAFE2D1AEFE745
:100050000823224631463046FFF702FF2D18F7D419
:1000600009B0F0BD1C3B05002DE9F04391B00F46EF
:100070001C220021804609A8FFF754FA01251C2202
:10008000002101A80895FFF74DFA394608AA11F991
:10009000046B009533461046FFF7E2FE314608A890
:1000A000FFF782FE013804B2012C07DC32466946B4
:1000B0004046FFF76DFE11B0BDE8F0833A46684652
:1000C0006946FFF720FE10AB601103EB80001FFABA
:1000D00084F909F01F0350F8202C05FA03F31342AA
:1000E00005D03B46424669466846FFF7CFFD09F119
:1000F000FF3424B2D8E770B5036813F00105064653
:10010000144605D013460A460146FFF7A9FE0546E8
:1001100021463046FFF71AFE45B104F18042013A0C
:1001200056F8223043F0004346F8223070BD70B5D7
:100130009DF910401E4623460546FFF761FE38B183
:100140002346324629462846BDE87040FFF788BE60
:1001500070BD2DE9F0438BB01446129D15F9046B68
:1001600000961F46804689462B460246214602A835
:10017000FFF7DDFF02A9129A0846FFF7C4FD129BA4
:1001800002AA41464046FFF781FD129B02AA214682
:100190002046FFF77BFD2B464A46394638460096F7
:1001A000FFF7C5FF129A394602A8FFF7ACFD02A976
:1001B0002B46424608460096FFF7B9FF02A92B4698
:1001C000224608460096FFF7B2FF2B4642462146DC
:1001D00020460096FFF7ABFF129B22464946484651
:1001E000FFF754FD2B4602AA414620460096FFF732
:1001F0009EFF129B224639463846FFF747FD2B46A5
:100200004A46394638460096FFF791FF324602A922
:100210002046FFF7BDFD0BB0BDE8F08370B59DF93A
:1002200010401E4623460546FFF71AFE30B9224607
:1002300029463046FFF797FD012807D0234632466E
:1002400029462846BDE87040FFF7DABD70BD2DE9AC
:10025000F0439BB01646229C14F9045B0095984627
:100260000746894623460246314612A8FFF75FFF3C
:1002700012A9229A0846FFF746FD229B12AA394688
:100280003846FFF703FD229B12AA31463046FFF79E
:10029000FDFC23464A46414612A80095FFF7BEFFE3
:1002A00023464A46414640460095FFF740FF234615
:1002B0003A4631460AA80095FFF739FF229B0AAA61
:1002C00049464846FFF7E2FC2346324639460AA82B
:1002D0000095FFF7A3FF229A41463046FFF713FD32
:1002E00023460AAA314630460095FFF720FF2346F1
:1002F0003246394602A80095FFF719FF229B02AA51
:1003000041464046FFF7C2FC23464A464146404626
:100310000095FFF70CFF229A12A902A8FFF7F3FC41
:1003200002A923460AAA08460095FFF700FF2346C4
:100330003A4602A90AA80095FFF7F9FE0AA9229BEE
:1003400012AA0846FFF7A2FC23464A460AA94846D5
:100350000095FFF7ECFE2A4602A93846FFF718FD84
:100360001BB0BDE8F0832DE9F04115468AB0044684
:1003700088461C22002103A8FFF7D4F82E1D95F90A
:10038000007003232A46414620460293FFF7BBFC38
:10039000334602AA214620460097FFF7C8FE2B46A7
:1003A000424621462046FFF771FC0097334605F18F
:1003B000840221462046FFF731FF0AB0BDE8F081F4
:1003C0000C4B1B78062B10D10B4B1B681A070CD15A
:1003D0000A4B186800F0F003302B08D000F0E00062
:1003E000A0F1400358425841704700207047012057
:1003F000704700BFE00F00F0E40F00F0E80F00F0DE
:10040000094B1B78062B0CD1084B1B681A0708D127
:10041000074B186800F0F000A0F130035842584133
:1004200070470020704700BFE00F00F0E40F00F0BD
:10043000E80F00F010B50C494A6E042A044611D0AA
:100440000B6E1344032B02F101024A6688BF043B82
:10045000182202FB031318460021FFF763F82060FF
:10046000012010BD0020FCE7F4A4002010B50446D4
:1004700086B01422002101A8FFF754F86088ADF877
:100480000800FFF759F92378ADF80600092B0CD8BE
:10049000DFE803F005051014161B1D0E1F210723AE
:1004A0008DF8043008238DF80C3001A8FFF7AAF965
:1004B00006B010BD0D238DF80430F6E70E23FAE7E1
:1004C00007238DF804300523EDE70F23F3E710230E
:1004D000F1E70523EFE706238DF80430A3680393C3
:1004E000A388ADF80630E0E708B5134644F20102F0
:1004F000904203BF5A6819889868002218F0EEF8F5
:1005000030B50B4B1B68012293F850100D338A4213
:1005100004DB405CB0FA80F0400930BD13F8014BB9
:10052000855CA54201D10132F1E70020F5E700BF6B
:10053000C09F002003681A78302A27D15A1C026015
:100540005A7802F0DF024F2A03D1023303600820F9
:100550007047582A03D10233036010207047422AA3
:1005600004D0082013F8012F22B97047023303602A
:10057000022070472E2A07D0A2F13801012903D9A1
:10058000303A092AEED970470A20EBE70A20704773
:1005900070B5244B0022C3F80025234A516831B1BD
:1005A0002249C3F8081322490420C1F88000D3F877
:1005B0000C55D3F81445D3F80815D3F810054FF0AF
:1005C000FF36B542C3F8146518BF05F5E075C3F8EA
:1005D0000C65C3F80865C3F810651EBF4FF0A04353
:1005E000022643F82560651C1FBF4FF0A04304F5A9
:1005F000E074022543F82450441C1FBF00F5E0704E
:100600004FF0A043022443F820404B1C1FBF4FF083
:10061000A04301F5E071022043F821000023D376C6
:10062000536070BD0020004080A0002084020200C2
:1006300000E100E070B58AB00C46014668461E46EF
:1006400026F04BF90022214605A826F046F9684617
:1006500026F031F8044605A826F02DF88442054618
:100660000DD003982BF062FD08982BF05FFD002C55
:1006700001DB002D00DA56B9601B0AB070BD002CFA
:1006800007DA03982BF052FD08982BF04FFD00205D
:10069000F3E7684625F0C7FD05A825F0C4FDD6E7B9
:1006A000044A138A9BB223F0410343F040031382B0
:1006B000704700BF602D00202DE9F04F85B08A46BD
:1006C0000390039C2578284625F004FC0746C8B90A
:1006D0002D2D1AD10134012303940193DDF80CB0C0
:1006E000BAF1000F01D0CAF800B003A8FFF722FF4B
:1006F0008046002835D1624D00242046294605B0A9
:10070000BDE8F08F01340394DBE72B2D04BF0134E7
:1007100003940190E2E71846029325F0A9FBB0F19B
:100720000009029B20DBC8451EDD404632F010FC6C
:1007300022462B4632F076FC04460D46484632F0FF
:1007400007FC22462B4632F0B7FA013604460D4626
:100750000396039E3378002BDDD1B8F10A0F37D111
:1007600013E000240025F4E7B8F10A0F30D12E2B56
:100770000BD10FF20419D9E9008901360396039EC3
:1007800030783038C3B2092B39D9039B1A7802F07C
:10079000DF02452A1CD15A1C03925A782D2A01D017
:1007A0002B2A05D12D3A574203F1020357410393F7
:1007B0004FF000080A20039A1378303BD9B2092978
:1007C00036D9002F39D12F4F0026B8F1000F46D16E
:1007D000039BBAF1000F01D0CAF800309B458AD0C4
:1007E0009BF800202E2A03D10BF1010B5B4582D030
:1007F000019B002B81D005F100431D467DE732F0BF
:10080000A7FB42464B4632F00DFC02460B46204603
:10081000294632F051FA002204460D464046494628
:10082000184B32F029FD0136804689460396A6E72B
:10083000013200FB08380392BDE7124FC8F10008EF
:100840000026B8F1000FC3D02046294632463B4669
:1008500032F012FD08F1010804460D46F1E720468A
:10086000294632463B4632F0DDFB08F1FF380446AC
:100870000D46AAE7AFF300809A9999999999B93FE3
:100880000000F87F0000244070B586B014460E4684
:100890000022014601A826F020F82546DDE90123C3
:1008A0009A4204D304982BF041FC601B04E02DB95C
:1008B00004982BF03BFC204606B070BD01A825F043
:1008C00005FF013D06F8010BE8E710B586B00A46C2
:1008D000014601A826F001F80023DDE9011291424A
:1008E00003F1010401D201330AD104982BF01EFC5C
:1008F000202022F003FB14F1FF340AD206B010BD11
:1009000001A825F0E3FE0A28EFD022F0F7FA2346EB
:10091000E3E70820EDE7000070B50D2021F080FB33
:100920000028264B46DB264C1871A17D01229A70C7
:1009300000293DD1234DA18204334FF48E71284606
:10094000A360A275FFF762F92146AA60FFF78DF94F
:10095000636893B92646A27DA38A9A420ED8A38AD9
:100960009BB2B3F5807F1BD0164BD3F81C21002A15
:10097000FBD00122DA600023A37570BDD5F81C31CD
:1009800023B9A38A9BB2B3F5807FF7D1A38A9BB228
:10099000B3F5807FE0D031462846FFF766F9DAE705
:1009A0000023A3750F210848BDE8704026F06CBAFB
:1009B0001121F8E700229A70DFE700BFC5A60020EA
:1009C00080A00020002000407A3D050030B58BB0AB
:1009D0004FF4D8230193054608B100230360202279
:1009E000002102A8FEF79EFD002202A94FF4D820A4
:1009F0002EF0E0FBD0B10024029B039A23F07F434A
:100A0000033323F00303203352B11C44032202A911
:100A100001A82EF057FC0028EED120460BB030BDC7
:100A2000002DF3D02A6813442B60EFE70446F4E767
:100A30002DE9F04F202291B000244FF4D8258246B2
:100A400088460DEB02002146CDE904540694FEF7DA
:100A500069FD012208A9284607952EF0ABFBA8B92D
:100A600005AB019306AB52464FF4EC21009304A86A
:100A700043462EF069FE049801382EF013FC0490D2
:100A80002EF0A6FE012011B0BDE8F08F099B002BCF
:100A90005DD0049E069BDDF81C901E444E4523D07D
:100AA000089B23F07F4320334B4401250D270293FD
:100AB0006A1E3E497A4302EB010B584603922AF024
:100AC00039FCA8B1DBF80010894508D8029B99428F
:100AD00005D2A6EB09030B44039A34495350013560
:100AE00040F6CA039D42E3D920230DEB030214E034
:100AF00058462AF029FC0028F1D0DBF800300C33EE
:100B0000B3FBF7F31D44EAE712F8011B0AF80410DF
:100B10000134B4FBF8F108FB114413F1FF33F3D2B5
:100B2000069B089E20330693079B26F07F460336DC
:100B300003F1200905AB26F00306019306AF0097E9
:100B400043465246494604A82EF0FEFD2EB9012226
:100B500008A907A82EF0B6FB81E7069B059AA8EB2B
:100B60000300A8EB0405854228BF0546A24203D92D
:100B7000121B954228BF15460293ADB1B54228BF5E
:100B8000354649460AEB04002A4632F05FFF029BD5
:100B90002C442B440693B4FBF8F308FB134405AB39
:100BA000761BA9440193CAE728466CE77C2D0020F8
:100BB00030B58BB04FF4D8242022002102A8019434
:100BC000FEF7B0FC002202A920462EF00DFB70B10A
:100BD000032202A901A8DDE901542EF073FB0028CD
:100BE000F6D124F07F4423352C4424F00304C4F5CB
:100BF000EC200BB030BD0000F0B40023124D0D27E7
:100C00001C4640F6CA0607FB03519A1CC87ACC72F0
:100C1000087B0C73C2F30B004A79087122F00F02B3
:100C2000013342EA1022B3424A71ECD147F2392330
:100C3000064AEC54537823F00F035370044B0122FF
:100C40001A80F0BC2AF0C6BB7C2D0020B59F002086
:100C50007A2D0020F8B50646437A807A000150EAE2
:100C600013100C4619D02AF09BF907462CF06AFBAA
:100C7000451C38462BF05AFA28462BF043F92146FA
:100C80002CF044F8044638B1014630462CF0D0FB35
:100C900020462BF04BFA681CF8BD0125ECE700005C
:100CA00038B5074C25780023EDB20246194623706B
:100CB0002DF068FE25700348BDE8384021F0BCBA2D
:100CC000782D0020818405002DE9F843394F037900
:100CD0001C2202FB03720646506820B132684FF4B2
:100CE0000174C2F808431C2202FB0373DA7D52B17F
:100CF0001A7E002A41D020B133684FF40172C3F844
:100D00000423112037E00120D875D9605A761A766D
:100D100035791C2303FB05739B7E1BB912B9304642
:100D2000FEF77CFF4FF01C0808FB05783068D8F808
:100D30000430002B35D14FF4A271FEF767FFC5EBED
:100D4000C50907EB89093068D0F82431D0F80821AB
:100D5000D0F84441A2B90CB9002BF4D01C2202FBFC
:100D600005750022EA750BBB14BBA97E336801220E
:100D7000A9B11A600020BDE8F88319610122C6E715
:100D8000002BEBD1002CE9D14946FEF757FF98F82C
:100D9000193098F817209A42D5D82346DEE75A60D2
:100DA000E8E74FF40173C0F80433E3E70320E2E718
:100DB0000F20E0E780A000200A490B4808B5FFF7A4
:100DC00083FF014610B1094826F05EF8084906483D
:100DD000FFF77AFF014620B10648BDE8084026F03B
:100DE00053B808BDC5A60020103B0500343D0500E2
:100DF000C6A60020573D050038B5002205462CF058
:100E0000FBFC044650B100231A460146284622F056
:100E10004BFE2046BDE838402BF088B938BD0000B5
:100E2000F7B500220191274906462CF047FC0546FC
:100E3000C8B1014601AB0122304622F035FE58B957
:100E4000214826F041F8214A1E491378304643F0E4
:100E5000040313702DF0C4F828462BF067F9012421
:100E6000204603B0F0BD0246194930462CF0C4FCC0
:100E700007462AF02EFB044628B9019A1449304649
:100E80002CF076FCEBE738462BF0B7FD06460198D0
:100E90002BF0B3FD3044B0F5007F05D90B4A137831
:100EA00043F0020313702C46B6F5007F06D2C6F558
:100EB00000730022019938462BF098FC38462BF03D
:100EC00035F9CDE7633C05006B3C0500792D00202A
:100ED0009F3C050070B5EFF3108672B60D4A94681A
:100EE0000123A4B993600C4B0C4DD3F8801029401A
:100EF0001160C3F88050D3F8841051604FF0FF3276
:100F0000C3F88420047006B962B6002070BD037077
:100F1000F9E700BF90A6002000E100E0FC06FFBC5E
:100F2000437882781B01120202F4E06203F030037E
:100F30001343027802F003021343C278120302F44F
:100F4000805213430279120402F4E02213434279DF
:100F5000120502F4801213438279120602F08072A5
:100F60001343054AC2F81835C379017AC2F814153B
:100F7000C2F81035704700BF0070004010B588B04F
:100F800012788DF80C200021FF2202918DF80D209F
:100F900001214FF6FF72104C01908DF81C10ADF836
:100FA0000E208DF8103020F0E9FC70B124F03AFDED
:100FB00058B914F1FF34F6D20849042026F0A4F8F9
:100FC00001A820F0EBFC08B010BD002CF4D024F0F8
:100FD00029FD0028F0D1F3E780841E004A3C05007B
:100FE00038B50B4C0B4D2B785BB124F01BFD40B991
:100FF00014F1FF34F7D208490420BDE8384026F048
:1010000083B8002CF7D024F00DFD0028F3D138BDB3
:1010100080841E00B0A60020EC3B0500F7B5354FDC
:10102000354C7E797601A31905465A7E002A5FD198
:10103000A2590AB101225A7695E80F0004EB060E78
:101040000EF1080C8CE80F0006F1180323445A79BE
:1010500022F003025A719EF81A20FF2A1FBF0123B3
:1010600093404FF0A042C2F80C352A6822B102F03A
:101070006043B3F1005F06D1AB6853B103F0604346
:10108000B3F1005F05D0344400236376102003B031
:10109000F0BD3B682979C3F84425C3F848152A7B7D
:1010A000A968C3F834150020C3F83825C3F818011F
:1010B000D3F818210192019AC3F850050122C3F810
:1010C00040051A61A2597AB9D3F81821002AFBD039
:1010D0003444A27EFF2A05D0012393404FF0A04262
:1010E000C2F808350020D2E74022C3F80423CEE737
:1010F0001120CCE7B42C0020C4A00020F0B5154688
:1011000085B01C4E07460C46FFF76AFF0123FF2DF2
:1011100033702B4628BFFF231FB3FA1816490A6005
:101120000CB3E218154900970A60154A0294002C86
:10113000A5EB0305DBB21560684614BF1A46002212
:101140008DF80C208DF80430FFF768FF024660B17F
:10115000002404200B49347025F0D6FF204605B04A
:10116000F0BD3A46DAE72246DCE7FFF739FF012017
:10117000F5E700BFB0A60020B4A60020ACA6002072
:10118000A4A60020D93B050013B51A4B1B780446D2
:1011900063B3FFF725FF184B1B68002201200421D1
:1011A000C3F80025C3F80005C3F80813C3F80821E5
:1011B000D3F80811009100991049E4B20870C3F8FF
:1011C0001C45D3F808010028FBD0C3F80821D3F848
:1011D000080101900198D3F818050A70C3F800259A
:1011E0000722C0B2C3F8002502B010BD4FF0FF3097
:1011F000FAE700BFA8A60020B42C0020B0A600206B
:1012000037B50B015BB249B2044643EA01008DF8E1
:1012100004001A4D50B20343120152B28DF805304A
:101220002B78114302438DF806108DF8072013B375
:1012300002AB03EB941302AA13F8040CC4F30113DA
:10124000134413F8043C43EA002017F0ADFC2B785C
:101250008BB102AAC4F3810304F0030413441444C1
:1012600013F8040C14F8043C43EA002003B0BDE872
:10127000304017F099BC03B030BD00BFA8A60020D5
:10128000C30914BF13020B0210F0400F70B50646DD
:1012900014BF10460846184314460D46FFF774FF66
:1012A000B1064CBF23022B0216F0100F14BF2046CC
:1012B00028461843FFF768FF32074CBF23022B0272
:1012C00016F0040F14BF204628461843FFF75CFFB2
:1012D000B3074CBF2002280216F0010F08BF2C46AE
:1012E0002043BDE87040FFF74FBF000020292DE9E3
:1012F000F0470BD9244A254E2139C9B200231446A0
:10130000DFB2B94205D814F801C0B6BB4008BDE849
:10131000F08712F8017B01333E44F1E7745CC82C7E
:101320001ED81EF80450DFF86C90194B4FF00008DF
:101330005FFA88FA54450DD803EB0509994511D198
:1013400001316145EADB0232504320F07040073042
:101350000009DCE719F801AB08F101085344E7E79D
:101360000023E9E713F8018BB8FBF7F407FB1484BB
:10137000E4B2A242B8BF2246E0E700210A46DFF805
:1013800014E00D27DDE700BF9B3D05007A3E050018
:101390009E400500D53F050010B5074A002332F8EE
:1013A000024B8C4203D1184100F0010010BD013303
:1013B000082BF4D10020F9E7C89F0020F0B5224B9C
:1013C0009F7C1C4600221D46D6B2B7420ED895F827
:1013D00078701D4C0022D6B2B74216D895F8DE5070
:1013E0000022D4B2A54220D800200DE0B4F814C0E9
:1013F000844502F1010204F10A04E5D142F64D23CD
:1014000001200B808870CE70F0BDB4F87AC06045C2
:1014100002F1010204F10A04DDD142F64D230B80F2
:1014200002238B70CE700120EEE7B3F8E060B0428B
:1014300002F1010203F10A03D3D142F64D230B80DE
:1014400003238B70CC70EEE748A2002010B50C4C43
:10145000226886B0034682B104208DF80400086833
:10146000D989ADF80C10123333F8021C0290ADF894
:101470000E10049301A92046904706B010BD00BF8E
:1014800048A200207FB54B89022B0FD1094A13686F
:1014900063B1097B0068029011F0010F14BF0221B3
:1014A00003218DF80410104601A9984707B05DF894
:1014B00004FB00BF48A2002070B50D4D002435F894
:1014C000026B964210D10122A240D2B2D543EDB2B6
:1014D000014410F8014B2BB11443884200F8014C31
:1014E000F7D170BD2C40F8E70134082CE7D1F8E7BC
:1014F000C89F002070B50023084C1A4641FA02F537
:10150000ED0706D504EB420600EB4305B688AE8036
:1015100001330132082AF1D1036070BDC49F00205D
:1015200010B586B004460022684615F0D1F8204672
:10153000009915F0FBF9204606B010BD38B501231F
:101540000B7004460D4629F0A2FE88B100220B491B
:1015500020462CF051F910B12CF0C4FE2870204622
:10156000002207492CF048F9BDE838402CF07EBC39
:101570002046BDE838402BF0E5BE00BFCC3B05005F
:10158000D13B05002DE9F04F2DED028B8DB0436A64
:10159000059390ED048B1F02836A07671E0246675E
:1015A000B0EE480AF0EE680A044606932FF0B0FB4E
:1015B00059EC108BB0EE480AF0EE680A2FF098FC58
:1015C00094ED067B404653EC172B49465BEC10AB81
:1015D0008DED007B31F050FE0022614B31F022FD99
:1015E0000022604B31F068FB31F0CCFFDDE90023D5
:1015F0000790A0675946504631F03EFE0022584BF6
:1016000031F010FD0022574B31F056FB31F0BAFF9C
:10161000E0670546059831F09BFC29F00043CDE9D1
:1016200008010698CDF80880039331F091FCDDE9BC
:101630000223CDE90A01DDE9080131F0F3FCD046CF
:101640002BF0004942468B464B468246DDE90A01B3
:1016500031F0E8FC02460B465046594631F02CFB6F
:10166000DDE9002331F0DEFC00223E4B31F024FBAB
:1016700031F088FF42464B468346DDE9080131F0F0
:10168000D1FCDDE90A2380468946DDE9020131F01B
:10169000C9FC02460B464046494631F00DFBDDE9E8
:1016A000002331F0BFFC2F4B002231F005FB31F05D
:1016B00069FF94F820305BB1226863680BEBDB7143
:1016C000A2EB6102226000EBD072A3EB62036360C5
:1016D0002368059A5B44A36063680344E360079B47
:1016E0000BFB03F3013300FB053303EBD373D20190
:1016F000A2EB6303C4F88030079B58430130069B7C
:101700000BFB150505EBD575D80194F82130A0EB3E
:101710006505C4F884503BB90DB0BDEC028BBDE843
:10172000F08F3B44C4F88030D4F88030002BF8DBD5
:10173000D4F880309F420BDDD4F88430002B0BDBD3
:10174000D4F884309E42E7DC9B1BC4F88430F7E772
:10175000DB1BC4F88030EBE73344C4F88430EBE79C
:10176000000070400000E03F1F4B204A1B6800BF94
:1017700000BF00BF00BF00BF00BF00BF00BF93425B
:101780002FD000BF00BF00BF00BF00BF00BF00BF21
:1017900000BF00BF00BF00BF00BF00BF00BF00BF51
:1017A00000BF00BF00BF00BF00BF00BF00BF00BF41
:1017B00000BF00BF00BF00BF00BF00BF00BF00BF31
:1017C00000BF00BF00BF00BF00BF00BF00BF00BF21
:1017D00000BF00BF00BF00BF00BF00BF00BF00BF11
:1017E00000BF0138C3D17047A42C00200024F400AE
:1017F00008B1FFF7B9BF7047084B5A6E013A5A66F5
:1018000022B907490A7822F002020A701A6E0132E0
:10181000042A08BF00221A66704700BFF4A4002003
:1018200039A2002030B5044685B00D4610220021B3
:101830006846FDF777FE237A012B0AD0022B0ED0E3
:1018400063680193236829469B686846984705B0FA
:1018500030BD23690293A38AADF80C30F0E7012371
:10186000A2898DF80030E389ADF80A20D31AADF8CB
:101870000830E5E728DF704729DF704738B51C4B93
:101880005A6E19465AB31C6E182202FB04331A7A98
:10189000012A07D0022A23D018460921BDE8384082
:1018A000FFF7C0BF1825D88A9A8A05FB0414D4E92B
:1018B0000314121AB2F5806F4FEA80000144B4BFDE
:1018C00092B24FF480622044FFF7D6FF11280BD16B
:1018D000084A137823F0020343F00403137038BD61
:1018E0009889FFF7C7FFF1E70028F8D0D4E700BFD9
:1018F000F4A4002039A20020054A137813F0060F43
:1019000004D143F002031370FFF7B8BF704700BF64
:1019100039A200202DE9F3411F4B1B781746DA0747
:10192000064688462BD51D4D1D4B9D4229D31D4B88
:101930009D4226D239B330B341EA00039B0724D13C
:101940002B68984223D36A6800EB87039A421ED320
:10195000FFB101A8FEF76EFD78B1019B0024C3E939
:101960000054019B01221A72C3E903869F82FFF78C
:10197000C3FF204602B0BDE8F0810720FAE701204E
:10198000F8E70220F6E70320F4E70620F2E7052057
:10199000F0E70420EEE700BF39A20020282D002048
:1019A000282D0020382D002038B5074B074A5968EC
:1019B000948810684A880332032592B200EB8400B1
:1019C0001D70FFF7A7FF38BD3CA2002098A500209E
:1019D00010B501220C460649FFF79CFF28B90549BE
:1019E00001EB041101238B7310BD0E20FCE700BF37
:1019F000B83C050054A4002008B502220149FFF7B5
:101A000089FF08BDBC3C050008B5034B03491868B5
:101A10000222FFF77FFF08BD98A50020C43C050007
:101A200073B51B4B1B78DB0705462BD5194E1A4B9C
:101A30009E4229D3194B9E4226D238B3C0F30B04E1
:101A4000D4B93368984219D3726800F580539A422A
:101A500014D301A8FEF7EEFC90B1019BC3E900642A
:101A6000019B02221A722D0B01229D811A82FFF71F
:101A700043FF204602B070BD0620FBE70520F9E7D2
:101A80000720F7E70120F5E70220F3E70320F1E75D
:101A900039A20020282D0020282D0020382D0020DC
:101AA00010B50B4C0B4B628803EB02139A892AB9D1
:101AB0005868FFF7B5FF0423237010BD052323707A
:101AC000054B022218689A80FFF7AAFFF5E700BFCE
:101AD0003CA2002054A4002098A5002008B5074B84
:101AE000191D5888FDF776FD18B1BDE80840FFF7CD
:101AF0005BBFBDE80840FFF7D3BF00BF3CA200209A
:101B000010DF7047002208B5114616F0E7FD00000F
:101B10002DE9F347254B1B681BB1984730B3FFF7FE
:101B2000F1FF234B1B7803F0FF07FBB1214D224E41
:101B30002C68DFF88C90B4FA84F46409B0463378EA
:101B4000A3B901A8FDF72AFD052812D00028E6D187
:101B5000019B0BB9FDF7FEFE184B1B680BB10198FA
:101B600098474CB10124EAE7002CFBD002B0BDE855
:101B7000F087002CFAD13C46DFF848A098F80030F6
:101B8000002BF3D1B9F80030ADF80430DAF80030AA
:101B900001A91846FDF700FD0528E5D00028BED1B3
:101BA0002A6818469047002CE8D1C8E728A20020F0
:101BB00094A50020FC9F002095A50020A0A5002052
:101BC000F89F002088A6002010B5084B9A685AB1EB
:101BD00050B9EFF3108172B6054A1C6814605C6856
:101BE0005460986001B962B6002010BD90A6002034
:101BF00000E100E02DE9F3411D4F7B6806460D46EC
:101C00009BB304292FD943697BB3437C0024012B68
:101C10000DF107000CBF8846A0468DF80740FFF77E
:101C200059F90DF10600FDF763FDD0B101230370F2
:101C3000104B4660D3F80435C0E90484C0E902358E
:101C40009DF806307B709DF80700FFF7BDFF24B9B3
:101C5000094B4FF48012C3F80021204602B0BDE8C2
:101C6000F0810424EFE70724F7E70824F5E700BF35
:101C7000D0A300200010014000E100E02DE9F34175
:101C8000CE0801F007044FF0010808FA04F4855D5E
:101C9000E4B22540074613D10DF107008DF8075037
:101CA000FFF718F9BB5D9DF807001C4202BF1C43FB
:101CB000BC554546FFF788FF284602B0BDE8F081D5
:101CC0000025F9E72DE9F3478146002701261FFA91
:101CD00087F84FEAD80A08F0070406FA04F419F85E
:101CE0000A50E4B2254008D00137B7F5807FEED125
:101CF000B846404602B0BDE8F0870DF107008DF808
:101D00000750FFF7E7F819F80A309DF807001C4262
:101D100002BF1C4309F80A400125FFF755FF002DBB
:101D2000E2D0E6E773B50546B8B1C1F3C70401F0E8
:101D3000070301269E40035D33420ED000230DF1C0
:101D400007008DF80730FFF7C5F82B5D9DF80700F9
:101D500023EA06062E55FFF737FF02B070BD0000DC
:101D600038B50A4B1A687AB15D686DB1FF280BD09F
:101D700084B221462846FDF75FFD28B1214628465A
:101D8000BDE83840FFF7CEBF38BD00BFD8A5002062
:101D90002DE9F74F9846531E072B81460F461546EF
:101DA00000F2BB80FF2800F2B88001465E48FDF7D4
:101DB00043FD0646002800F0B08039464846FDF74E
:101DC000FBFC044600283ED0C3689D4247D805D29C
:101DD0005FFA85F9E368207C994543D394F8109025
:101DE000B9F1FF0F40F09780504B1A689B46002ACC
:101DF00041D14FF6FF732380A3700023C4E9013360
:101E0000E360238A03F4784343F0FF032382112025
:101E100084E0237C1844C0B2FFF7A2FFE3685FFAB6
:101E20008AF083420AF1010AF3D84FF6FF73238048
:101E3000A3700023C4E90133E360238A03F47843E9
:101E400043F0FF032382FF214FF6FF70FDF7B4FC40
:101E500004460028DBD0A0F800908770BEE74FF062
:101E6000000ADBE74844C0B209F10109FFF778FF37
:101E70005FFA89F9AEE75B68002BBAD00023DBF884
:101E800008205FFA83FA924502D34FF0FF0912E06F
:101E9000DBF8040060B351460193FFF7EFFE019BAE
:101EA00030B3B9F1FF0F08BFD146AAEB090A0AF116
:101EB000010AAA4521D1B9F1FF0F84F8109098D0FA
:101EC000E560207CFDF7C8FC58B305EB85052D01C6
:101ED000ADB2AD0888F80270C8F80400A8F8005048
:101EE00026B1082F02D1AD00063D8580002015E007
:101EF000B9F1FF0F0CD14FF0FF090133BFE748469E
:101F0000019309F10109FFF72BFF019B5FFA89F9A2
:101F1000D145F4D3EFE70026D2E7072003B0BDE8B0
:101F2000F08F0320FAE700BFACA40020D8A5002062
:101F300038B504460025E368AB420ED84FF6FF7370
:101F40002380A3700023C4E90133E360238A03F4F0
:101F5000784343F0FF03238238BD207C2844C0B27D
:101F6000FFF7FEFE0135E6E737B5FDF725FC054630
:101F7000A0B144682CB10A4B01941B789B0706D48E
:101F800003242846FFF7D4FF204603B030BD01A844
:101F9000FDF706FB04460028F3D0F1E70524F3E73C
:101FA00038A20020FF2810B5044609D8014605488C
:101FB000FFF7B8FE21460448BDE81040FFF7B2BE67
:101FC00010BD00BFACA40020CCA4002013B50DF1BF
:101FD00006010446FDF726FB70B1BDF80620084B4C
:101FE00003EB02139A894AB1A17A39B1013A002070
:101FF0009A81A07202B010BD0A20FBE70620F9E723
:1020000054A4002037B50D460DF106010446FDF736
:1020100009FB88B1BDF80620084B616803EB021389
:1020200000209A8901329A81296063680C336B60C1
:102030000123A37203B030BD0A20FBE754A40020A3
:102040002DE9F043DFF88480D8F874E0BEF1030F87
:102050000F46944635D81C4E756CC1F108039D425D
:102060002FD8D8F8704074441C2304F00304814630
:1020700003FB0484B9E80F000FC499E807000EF1D0
:10208000010384E80700C8F87430C7B1336C2B44EF
:1020900003F0070306EBC303002206F138040CEB40
:1020A000C20103C9A34202F1010283E8030014BF85
:1020B0000833054B9742F2D1736C1F4477640120BB
:1020C00000E00020BDE8F08308A10020D8A3002094
:1020D0002DE9F0411C46184B1B789B0706460F461E
:1020E000154627D5DFF85880A3880BB10A201FE0DA
:1020F00098F800302BB92146A088FDF76BFA20B97B
:102100002060A3880133A380EEE723681EB199887D
:1021100032889142EFD11FB119883A889142EAD1B1
:102120009B682B6023686B60044B1B892B8100200C
:10213000BDE8F0810220FBE738A200203CA200208D
:1021400054A4002030B587B04CF2070305460C4676
:10215000ADF8043003AA0F4B01A90020FFF7B8FF28
:1021600010B1002007B030BD01A903A8FFF74AFF56
:102170000028F6D10723A370019B5A882280029A77
:1021800062609B8803F580432B8003A8FFF71EFF46
:102190000120E7E72CA200201FB50023A0F5804016
:1021A000A1F58041CDE90233ADF80400ADF8061089
:1021B00002AB0DF1060101A8FFF78AFF002818BF46
:1021C000052005B05DF804FB2DE9F04102230B80EA
:1021D000164B00251C6800F5805E2F4608304FF630
:1021E000FF7870450AD305B11C6002B11770BDE8D5
:1021F000F08101270EE0344601250BE00668013628
:10220000F1D086884645F4D00688002EF1D0866845
:10221000A642F0D8468806F1030C00EB8C00B1F81A
:1022200000C00CF1030C66440E80DAE7C4A3002062
:1022300070B5064D0646002455F8043B0BB13046F8
:1022400098470134082CF7D170BD00BFE4A00020EE
:102250002DE9F047AA4C266F1C2707FB06F586B030
:10226000635D013B8046052B00F22A81DFE813F015
:102270000600640064001D011D017E0130B1A14A09
:10228000137823F00103137001201FE025442B79FC
:10229000032B15D8DFE803F002072C34FFF7B4FB5B
:1022A00001232B7109E0984D2B78022B40F03C82E2
:1022B0006868FFF7A1FB00232B70002800F0F08076
:1022C000904A137823F0010313700E201C237343EC
:1022D000E218E35C0290023B012B00F232818B4B4F
:1022E000907D196C5A6C0144121A19645A6428E1E1
:1022F000874F3868FFF794FB0223BB800023D0E7A9
:10230000834FDFF804823868FFF776FB814BD7F8FC
:1023100000E05B88B7F804C01B0108EB03025168BA
:10232000A2F808C0C2F804E00222BA800022396094
:1023300008F803202A71C0E707FB0647724BB7F87D
:1023400012A04FEA0A1A03EB0A029946118960B1FA
:10235000FB8803F103088844C3F57F435189A2F841
:102360000880FD330B4453818EE7536803EB8108EB
:102370003B7C062B00F29780DFE803F02D733C4D89
:102380001F84040041F61D501C2303FB0643D14467
:10239000DB88B9F80810DA1C0A44A9F80820C3F54C
:1023A0007F43B9F80A20FD331344A9F80A3041F6F7
:1023B0001D53984200F0C38088E7574857490023CF
:1023C00043601C2303FB06439B690360FDF72AF966
:1023D000002800F04C81291D012221444046FFF7CE
:1023E00099FA1C2303FB064302221A74002857D0D3
:1023F0000E20C9E705F10C010122214408F1080073
:10240000FFF788FA1C2303FB06439A7D002A14BFBA
:1024100003220122E9E73D4B5A6C002A00F08C812F
:10242000196C1C2505FB0645481C00F0070003EB52
:10243000C1071864A88A53F83110013A5A6408EBAE
:102440008000BA88FFF766FAAB8ABA881344AB8279
:10245000AB7D013BDBB2AB75002BC7D101232B74E5
:10246000C4E705F108010122214408F10400FFF747
:1024700051FA1C237343E25C032A0CBF0522062297
:102480002344B2E7254B1988234B5868FFF7A0FA7D
:102490001C2303FB064306221A7400287FF474AF42
:1024A00006B0BDE8F0870F206EE700287FF4ECAEA1
:1024B00007FB06473B79012B32D01BB1022B3ED0E4
:1024C0000F2003E7CDE90200FB6801930DF1020143
:1024D00001A8FDF7A7F880B10298BDF80210838823
:1024E000FB8003883B81FFF773FA1C2303FB064341
:1024F00002221A710028D3D059E70A20F5E700BF5D
:10250000D8A3002038A2002054A4002008A1002055
:1025100098A500203CA20020542D00209CA600205D
:10252000864FA81D3B4601AA41462044FFF7D0FD37
:10253000B8B9B9880298FFF74BFA0A28DAD1002314
:1025400002931C2303FB06F2A25C013A052A00F267
:10255000B580DFE812F08E009200A000CB00D5001D
:10256000E1000A28C7E90088E9D020E700287FF4C5
:102570008BAE734BDA7AAAB1D8721A78013A062A6E
:102580009ED801A151F822F039260200332602001C
:10259000492602004F260200C124020055260200EF
:1025A000652602001A78072AE7D801A151F822F01F
:1025B000D12502007B2502007B250200ED250200CB
:1025C000012602001F2602001F260200E925020044
:1025D0001A8901321A8100225A80DA72594A127815
:1025E000B2FA82F252099A72012207E056495868FB
:1025F0008A884088033202448A8002221A70BCE72B
:102600005D88504A504902EB0512086855685060D1
:102610008888108102228A800D600622EEE7072258
:10262000ECE7484900229A728A8942B9897B31B124
:102630005A80FFF753FA5DE79A7A002AF1D1002217
:102640001A705A805A607AE7FFF7AEF952E7FFF73F
:1026500027FA4FE75A883B4B03EB02135868FFF702
:10266000CBF947E700225A60FFF7CEF942E70A208C
:102670002CE600238DF8043020E003FB0643012202
:102680008DF804201A89ADF810209A88ADF8122030
:10269000DB68039312E003FB064302228DF804205B
:1026A0001A89ADF810209A88ADF81220DA681B7CE0
:1026B00003929A1F534253418DF8143001A8FFF73B
:1026C000B7FD206F1C22002102FB0040FCF72AFF0F
:1026D000636F1BB3226F013202F00302013B2267DA
:1026E0006367DBB10020FFF7B3FDD9E603FB0643C8
:1026F00003228DF80420DA88ADF810201A89C5E786
:1027000003FB06430422DB88ADF8103000238DF86C
:102710000420ADF81230D1E70523ABE70B4A13785C
:1027200023F004031370BBE6084A137843F0020356
:1027300023F00103137002E71368FFDEBCA600203C
:102740003CA2002054A4002098A5002038A200201C
:102750000846FFF77DBD0000054A137813F004001A
:1027600004D143F004031370FFF772BD704700BF3C
:1027700038A20020F0B51C463D4B1B789E0789B05F
:1027800007460D466FD509884FF6FF7399426CD006
:102790006B88002B69D06968B5F808C000239C4598
:1027A00003D8BAB9164604310AE051F8330080075D
:1027B00057D10133F3E731F83200304486B20132A9
:1027C0009445F8D80DF102013046FCF773FF28B1AB
:1027D00009B0F0BD13885688ADF8023000238DF89B
:1027E0001430BDF80230ADF816300323ADF81830C0
:1027F000204B8DF804401A6829898DF81A1001328F
:102800001A602B88ADF80C30032C6B88ADF80830BB
:1028100004BF04238DF81430049208BF3B686A6833
:1028200008BF0793002401A8ADF80A60ADF80E4078
:10283000FFF706FC50B9BDF802200F4B03EB021363
:1028400058890338801B58810820C1E7049B3B60EE
:102850000A4B7C601B89BC723B81FFF77DFF2046E1
:10286000B6E70320B4E70220B2E70420B0E700BFD8
:1028700038A20020C4A3002054A400203CA20020C1
:1028800030B58BB0FF28044601921D4645D88B78A1
:102890001846FCF767FF00283FD04A6802920A8872
:1028A000ADF80C20A4F58042ADF81C20A3F58042C1
:1028B000ADF81E2002AA08920122ADF82420194684
:1028C00004AA2046FFF768FC0528019A0ED10223CE
:1028D00052B907A904A8FFF74DFF07281FD010D849
:1028E000B0B103200BB030BD01AAF2E732B10E4BFC
:1028F0001B789B0702D501A8FCF752FE0323002298
:10290000E7E708280DD00E280CBF11200320E9E7C7
:10291000002DE7D0049B2B60E4E70720E2E7862048
:10292000E0E71120DEE700BF38A2002073B5154EA6
:10293000736805461BB343690BB3002404740DF19F
:1029400007008DF80740FEF7C5FA0DF10600FCF709
:10295000CFFE90B1022303709DF80630456073707E
:102960009DF80700FFF730F924B9074B4FF48012A8
:10297000C3F80021204602B070BD0424F0E708240B
:10298000F8E700BFD0A3002000E100E02DE9F84304
:102990002649274B0025C1F84051C1F84451C1F8E0
:1029A0004851C1F84C51C1F80051C1F804511B689D
:1029B000002B39D0D1F804451E49DFF88C80096816
:1029C000641A24F07F442F461A68A24217D8A41A2A
:1029D00015441A7CDE6982B1D8F800901F74D3E9DF
:1029E0000521B9F1000F06D01046C84728B1FFF7FE
:1029F00089F83346E8E708469047002EF9D10E4A99
:102A00000E4B11781B788B4205D10133DBB2022BC0
:102A100008BF002313701278094B43F82250094B6A
:102A20004FF48012C3F80021BDE8F8830010014084
:102A30008CA60020B0A50020ADA50020ACA50020EC
:102A4000A4A5002000E100E024A200200D4B0E49C7
:102A50004FF4003210B5C3F8802001244FF48033C6
:102A6000C1F848332F20C1F808334C60FEF77CFED4
:102A7000064B8C602F2000211960FEF775FE044B79
:102A8000197010BD00E100E000100140B0A5002069
:102A90008DA500202DE9F04FB64AB7491378097883
:102AA000B64D85B09942D5F80080019500F095802B
:102AB0000133DBB2022B08BF002313701278B04B36
:102AC00053F82260019A08EB060323F07F4313605A
:102AD0000127AC4BAC4A18680290AC48117890F8CA
:102AE00000904FF0000CE2465078884278D1BCF15B
:102AF000000F02D0A54981F80090002F40F0BB8064
:102B00001F6802997F1A18BF0127002019680291D7
:102B10009E49039191F800E000244FF0010800283D
:102B200040F0AD8092F80190D2F804C092F802A073
:102B30001178494540F0C1801B68029A9A4201D140
:102B4000002F44D0002B00F01281D3F80090904C5D
:102B5000019BD4F8046519688E4F751A3B7825F0EF
:102B60007F450335A3B94FF48033C4F84433C4F828
:102B70000433894B4FF400324FF00108C3F8802131
:102B80002F201A60C4F80080FEF7EEFD87F8008061
:102B9000A9452CBF4944491921F07F41C4F840158B
:102BA000D4F804359B1B23F07F43891B033321F0AA
:102BB0007F418B420BD9D4F80435C4F840352F201F
:102BC000FEF7D2FD744B4FF40032C3F80021039A94
:102BD0000023137005B0BDE8F08F0026374678E774
:102BE00001EB4104506892F802B000EBC40E0131D1
:102BF00010F834401868C9B28B4508BF0021022C78
:102C000004D0032C7FF470AF002410E0DEF804B091
:102C100004468646002C3FF467AFA34500F0C08011
:102C2000A646E469F6E780F810A0C06901240028F0
:102C3000F9D1002C3FF458AF186055E7D4F80C9048
:102C4000C4F800E0761A8C44E1691960B9F1000F0C
:102C500007D008EB0C0121F07F41C4E90119E061C4
:102C600020461C68002C3FF451AF2168B142E5D9E1
:102C70008E1B26604AE7002084468646F1E701461F
:102C8000C069019DD1F804A02E68444DD1F8089088
:102C9000AAEB060C2CF07F4CAC4535D80CEB0906A2
:102CA0000E60D3F800C081F81080C1E90144CC6106
:102CB000BCF1000F33D1196031E701EB410B013159
:102CC000C9B2514514BF117014701CF83B10012992
:102CD0000CEBCB067FF42CAF716891F810B0BBF110
:102CE000000F7FF425AFD6F808C0C1F804C0F5681E
:102CF0008D603569CD6076698E61BEF1000F0CBFC5
:102D000066465E464E60BCE7A6EB0A0626F07F46A6
:102D10004E4502D2A9EB0606C2E70C60C1E7D1F826
:102D20000090DCF80060B1451FD8A6EB0906CCF88E
:102D30000060C1F81CC0BEE7A9EB0A09D6F81CA0C8
:102D4000B446BAF1000F0AD05646D6F800A0CA45DC
:102D5000F2D3AAEB090AC6F800A0B2466646C1F84B
:102D60000090C1F81CA0F161D9E66646EDE7FFF7D7
:102D70006DFE2CE7ACA50020ADA50020B0A500207D
:102D8000A4A500208CA60020D0A300208CA50020A4
:102D9000001001408DA5002000E100E0FEFF7F0053
:102DA00074450FD1D0F81CB0C3F800B0BBF1000FD0
:102DB00008D10A4D0120A86001984FF0010CC0F81D
:102DC00000B0E1462068E469CEF81C40002C3FF4D6
:102DD0008BAE25682844206086E600BF00100140C5
:102DE00037B5074B054693E803006C46002384E89B
:102DF00003001A4621462846FFF742FD03B030BDC6
:102E0000EC3A0500FDF732BB10B54FF6FF730446F0
:102E10009C42084609D1FEF755FFB0F5807F044675
:102E200001D14FF6FF74204610BDFF2CF9D8214682
:102E3000FEF724FF0028F6D1F3E710B5044601F0B1
:102E4000EFFC2046BDE8104000F02EBF1FB5037810
:102E500093B90279072A0FD1448803932046CDE91C
:102E600001338DF80420FCF767FCADF8060001A8DB
:102E7000ADF80840FFF7E1FF04B010BD1FB5002317
:102E8000CDE901330393ADF80600022301A88DF8C4
:102E900004308DF80810FFF7D0FF05B05DF804FB93
:102EA00086DF704738B504884CB9821C00F10A05EA
:102EB00012F8013B1BB99542FAD100200AE00B88B9
:102EC000A342FAD108220231023030F0B1FDB0FA4B
:102ED00080F0400938BD08B570B171B103780A7847
:102EE000534013F0FE0F08D106220131013030F0BB
:102EF0009FFDB0FA80F0400908BD0020FCE710B546
:102F0000044600F0BDFF2046BDE8104000F04ABF77
:102F100043DF70476FDF7047024B0022C3E9002296
:102F2000704700BF2CA20020F0B5FF2887B00446F0
:102F30000E4615461F4629D80846FCF713FC28B351
:102F400003AA2046FFF728F918B10524204607B048
:102F5000F0BD01A903A8FFF755F804460028F4D1F5
:102F6000019BAE705A882A805FB13B6892009A42FA
:102F70000AD30299686830F069FD03A8FFF726F8C4
:102F8000E4E7029B6B60F8E70424DFE70724DDE752
:102F90002DE9F041CEB020AE502380460CADB822D2
:102FA0000021304601930395FCF7BCFA0DF197031D
:102FB00005930DF1AE0306930DF1C503079337ABEF
:102FC00008930DF1F30309930DF585730A931C4FD4
:102FD00004960DF221130B930024444507D1E2B26D
:102FE000002104A8FFF796FF4EB0BDE8F081502203
:102FF00000212846FCF796FA01AB02AA072137F810
:10300000020BFFF791FF20F002000528ECD06B7C4B
:10301000032B12D817230DF1310203FB04630DF1CA
:10302000450152F8040B43F8040B8A42F9D1118888
:10303000198092789A700134CFE743F20220D3E7E7
:10304000B6A500202DE9F04110220546A6B00021CA
:103050002D48FCF767FA35B929462846FCF780FB6E
:1030600026B0BDE8F0816A0028492748DFF89C8037
:1030700004AE30F0EBFC382200213046FCF752FA67
:1030800000245023CDE9013412AF039750220021D0
:103090003846FCF747FA01AB02AA072138F8020BC1
:1030A000FFF742FF20F002000528D9D09DF85930E3
:1030B000032B26D8C4EBC402B318DDF85910B15065
:1030C0000134BDF85D209A80A5429DF85F209A7179
:1030D000DCD10DF1170313930DF11E0314930DF1C1
:1030E000250315930BAB16930DF1330317930DF1D5
:1030F0003A0318930DF1410312961993E9B2384639
:10310000ACE743F20220ABE7C6A50020B6A500203D
:103110002DE9F043037889B00546002B3FD10179B2
:1031200007293CD104AA4088FFF7FEFEB8BBFFF791
:10313000F3FE02A90DF10600FFF704F878B36E88DC
:10314000BDF80670BE42F4D0059C631C18461134CD
:1031500013F8012B12B9A342FAD1EAE7DDF80C808B
:10316000102208F1010130F063FC08F111018146E1
:103170002046FFF7B0FEB9F1000F01D00028D8D0EB
:103180003046FCF7D9FA0023ADF81A0006A88DF8EE
:103190001830ADF81C60ADF81E70FFF7B0FE09B036
:1031A000BDE8F083CA1F012A73B5064654D800252E
:1031B000CDE900558DF80210FCF7FEFA0446002810
:1031C0004CD0437CDB074BD4007CFCF745FB10B9AB
:1031D000032002B070BDE368019003EB83031B0181
:1031E0009BB29B086846ADF80030FCF7C3FA6268F2
:1031F00004F1080369463046FFF742FB637C03F0A5
:103200000603062B01BF174A136803F1FF3313604F
:1032100030B9637C23F0070343F001036374D8E7FC
:1032200011280BD10F4A136801331360637C23F01C
:10323000060343F0040363740020CAE7862809D11B
:10324000084A136801331360637C23F0060343F0DC
:103250000203E3E70728BBD10720BAE70520B8E758
:103260002846B6E7CCA300202DE9FF4105461022F1
:1032700000216846FCF756F968882979ADF8020004
:103280008DF80410FCF798FA2B78454E092B5ED880
:10329000DFE803F00505684D4D6C7173757D0028FE
:1032A0003FD0437CDC073CD5FEF742FE2B78581E0E
:1032B00043424341002468468DF800408DF80830B1
:1032C000FCF76CFA33684BB3364E002537464FF0A7
:1032D000140808FB05735B7C5A0703D49B0759D578
:1032E000002C57D0B1783088FFF75CFF002851D010
:1032F00014235D437B1986289B788DF804307A5B14
:1033000016BF0290082309236846ADF802200CBFBF
:103310008DF800308DF80030FCF740FA04B0BDE8BD
:10332000F08101238DF80030AB68029316E080B184
:103330008268AB689A420CD1437CD90709D53268C0
:1033400023F00503013243F0040332604374002488
:10335000B8E702238DF80030EB6803936846FCF76A
:103360001DFAF4E703238DF80030F7E704238DF806
:103370000030EB68D9E70523F5E70623F7E70723D5
:1033800068468DF800300124FCF708FA9AE7EB68EC
:103390000293DCE70135082D06F1140699D1BDE74B
:1033A000CCA30020E8A5002070B500238CB02D49E7
:1033B0002C4E4FF6FF70CDE90033FCF7B1FA4FF613
:1033C000FF750446AC420BD0A4F58043ADF8143031
:1033D00002AA6B46002105A8FEF77AFE0A2822D031
:1033E000214B1A781846E2B94FF6FF718C4218D07B
:1033F0001E4E367801251D70B607A4F580439BB29A
:103400001DD58B422CD005218DF8141005A811462E
:103410008DF81850ADF81A30FEF712FE60B1FFF7C4
:103420009BF90CB070BD2046FEF7BCFD204631462E
:10343000FCF776FA0446C5E70D4B1D70F1E7022351
:103440000022092102708DF8141005A8FF21ADF8A3
:1034500016408DF81810CDE90723FFF705FFE0E7C8
:103460000423EDE7CCA4002065A4002038A20020AE
:1034700066A40020F0B5426805783D4C85B0B2FAEC
:1034800082F149090391691E0346042924D8DFE823
:1034900001F0030330496A009989DE8901F5804112
:1034A00089B243F6FE77B94204D906F5804080B26E
:1034B000B84211D8012DADF802108DF8046013D177
:1034C000002A14BF032100218DF8001003929B688D
:1034D00002936846FFF7C8FE23781BB100232370D0
:1034E000FFF762FF05B0F0BD002A14BF04210121DF
:1034F000EAE79989DD8901F5804189B243F6FE76D4
:10350000B14204D905F5804080B2B042E4D8002A27
:103510000CBF02220522ADF802108DF804508DF880
:103520000020D4E7988900F5804080B243F6FE7110
:103530008842D1D8DB89002BCED1FF23ADF8020021
:103540008DF804305AB906238DF80030FEF72AFDB5
:10355000084A002323701370FFF726FFB9E70723FB
:103560008DF80030F4E708238DF80030B1E700BF94
:1035700066A4002065A40020F8B50D490D4DFCF7A8
:10358000CFF94FF6FF760446A5F12007B44201D1EA
:103590002046F8BDFF2CFBD821462846FCF74CF905
:1035A0000028F5D020463946FCF7BAF90446EDE785
:1035B000ACA40020CCA4002073B5104B104C93E8B1
:1035C00003006D46002385E803001A46294620883B
:1035D000FFF756F94FF6FF762388B34201D0112842
:1035E00001D102B070BD1846FFF7C6FF00231A468E
:1035F00029462080FFF744F9EEE700BFF43A0500C2
:1036000014A200201FB50378012B044615D10179BF
:10361000012912D1002302AA4088FFF785FC60B976
:1036200002238DF800306388ADF80230039B6846B2
:103630001B788DF8043000F0B5FD054B1A884FF665
:10364000FF739A4201D0FFF7B7FF04B010BD00BF6F
:1036500014A2002070B504468AB0142200216846E6
:10366000FBF760FF6588ADF804502846FCF764F866
:103670002378ADF80200092B15D8DFE803F0051612
:103680003048525E8614A1A507238DF800302379B7
:103690008DF808309DF80A3043F001038DF80A30A8
:1036A0006846FCF7AFF80AB070BD07238DF800300C
:1036B00023798DF808309DF80A30444AA1680391B7
:1036C00043F001038DF80A301368002BE8D09942CB
:1036D000E6D1002313603E4A03931580E0E70823F8
:1036E0008DF8003023798DF80830E3680493374B68
:1036F000A1681A680391002AD2D09142D0D13549ED
:1037000000221A600B680392013B0B60C8E7072395
:103710008DF8003023798DF8083001238DF80930B9
:10372000BEE708238DF8003023798DF80830012397
:103730008DF80930A3680493B2E7274D09238DF86B
:1037400000302B78002BABD04FF6FF70FFF714FF43
:103750004FF6FF7398420646A2D12049FCF7E0F8E5
:10376000B04204469CD1142200210DEB02002970C6
:10377000FBF7D8FE0B238DF81430ADF81840ADF8E8
:10378000164005A8FCF73EF88AE70A238DF80030BA
:10379000114BA4681A780294002A81D014220021C7
:1037A0000DEB02001970FBF7BDFE0C238DF81430F1
:1037B0004FF6FF73ADF81830ADF816300794E0E718
:1037C00005238DF800306BE70623FAE7A8A4002054
:1037D000C0A3002010A2002016A20020CCA400202C
:1037E0002DE9F047474B1B788AB00546002B00F0C7
:1037F0008780454B454F93E803003C7803AE86E84D
:103800000300BCB94FF6FF70FFF7B6FE0123ADF819
:10381000143001AB06930423029305AA02AB0621E0
:1038200080460194ADF81640FFF77EFB07284AD189
:1038300001233B70364B1C689846002C5AD1354A00
:10384000354F12883B68AA4241D1002B3FD0142249
:1038500021460DEB0200FBF765FE072328468DF895
:103860001430FBF769FF0623ADF8160005A8ADF884
:1038700018508DF81C30FBF7C5FF20460AB0BDE894
:10388000F087CDF804A0019B4046A34224BFC14667
:103890001C46FFF771FEBDF814309B00029305AA89
:1038A00002AB06218046FFF73FFB0028EBD005283E
:1038B000E7D04FF6FF7398451CD1164BA3F8009044
:1038C000154B1C60B4E74FF6FF79A246EDE70133D4
:1038D0003B6000220E4B31462846FEF7D1FF002800
:1038E000CCD00023C8F800303B68112803F1FF3327
:1038F0003B6001D11120C1E7862818BF0320BDE736
:103900000820BBE7C8A30020FC3A0500A7A40020BC
:10391000A8A40020C0A3002010A2002063DF7047ED
:10392000A6DF7047A2DF70472DE9F04391B09846BB
:1039300011238DF8043013788DF8053000241646D5
:1039400001254FF0000365F34203074689461C2218
:10395000214609A88DF80630FBF7E4FDB3788DF811
:103960000930C3F30302A24214BF1A2212228DF8B7
:10397000242001AA0E9203AB72788DF808200493DC
:10398000224602AB65F34202059308238DF80A2014
:10399000CDE9064404AAADF81C3009A9434638888D
:1039A0008DF80E50ADF80C900894FFF7BBFF11B0E6
:1039B000BDE8F083A0DF7047044A0123116883400B
:1039C0000B401ABF1218507E18467047C49F002043
:1039D00070B4094D134601262A6806FA01F4144210
:1039E00007D001F1190402463146281970BCFDF7D1
:1039F00063BD70BC704700BFC49F00201FB500238B
:103A0000CDE9013303938DF80A201A46074BADF830
:103A1000081006241978ADF806008DF80440FFF769
:103A2000D7FF01A8FFF709FA04B010BDAF2C0020A2
:103A300010B4084A012314688B40234006D00A447E
:103A40005DF8044B0146507EFDF7A6BC18465DF8B4
:103A5000044B7047C49F002010B50A4B19780446E8
:103A6000FFF7E6FF58B1084B00205A88A24201D167
:103A7000C0B210BD0130082803F10C03F5D1FF20BE
:103A8000F7E700BFA4A10020A6A100202DE9F8437C
:103A90000546FBF751FE234B0746002214209846AB
:103AA00000FB02F1CC5AAC422AD10B44002634462A
:103AB0004FF014095BB199782846FEF755FA10B11A
:103AC000052818BF032401363246072A1DD9A4B998
:103AD000FF2D24D8144928464FF6FF75FFF794F9B7
:103AE000FFF762FCAF4208D03846FFF7B5FFFF286A
:103AF00003D00C2343430D4AD5522046BDE8F8833A
:103B00000132082ACCD10023D0E709FB02F338F8B0
:103B10000310A94201D14344CCE70132D5E7072481
:103B2000EBE700BFE8A50020CCA40020A6A1002060
:103B30002DE9F0411F46154B9DF818400E46904662
:103B400019780546FFF744FFB8F1000F17D0104B66
:103B50003A4619782846FFF73BFF0E4B2246197864
:103B60002846FFF735FF44B12846FFF775FFFF28C9
:103B700003D00C234343084AD652BDE8F081002C01
:103B8000FBD03046BDE8F041FFF780BFAF2C0020EE
:103B9000B12C0020B02C0020A6A1002008B5FFF712
:103BA0005BFFFF281DBF0C234343034A4FF6FF7002
:103BB00018BFD05A08BD00BFA6A100202DE9F043D0
:103BC00085B00546FFF7EAFF4FF6FF7398420746B8
:103BD00041D001224FF0030901AB0821384602F120
:103BE0000108FEF7D5F81FFA88F8064648BB029987
:103BF0000A46032342F8049B06312846FBF790FD52
:103C0000044660B908213846FFF7CCFA0446112C67
:103C10003FD01AD80CB30C2C2FD107231EE00C2850
:103C20000DD0052800D1344608213846FEF79CF90E
:103C3000002818BF03244246002ECDD1E7E7012615
:103C4000F2E70728E9D00446E1E7862C13D043F2D7
:103C500002039C4211D100221CE0012328468DF86A
:103C60000430ADF80850FFF799FFADF8060001A841
:103C7000FFF7C8F8EFE70823F0E7092328468DF897
:103C80000430FFF78BFFADF80850ADF80600039441
:103C9000EDE70122034B28461978FFF799FE05B09E
:103CA000BDE8F08335A200200378072B02D14088BD
:103CB000FFF784BF704700002DE9F0434FF6FF7512
:103CC000A84285B0044668D0FFF768FFA84227D114
:103CD00000260327B0464FF001093B4632464146D5
:103CE0002046FBF71FFD042805464DD0082847D085
:103CF0000B282DD117F002031FD1B8F1000F20D1EE
:103D00001EBB032320468DF80430FFF747FFADF8B4
:103D10000840ADF8060001A8FFF774F8002237E06C
:103D2000002301AA0821FFF7FFF80028D0D1029B49
:103D300003F106089E881F68CDE701274FF00009B0
:103D4000CBE703271E469846F8E703274646F5E7E4
:103D5000B9F1000FD5D0112819D043F202039842CF
:103D6000DCD008B90223CDE7092320468DF80430C2
:103D7000FFF714FFADF80840ADF806000395CAE759
:103D8000B9F1000FEED1BCE7B9F1000FB9D00122B3
:103D9000034B20461978FFF71BFE05B0BDE8F08302
:103DA00034A2002037B50578012D044614D140888F
:103DB000FFF782FF6088FFF7F1FE00236A4629467D
:103DC000FFF7B2F840B9019B1B782BB1034B608819
:103DD00019782A46FFF7FCFD03B030BD36A200205B
:103DE000F0B587B004460E461746FFF7D7FE4FF6EC
:103DF000FF739842054624D01E4B20461978FFF7E2
:103E000017FE80B30023CDE90033029304238DF81D
:103E10000030194BADF802401978ADF80460204627
:103E20008DF80670FFF704FE68B12846FFF72EFEF6
:103E3000124B204600221978FFF7CAFD6846FEF7AC
:103E4000FCFF07B0F0BD07212846FEF78DF80528D6
:103E5000EED10923049003A88DF80C30ADF80E4084
:103E6000FEF7EBFFE4E73A4631462046FFF7C6FD92
:103E7000E7E700BFB12C0020B02C0020AF2C0020C1
:103E800010B5027886B004461AB1012A09D006B0EE
:103E900010BD0E4B1B78002BF9D0C088FFF7F6FD44
:103EA000F5E70B4B40881978FFF792FD14220021AB
:103EB00001A8FBF737FB6088ADF80600FFF76EFE40
:103EC000ADF8080001A8FBF79DFCE0E7C8A30020BF
:103ED00000A0002070B5044686B01422002101A87D
:103EE000FBF720FB23786088ADF80600013B0B2B25
:103EF00000F29080DFE803F02106233A4E585C6818
:103F0000747A7C8C2679444B321C19784FF0010569
:103F100018BF01228DF80450FFF75AFD731B5A4257
:103F20005A413E4B60881978FFF752FD6088FFF7D1
:103F300035FEADF80800002D42D106B070BD022359
:103F40008DF804302379002B14BF012302238DF850
:103F50000C30314B01221978FFF73AFD2F4B2279B3
:103F600019786088FFF734FD0125DFE703238DF81A
:103F700004302A4B1978FFF75BFD002814BF01239A
:103F800002238DF80C30A3798DF81030A388ADF89A
:103F90000E30E9E7204B1978FFF74AFD0028CCD115
:103FA00002238DF80430DFE703238DF80430EAE7BD
:103FB0000723A2888DF80430ADF808208DF80C3066
:103FC00001A8FBF71FFCB8E708238DF80430A3888D
:103FD000ADF8083007238DF80C30A3680593EFE7A0
:103FE00006238DF8043063680393BDE70523D8E703
:103FF00003238DF80430094B1978FFF719FD0028C9
:1040000014BF012302238DF80C3041F20113BEE7E7
:104010000423C6E7002589E764A4002000A000204F
:104020001FB50D294FF0000301930393ADF806006F
:10403000029108D10B2301A88DF80430FFF74AFF45
:1040400005B05DF804FB86290CBF0A230923F2E7BB
:1040500030B508490A680023012505FA03F4224215
:10406000D8B202D122430A6030BD0133182BF4D1FB
:104070001846F9E7C49F002010B50378182B0446B2
:1040800002D1FFF7E5FF207010BD000010B5024B14
:10409000197DFDF72FFA10BDC49F00202DE9F04FC8
:1040A0003D4D89B02878FFF787FC60B103A8FFF782
:1040B000EDFFDFF8E8A0DFF8E8B00DF11009002708
:1040C000039B9F4202D309B0BDE8F08F39F8024B41
:1040D00029782046FFF7ACFC064678B39AF8001022
:1040E0002046FFF7A5FC804640BBBBF800304FF6EA
:1040F000FF7219462046FBF717FB43F2030290427A
:1041000029D10133ABF80030EFE7052320468DF8C5
:104110000030FFF743FDADF802006846ADF80440FB
:10412000FEF770FEB046324629782046FFF750FC75
:1041300042469AF800102046FFF74AFC0137BFE7D5
:104140002046FFF72BFDFEF74BFE0026EBE720464F
:10415000FFF7B2FDE7E70828F2D012D80028D4D044
:104160000628EDD00923029020468DF80030ADF8E6
:104170000440FFF713FDADF802006846FEF742FE6B
:10418000D1E743F202039842CDD043F20143984273
:10419000DDD01128E6D1C6E736A2002037A20020E4
:1041A000B8A600201FB5044640882378ADF8060065
:1041B000012B10D05AB21AB1022B15D004B010BD89
:1041C00001A88DF80420FEF71DFE6088FBF7B4FA05
:1041D000FFF772FDF2E78DF8043001A8A388ADF86F
:1041E0000830FEF70FFEE9E72379002BE6D0FBF756
:1041F000A3FA4FF6FF739842E0D0044B01221978DE
:10420000FFF7E6FBFFF74AFFD8E700BF36A2002022
:1042100038B5074C0146207DFDF7BEF830B1A07DD2
:10422000FDF7BAF8002814BF0220012038BD00BFF6
:10423000C49F00202DE9F0478CB089461646804681
:10424000FFF7E6FF20228246002104A8FBF76AF967
:10425000BAF1000F46D0B9F1000F17D099F800500D
:1042600015F001054FF6FF7415D04046FFF796FC98
:10427000A042074639D14048FDF724FDB0F5807FC4
:1042800001D0B84275D10025032470E04D46852643
:104290004FF6FF775FE02E4627465CE04A46314600
:1042A0004046FBF745FA0446B9F1000F5DD00028FF
:1042B0005DD199F8003013F0010F14BF01210221E4
:1042C0004046FEF7DBFDB6F1850218BF012200244F
:1042D0000095012339464046FFF72AFC20460CB0E2
:1042E000BDE8F08743F20204F8E7002502AB0122A3
:1042F00007213846FDF74CFD0446002837D12146FA
:1043000050220398FBF70EF9039B83F800A0039C4F
:10431000079604F13403049304F118030893631C13
:1043200009934046154B0B93FFF796FBFF280CD0E3
:10433000134A0C2101FB002050F8042FC4F811206F
:104340008288A4F815208279E2753846FBF79CFA3A
:10435000044660B90646BAF1020F04AB9ED10022B2
:1043600031464046FBF7E4F90446002CABD000226E
:10437000AEE707460125B9E7ACA4002067A40020FA
:10438000A6A10020F0B585B00446FFF741FF324FEB
:10439000012806463D7831D12046FFF7FFFB4FF656
:1043A000FF7398422AD0204632462946FFF710FB79
:1043B0000023CDE90133039301A80C238DF80430C9
:1043C000ADF80640FFF786FD244B1B78E3B1397842
:1043D0002046FFF72DFBB8B9214B22491A68204629
:1043E000FFF728FF8628054632D011280FD070B17C
:1043F00029462046FFF714FE05B0F0BD00222946ED
:104400002046FFF7E5FADFE700221146E7E7A5F1CE
:1044100011035E425E410022134B20461978FFF7DC
:10442000D7FA124B324619782046FFF7D1FA104BD3
:10443000002219782046FFF7CBFA0E4B002219789C
:104440002046FFF7C5FA002DD6D0112DD4D0CFE7E6
:1044500000260122E0E700BFAE2C002093A500203B
:1044600050A400208EA50020AD2C0020AC2C0020F4
:10447000AB2C0020AA2C0020F0B587B0074601A87D
:10448000FFF704FE02AD0024019B9C4201D307B05C
:10449000F0BD35F8026B39463046FFF7C9FA10B166
:1044A0003046FFF76FFF0134EEE700002DE9F04FD3
:1044B000054687B0904699460F4639B9A14B1B78FF
:1044C000F3B90524204607B0BDE8F08FFFF7A0FE42
:1044D0000138C0B2012800F22D8100212846FBF7E7
:1044E00029F90446862C00F0B080112C00F0998048
:1044F000002C00F09680B9F1000F00F0BF80B9E009
:10450000FFF786FE012800F09E80022840F012810D
:104510008D490B78284613F001048B4614BF4FF0E9
:10452000010A4FF0020AFFF739FB4FF6FF7398427A
:10453000064659463AD03B4602AA0721FEF7F4FC4C
:104540000446F0B9039B93F84420D10740F1C7809B
:10455000B8F1000F40F0D68003F1340202F11201ED
:104560002846FBF7E3F84FF0000A044600230093C7
:10457000BAEB030318BF0123B4FA84F2520931469F
:1045800045E00528F2D1BDE004AB01220721304609
:10459000FDF7FEFB0446002840F0C1803046FBF7E3
:1045A00073F90446002800F0B280B8E0002C41D036
:1045B0006648FDF787FBB0F5807F834637D0B04271
:1045C00036D004AB01220721FDF7E2FB044650B9C7
:1045D0005846FBF759F9044628B95B492846FBF7CA
:1045E000A9F8044638B107215846FDF7BDFC10B1C3
:1045F000052818BF03244FF6FF73BBEB030318BF56
:104600000123B4FA84F20093520901235946284643
:10461000FFF78EFA002C7FF465AF51462846FEF76F
:104620002DFCA4F111035E425E4100220FE0B3466F
:104630000324E0E72846FBF77DF8009704460123B2
:10464000B0FA80F29AE7404948E700260122404B41
:1046500028461978FFF7BCF93E4B324619782846B0
:10466000FFF7B6F9B9F1000F08D0002C3FF42AAFDC
:10467000112C17D021462846FFF7D2FC0D2C3FF411
:1046800021AF06D8002C3FF41DAF082C18BF03241F
:1046900018E7862C14D043F202039C423FF412AF79
:1046A000112C1AD12C4B3A4619782846FFF790F96D
:1046B0002A4B424619782846FFF78AF9002401E779
:1046C000254B3A4619782846FFF782F9234B424694
:1046D00019782846FFF77CF9F4E60324F2E6B8F1EE
:1046E000000F0FD1598D03F1180200297FF436AF66
:1046F00003F12C01343311F8010B00287FF42EAFA5
:104700008B42F8D19BF80030DA073FF53DAF0E49F8
:104710002846FBF70FF8044600283FF427AF07218F
:104720003046FDF721FC00283FF420AF052818BFD4
:1047300003241BE743F20204B9F1000F3FF4C2AEB9
:1047400098E700BF93A500208EA50020ACA4002010
:10475000AB2C0020AA2C0020A92C0020A82C002083
:104760002DE9F04786B00746FFF726F958B101A8B2
:10477000FFF78CFCDFF84880DFF8489002AE002598
:10478000019B9D4202D306B0BDE8F08736F8024B8C
:1047900039462046FFF74CF980B198F800102046C2
:1047A000FFF746F999F8001082462046FFF740F9D6
:1047B0000123014652462046FFF778FE0135DFE728
:1047C000A82C0020A92C002010B50378062B0ED9A8
:1047D000072B1BD10E4B1C782046FFF7EDF810B1CC
:1047E0002046FFF749FE0B4B1878FFF7B9FF0A4B3D
:1047F0001C782046FFF7E0F810B12046FFF73CFE9A
:10480000064BBDE810401878FFF7AABF10BD00BFE7
:10481000AD2C0020AB2C0020AC2C0020AA2C0020BA
:104820001FB503780446092B09D8DFE803F0050A11
:1048300020202020202020204088FFF7A3FD04B066
:1048400010BD144B197819B3134B00791B7803F082
:104850000102904206D86179C3F34003994294BFA4
:1048600000210121012300226088FFF71FFE237829
:104870008DF80430043434F8023CADF8063094E886
:10488000030004AB03E9030001A8FFF723FBD6E70D
:104890000121E7E793A500208EA5002037B5174B2F
:1048A000174A5B881188174C174D994208D85288CF
:1048B0009A4205D36369FBB900232B7003B030BD66
:1048C0002B783BB16369002BF6D000228DF80420D1
:1048D00001A80FE00D490E480978D4E90123002909
:1048E0000CBF11461946FDF785F90028E4D0A369ED
:1048F000002BE1D09847DFE70122E7E706A200207E
:10490000ECA4002068A1002004A10020B4A5002090
:1049100084A100207BDF70477ADF704776DF704725
:1049200075DF704737B5164B18884FF6FF739842FE
:1049300010D0144A144D1378297B0133DBB299420D
:1049400013702C4608D31149FFF7EAFF10B1AB6989
:1049500003B1984703B030BD002313702B7C33B1F3
:104960003B21FFF7DBFF10B1AB6903B198476369E7
:10497000002BEFD000228DF8042001A8E9E700BF4A
:1049800064A10020B4A5002068A10020ECA40020B0
:1049900065DF70472DE9F74F0C9CBDF834B02788D0
:1049A000002580468A4691462E46B8F80020B2423D
:1049B0000BDC35B12288013AD21B92B2FF2A39D8DA
:1049C000DA55002003B0BDE8F08FD8F8042052F883
:1049D0002600019000220DF1030101A8FFF7D8FF86
:1049E0000028EFD19DF803204A4521D12288002DCF
:1049F00014BF0020022002EB09010144594519DCD3
:104A00003DB9013292B2228003F802A0228801321D
:104A1000228022880DF103011A4401A8FFF7B8FF94
:104A20000028CFD121889DF803200A442280012547
:104A30000136BAE70C20C5E72DE9F341089CBDF823
:104A400024501746CDE9004502220646FFF7A2FF93
:104A500048B9102239463046CDE9084502B0BDE8D4
:104A6000F041FFF797BF02B0BDE8F0812DE9FF47A5
:104A70000023138090F82D3006460D4614463BB3B4
:104A800002A8FAF7D7FE002840F0FB80138808221E
:104A9000CA54238801339BB21B222380CA54238823
:104AA00001339BB2CA18DDF809102380E950BDF824
:104AB0000D30938023889DF8082006339BB212F0B6
:104AC000FE0218BF01222380EA5423880133238089
:104AD000B378FBB1238804331F2B21D802A8FAF73F
:104AE000A7FE002840F0CD8023880322EA542388C3
:104AF00001339BB219222380EA542388BDF8082091
:104B000001339BB2E9182380EA54120A4A702388C1
:104B100002332380F278AAB12388D91C1F2901D936
:104B20000C20AEE00221E954238801339BB201211D
:104B30002380E95423880B449BB22380EA542388C2
:104B40000B4423807268AAB12388D91C1F29E7D897
:104B5000022192F90020E954238801339BB20A21F3
:104B60002380E954238801339BB22380EA542388AD
:104B7000013323803389002B76D1338A5BB11F2325
:104B8000CDE9004307222B46032106F11000FFF771
:104B900053FF002875D1338B5BB11F23CDE9004350
:104BA00015222B46142106F11800FFF745FF0028B7
:104BB00067D1326A002A67D1776A4FB3BB882188F0
:104BC000981C8A1C02441F2AAAD8FE28A8D803339E
:104BD0006B54238801339BB2FF222380EA5423883D
:104BE00001339BB223803A88EA54E918120A4A70CA
:104BF0002088023080B22080BA884AB1B968002982
:104C00004AD028442EF022FF2388BA8813442380F8
:104C100096F82C30002B79D1307890B33388012B63
:104C20003AD023889F1C1F2F3FF67AAF012805D169
:104C3000727802321A441F2A3FF672AFC3F11D0385
:104C40009BB202A9E819ADF80830FAF7EFFDC0B938
:104C50003278022A40F09880BDF808209A4240F24B
:104C6000AE80ADF8083098E01F23CDE9004306225E
:104C70002B46022106F10800FFF7DEFE00283FF474
:104C80007CAF04B0BDE8F0872788BB1D1F2B3FF623
:104C900047AF1188052901D80720F2E76FF4486C67
:104CA00001EB0C039BB24FF27D3C6345F4D9538872
:104CB000052BF1D96FF44860181880B26045EBD924
:104CC0004FF6FF70814203D0834201D09942E3D86E
:104CD0000523EB55238801339BB212212380E9542D
:104CE000238801339BB223801188E954E818090A0C
:104CF0004170238802339BB223805288EA54E9181A
:104D0000120A4A7023880233238055E7B36A002BC6
:104D1000C2D04FF000084FF00C094FF0160A96F879
:104D20002C305FFA88F293427FF676AFB16A09FBC6
:104D300002F28F18BB88981CFE283FF6F1AE20883F
:104D400003332B54238801339BB2238005F803A03F
:104D5000238801339BB223808A5AEA54E918120A45
:104D60004A702088023080B22080BA884AB1B9687F
:104D7000002991D028442EF069FE2388BA88134474
:104D8000238008F10108CAE7012A7FF46AAF72782C
:104D90009342FFF466AFADF808200821BDF8083053
:104DA000FE2B3FF6BDAE22880133AB542288013280
:104DB00092B22280A95422881344238061E70921FA
:104DC000ECE7000007B5144B1A686AB100201860C0
:104DD0001B6800934FF08042009B0123C2F8083308
:104DE0000E4A5370FAF7B6FD0D4B1A688AB10022CD
:104DF0001A601B680193019B4FF080430222C3F8A5
:104E00000823064B0120987003B05DF804EBFAF715
:104E1000A1BD03B05DF804FB0001004050A10020DB
:104E2000040100400E4BD3F8183182B0B3B10D4BE2
:104E30000D4800221A601B680193019B0B4B997E61
:104E4000FF291FBF01228A404FF0A041C1F8082569
:104E500000225A761A711B6802B0184702B07047D8
:104E60000030004018310040C8A00020C4A000203D
:104E700070B52D4C86B094F82130019394F8203011
:104E80000093E36904F1260204F123014FF040206E
:104E9000FAF77AFD2346E0B994F82360A56906BBCA
:104EA000217B8A1E012A1CD8E0692269904218D110
:104EB0006269E37BE261C5F34015032984F8203081
:104EC00084F8215007D100954FF040212046FAF791
:104ED00032FE06B070BD4FF040212046FAF7CEFDFD
:104EE000F7E7124A07CA06AC04E90700C6B14FF05B
:104EF0004021D1F8C424C1F8C42490070CD5012264
:104F00008DF80820002283F824206A07E1D4D3E931
:104F1000002102A89047DCE75107F3D50222EFE712
:104F20008DF80860EEE700BF9CA00020A8A000203C
:104F3000F7B515464FF0FF32C1F8082390F824204A
:104F400004460F4602F0FF0E2AB18368C1F804330D
:104F5000112003B0F0BD012680F82460836100F1C8
:104F60000C0C95E807008CE80700AA7884F820204C
:104F70006A68E2616A78C7F888252A78B24212D056
:104F800012B91E1C18BF012684F821600096AB7868
:104F90006A6839462046FAF7CEFD2368002BD8D13F
:104FA00084F82430D5E784F821E0AB786A68394684
:104FB0002046FAF763FDF0E730B54A4AD2F80433E9
:104FC00013F4007F85B015464AD0D2F82431002B67
:104FD00046D04FF492711046FAF718FE4FF4017361
:104FE000C2F80833404B997E09B9012151603D490F
:104FF00002228DF80020D1F88024C1F88024039289
:10500000DA7D8DF80820DA6801920022DA751A76C6
:105010006846D3E9001290473248D0F81C313BB1C2
:10502000314A938A917D994247D91146FAF71DFE7C
:105030002C4AD2F844318BB14FF4A2711046FAF7E2
:10504000E5FD294B997E09B101211160DA7D2AB174
:105050000022DA75587ED968FAF78CFA05B030BDAF
:10506000D5F804335B07D7D5D5F80831002BD3D05A
:105070001D4C1C482146FAF7E1FD637EE27D9A4211
:105080002346C9D1227E52B12369E168E36000233F
:10509000607EE27523766376FAF76CFABCE7A27E4F
:1050A0000AB901226A600F4A4FF40171C2F808136D
:1050B0000022DA75587ED968EEE74FF48E71FAF760
:1050C000A5FD917D0029B3D000238DF808109168CB
:1050D0008DF80030019193756846D2E90013984726
:1050E000A6E700BF0020004080A00020800000F163
:1050F000A040D0F8003723F44033C0F80037D0F890
:10510000003743EA0141C0F8001770470E4B0344D3
:1051100093F94020072A02DD0021FFF7E7BFD3B251
:10512000072B10D8930003F1804303F5C043D3F855
:10513000101521F00101C3F81015012303FA02F242
:10514000024BC3F80823704714A000200060004001
:1051500000F1804000F5C040002382B00360036886
:105160000193019B02B070472DE9F04F85B00024F8
:10517000594D01944FF48072012102F1804303F5EF
:10518000C04390B21B68012B06D1D5F804330B4203
:1051900002D0FFF7DDFF0C430432B2F5907F4FEAF7
:1051A0004101EAD14D4B1B68012B0AD14FF4BE706F
:1051B000FFF7CEFF4FF0A04344F00044D3F8103582
:1051C000019314F0FF0F1AD0454F012600253442F9
:1051D00010D0AB0003F1804303F5C043D3F81005B2
:1051E000D3F8101557F8253023B1C1F30141C0F3AE
:1051F000042098470135082D4FEA4606E7D1002CD8
:1052000063DA4FF0FF330022CDE90232344D354EE0
:105210000024A24601274FF0A04816F9012B531C89
:1052200046D0D2B222F0C0094FEAD90104A80844FE
:1052300002F0070310F808CC07FA03F31CEA030F87
:1052400036D005EB090C92099CF940C055F82CB0FA
:10525000BBF1000F0AD1032A2AD10DF10C0E1EF862
:1052600001C04CEA030C0EF801C001E0032AF4D09F
:1052700009F5E07110F80C0C58F821101842C1F330
:10528000014105D0022913D1032A0BD1114604E0B4
:1052900003290DD1032A05D102214846FFF726FF35
:1052A0000134E4B2BBF1000F02D011464846D847A2
:1052B0000AF1010ABAF1080FAFD134B14FF0A0439F
:1052C000019AD3F81035934202D105B0BDE8F08FB2
:1052D0000193039B02939AE7006000407C610040C9
:1052E00014A0002074A000200028C3B2A8BF00F1C1
:1052F00060424FEA501010B5BABF0D4A03F00F04D8
:1053000002F561424FEA41114FEA8000C9B200F153
:105310006040B4BF115582F8001300F5614003F0FE
:105320001F0201239340C0F88031036010BD00BF0D
:1053300014ED00E02DE9F8430568EB175906674BBB
:1053400041EAD51104464FF0FF3268068B4208BF90
:1053500082420AD3624A00232EF0ACF900F50060C5
:1053600020F47F6727F00F072FB929465D48BDE875
:10537000F84321F0A9BD20791DF0BAF840B9607951
:105380001DF0B6F820B95848BDE8F84321F09CBD9F
:10539000E279E17A0D201DF03BF9237B534A002B83
:1053A00000F08A80537843F01003514E5370F37825
:1053B0001BB10023F370FBF7EBF825790023284697
:1053C000F3701DF095F820B14FF44071284614F0A9
:1053D00027F8657928461DF08BF820B14FF49851D5
:1053E000284614F01DF8637A2579002B284614BF4F
:1053F0004FF00E094FF000091DF07AF800285FD039
:105400003C4B05EB45051D4495F801806479204629
:105410001DF06EF8002856D0364B04EB44041C44B3
:105420006378354CE27E002A50D15A1C0AD04FF0E6
:10543000A04101229A40C1F8082503F5E07203203B
:1054400041F82200B8F1FF3F2C4D1FBF4FF0A041A3
:1054500008F5E072002041F82200C5F82475C5F86F
:105460006C950027C5F81485C5F80C35244B63608E
:1054700028464FF48E712760FAF7C8FB4FF4A271EB
:10548000FAF7C4FB1F4BC5F8043302210846FFF7A7
:105490002BFF0423C5F80035B8F1FF3F4FF48073AC
:1054A000E7822776638315D01748FAF7B7FB012305
:1054B000A376FBF781FC0DE0537803F0EF0374E76C
:1054C0004FF0FF38A2E74FF0FF33AAE708210F485B
:1054D00021F0DAFC0123F370BDE8F88347E801000E
:1054E00048E80100FC3B0500113C0500BE9F002080
:1054F000C5A60020CC3C050080A000200020004074
:10550000DD82030080000200103B0500273C0500FF
:10551000F8B50E46D11C48BF911D144641F38701D2
:105520000546671EFAF760FC00214AB2A24201F16B
:10553000010100DBF8BDBB1A23F00300B25C03F0ED
:105540000303DB0002FA03F32A581A432A50ECE75C
:10555000F0B500254F1E6CB28C4205F1010500DB51
:10556000F0BD3B1B23F0030603F003039659DB0059
:1055700026FA03F30355EEE72DE9F041B3F90240B3
:1055800014F11F0548BF04F13E050F4603F1240640
:1055900045F34715904601462B4632463846FAF702
:1055A0005FFCB8B9B4EB451F16DA6211012304F0B1
:1055B0001F0403FA04F457F822301C4214BF0124DC
:1055C00000242B46324639464046FAF749FC20462D
:1055D000BDE8F0810124F4E70446F2E710B50023AA
:1055E0001A465CB2A14203DCB2FA82F0400910BD57
:1055F00050F8234001332243F3E700002DE9F04F38
:105600008A46234F8BB00646114650461446FAF799
:10561000CBFB3B68FBB10425C0EB441014FB05FB3E
:1056200000B205FB04654FF0FF38043D28FA00F88E
:105630004FF040093B6859463046984758B12B68AF
:1056400003EA08032B6021463046FFF7C7FF20B16D
:10565000B9F10109EED1002017E023463246514648
:1056600002A8FAF7CDFB2146019002A8FFF7B6FF8A
:10567000019B003318BF01235B00002814BF584270
:10568000C3F10100C0B20128E2D10BB0BDE8F08F38
:10569000742D00202DE9F04FD1B0CDE905015B9DBF
:1056A00095F9004048A8914622461F46FAF770FB3C
:1056B000A3000793069BA20013441946224638A86C
:1056C0000293FAF765FB95F90060002F00F08C80DB
:1056D0003246394628A8FAF75BFB0DF5807A324648
:1056E00030AF48A95046FAF753FB38A93846FAF7C5
:1056F0004FFB2B4628AA38A948A8FAF708FB2B46E7
:1057000028AA38A948A8D5F8A460B0472B4628AAEB
:1057100039465046FAF7FBFABDF968310497023B67
:105720001BB2002B67DCD9F80030009503F00108AC
:105730004FEA481840AADB4302EB080A03F00103D2
:1057400030AA90445B0140AA1A44039230AAD318AD
:105750004146039A0493504605F10409FAF777FD90
:105760004B4640AA48A908A80094FAF7E0FC08A90B
:1057700008462B464246FAF789FA08A908462B46FE
:10578000069AFAF783FA214608A8FFF727FF0028B0
:105790005DD008A8FAF728FB08A92B46029A08460C
:1057A000FAF774FA08A92B4652460846FAF76EFA39
:1057B000DDE90301434652460095FAF7CAFC2B4641
:1057C00008AA30A940A8FAF7A2FA224640A90598EB
:1057D000FAF7DEFA059B079C234430A91846FAF72E
:1057E000D7FA51B0BDE8F08F314628A8FAF7FCFA95
:1057F0000123289371E71FFA83F85B1108F01F0259
:1058000059F823300095012101FA02F21A42049B53
:1058100013BF20270027202600260AEB070B1F4472
:105820000AEB06030393049B039A1E44334639464E
:105830005846FAF70CFD08F1FF383B4600955A46EA
:1058400031460398FAF785FC0FFA88F369E710AF41
:10585000224608A938460DF1600BFAF799FA20AEF6
:1058600049465846FAF794FA30462146FAF7BCFA08
:10587000012328A82093FAF7B7FA2246594638465A
:10588000FAF771FA28B9224620A908A8FAF780FA8F
:1058900082E73B68DA0709D421463846FAF756FA18
:1058A000224649463046FAF726FCE6E7189BDB0716
:1058B00007D421465846FAF749FA2246494628A80D
:1058C000F1E7002823461CDD5A4639463846FAF7E8
:1058D00097FA21463846FAF739FA224628A930467F
:1058E000FAF741FA002805DA23464A46314630469F
:1058F000FAF7B6FA234628AA31463046FAF780FA74
:10590000CEE73A4659465846FAF77AFA21465846BB
:10591000FAF71CFA2246314628A8FAF724FA00289A
:1059200005DA28A923464A460846FAF799FA28A92B
:10593000234632460846FAF763FABEE72DE9F047F8
:1059400093F9006092B004468946104631461546E8
:105950009846FFF743FE002840F0918042464946B2
:105960000AA8FAF7D0F943460AAA214602A8FAF78C
:105970008DF90AA908464246FAF7C5F943462A4670
:1059800049464846FAF782F908F104074246294693
:105990002846FAF7B8F93B462A46214620460096A3
:1059A000FAF73CFC3B462A46294628460096FAF779
:1059B00035FC3B462A46214628460096FAF7B7FBB7
:1059C00043462A4621462046FAF760F93B462246DE
:1059D000214628460096FAF721FC3B4600962A46C7
:1059E00021462046FAF71AFC2368DB074AD53346DE
:1059F0003A4621462046FAF733FA31468246204697
:105A0000FAF7A4F906F18043013B54F8230040EA79
:105A1000CA7044F82300424621462846FAF773F933
:105A20003B4602AA294628460096FAF780FB3B46E9
:105A300002AA294628460096FAF779FB02A90846E9
:105A40003B462A460096FAF772FB434602AA2146D5
:105A50002046FAF71BF90AAA3B4610462146009653
:105A6000FAF765FB324629462046FAF791F949468E
:105A70002846FAF78DF90AA94846FAF789F912B0CB
:105A8000BDE8F08731462046FAF760F9C3E7000029
:105A900073B500230DF102008DF80230FBF71AFAFE
:105AA000264B1B7803F0FF04002B41D1244B1A68CE
:105AB000002A3DD0234AD2F80813C90738D51C6004
:105AC0001B68214D01930DF10300019BD2F808657D
:105AD0008DF80340FBF7FEF96A6829681F2A98BF12
:105AE000541CA142F6B26C6004D1202C14BF611C7E
:105AF0000021296015499DF803008E542A689442BC
:105B00003ABFC2F121021319A31AAA689A4238BFF8
:105B1000AB60FCF759F86B682A681F2B94BF013300
:105B200000239A4201BF074A0123C2F80833536099
:105B30009DF80200FCF748F802B070BD94A5002063
:105B400000D1004000D0004080A500205CA50020CE
:105B500030DF70472DE9F74F3B4F06468846B8F1D6
:105B6000000F03D1012003B0BDE8F08F4546202D82
:105B700028BF20255FFA85FB002400230DF10200D9
:105B80008DF80230FBF7A6F9304B1B7803F0FF09C4
:105B900093BB0DF103008DF80390FBF79BF9D7E958
:105BA00000148C4204D3641AA54207D9052414E0DA
:105BB0002134641AA542F9D8C1F12104244BA5422D
:105BC000194431D82A4630462DF040FF3B682B441B
:105BD000212B28BF00233B6000249DF80300FBF726
:105BE000F3FF1C4B00221A601B680193019B1A4BA8
:105BF0000122C3F804231A609DF80200FBF7E4FFBA
:105C0000B9F1000F08D059463046FFF7A1FF42F224
:105C1000070398420446ADD0022CAED0002CA9D187
:105C2000A8EB05082E449AE7224630462DF00EFFD9
:105C3000074BA5EB040A5246194630192DF006FF12
:105C4000C7F800A0C8E700BF80A5002094A50020E9
:105C50005CA5002000D1004000D0004017B4314ABC
:105C6000314B116889B90021304A106820BB0020EF
:105C70005A79D40740D408B9002949D01C68DA8879
:105C8000234603B05DF8044B1847002111601268E9
:105C9000D9680092009A0029E5D0254AD2F840053B
:105CA000814204BFD88801EB8001C2F840155A79BF
:105CB00042F004025A71D7E7002010601268986819
:105CC0000192019A0028D2D0194AD2F83845A04250
:105CD00004BFDC8800EB8400C2F838055A7942F032
:105CE000020214075A71C3D512F0010402BF64F313
:105CF000C3025A712046BBE702F00601062907D10C
:105D000022F0060211075A7106D56FF3C3025A71C9
:105D100003B05DF8044B7047054AD2F83805D2F855
:105D20004015ABE71451024004A00020045102408A
:105D300000500240A5DF7047A4DF7047A3DF704723
:105D40002DE9F0470E4690B016F0100581469246B8
:105D50009846189C0CD011238DF8083023788DF8C4
:105D6000093001224FF0000362F342038DF80A303C
:105D70001C22002109A8F9F7D5FB8DF8246005B194
:105D800002AD42F64D23ADF80C3063789DF86410F7
:105D90008DF804300022A3788DF80530134661F3A6
:105DA000C303DBB243F00303CDE906220E950127BE
:105DB00001AD8DF80630089203AE1A9BB9F80000C9
:105DC0008DF80E7004AA09A9CDE90465ADF81CA0F0
:105DD000FDF7A8FD58BB42F60813ADF80C30637808
:105DE0008DF80430A3788DF80530034667F342033D
:105DF0008DF806301A9A98F800308DF8003098F82F
:105E00000130CDF81A00ADF81E008DF8013032F8DF
:105E1000080B8DF80E70022304A9CDE90465ADF8D6
:105E20001830ADF81C30CDF820D0FFF787FF10B048
:105E3000BDE8F087A1DF704708B5FAF7E1FA10B1C5
:105E4000774B784A1A60FAF7BBFA28B1764B774A53
:105E50001B68C3F342331360FAF7D2FA20B1744AD5
:105E6000D36823F08073D360FAF7AAFA40B14FF0F9
:105E700080430022C3F80C21C3F81021C3F8382551
:105E8000FAF7BEFA10B16B4B03221A60FAF7B8FAB0
:105E900040B1694B05221A6001229A6700229A607C
:105EA0003F225A60654B1B78062B50D1644B1B6810
:105EB00019074CD1634B1B6803F0F003502B46D1FC
:105EC0004FF08052604BD2F80414C3F82015D2F87A
:105ED0000814C3F82415D2F80C14C3F82815D2F806
:105EE0001014C3F82C15D2F81414C3F83015D2F8D6
:105EF0001814C3F83415D2F81C14C3F84015D2F89E
:105F00002014C3F84415D2F82414C3F84815D2F865
:105F10002814C3F84C15D2F82C14C3F85015D2F835
:105F20003014C3F85415D2F83414C3F86015D2F8FD
:105F30003814C3F86415D2F83C14C3F86815D2F8C5
:105F40004014C3F86C15D2F84424C3F87025FAF74E
:105F500037FA28B13D4B3E4A1B6803F04F031360EC
:105F60003C4AD2F8883043F47003C2F88830BFF35B
:105F70004F8FBFF36F8F4FF01023D3F80C22D2074F
:105F80001ED5354B0122C3F80425D3F80024002A7E
:105F9000FBD04FF01022D2F80C3223F00103C2F8EC
:105FA0000C322D4B1A46D3F800140029FBD00021E7
:105FB000C3F80415D2F80034002BFBD004F0ACFE7B
:105FC000D3F80022002A03DBD3F80432002B23DAB3
:105FD000214B0122C3F80425D3F80024002AFBD06A
:105FE0004FF010221521C2F80012D3F80024002A25
:105FF000FBD04FF010231522C3F80422164B1A468B
:10600000D3F800140029FBD00021C3F80415D2F8FE
:106010000034002BFBD0D1E7104B114A1A6008BDA9
:1060200074C007400DF0ADBA440200103C050040BA
:10603000F0ED00E0A005004010560040E00F00F039
:10604000E40F00F0E80F00F000C00040580200101C
:10605000E40E004000ED00E000E00140A42C002030
:106060000090D00370478DDF704777DF7047D0E92D
:106070001F32816F1A44D0F88430C0F880200B445E
:1060800090F82110C0F88430C9B1016F002ABCBF5C
:106090005218C0F88020D0F880208A42A4BF521A3B
:1060A000C0F88020426F002BBCBF9B18C0F8843022
:1060B000D0F884309342A4BF9B1AC0F88430704754
:1060C000D0F88030C0F88830D0F88430C0F88C30F8
:1060D00070470368C91A436870B5D21AD0E91E63C5
:1060E00002FB03F4724301FB064501FB1322D0F8C7
:1060F0008040D0F884302C441A44C0F88040C0F866
:10610000842070BD01381F289DBF034B23FA00F087
:1061100000F00100002070478B80808030B551EC8A
:10612000100B85B053EC112B8DED000B55EC124B81
:106130008DED021B2DF0E8F99DED000B28B19DEDD2
:10614000021BB0EE410AF0EE610A53EC102B204620
:1061500029468DED000B2DF0D7F99DED000B08B110
:1061600045EC104B05B030BD38B555EC104B002256
:10617000002310EE100A29462DF0C6F910B105F1E2
:1061800000431D4645EC104B38BD00002DE9F04F93
:1061900089B00E4600AF0023044607F114013046D3
:1061A0007B6126F075FC05465EB318BB304624F0D3
:1061B000E3F9804678611FF03DFC08F58073834267
:1061C0000CD9A949012020F09FFF3246A7490120A0
:1061D00020F09AFF2437BD46BDE8F08F08F1070391
:1061E00023F00703ADEB030D6D46424629463046CA
:1061F00024F0E6FA7E693EB99D49012020F084FF33
:10620000E8E70028F6D1E0E74FF00308B6FBF8F323
:1062100003EB43039E4201D09649EEE720461CF073
:1062200067F908B99449E8E7944BC7F808D004EB3C
:1062300044041C446378924C2179002940F00B817E
:10624000904A0120C2F80415FF2BC2F82415C2F8A9
:106250002015C2F81C05C2F82815C2F818154FF011
:10626000C051C2F81415C2F810054FF0A04118BF74
:1062700003F5E070C1F85887C1F8FC8A18BF41F8EF
:1062800020804FF01601C2F864154FF0FF01C2F8EC
:10629000681508BF4FF0FF334FF0FF31C2F86015AB
:1062A0002520C2F87035C2F86C15774B23600221A7
:1062B000FFF71AF8012323710323B6FBF3F39BB214
:1062C00003EB430808F1010828F001029100ADEB4F
:1062D000010D6846FA606D4A3A6041184FF0000CB3
:1062E000796082F800C0E91C4FF0EE09851C4FF080
:1062F000880A4FF08E0B63455FDC0C2202FB030320
:1063000000227968994200F29E802679012E40F0A1
:10631000A28000F06043B3F1005F40F0A280FB6810
:10632000C3F34E02574B0021C3F85025C3F838156C
:10633000C3F80815C3F84005C3F80C656579E28019
:1063400025F0090545F008056571C4E90210C3F898
:106350000065022323710D46002977D04FF6FE72A7
:1063600008EA0202F9F7DEF8494B00221A601B68BE
:10637000FB61FB69474B1A601B68BB61BB69414B02
:106380002222C3F8042301221A603A681278042AF0
:10639000FBD94149002222250120C3F80853086097
:1063A000C3F80025C3F808530860C3F800253B4B29
:1063B0002021C3F88410227150E011F8026C11F80A
:1063C000032C360246EA024611F8012C05F10C0EA8
:1063D000164306F44012B2F5001F1ED0B2F5401F5E
:1063E00020D0B2F5801F20D105F802BC06F440028F
:1063F000B2F5000F1CD0B2F5400F1ED0B2F5800FE1
:106400001ED105F801BC0235AE454FEA0616E0D1B3
:106410000CF1010C033175466DE76FF0170205F8BA
:10642000022CE3E705F8029CE0E705F802ACDDE7A3
:106430006FF0170205F8012CE5E705F8019CE2E78B
:1064400005F801ACDFE703F8012B5AE701462368A2
:106450002846984788E70820FBF754FBD7F808D070
:10646000B8E61020F8E700BF98530500BF530500B9
:10647000EB5305000B54050036540500CC3C0500D9
:1064800004A000200050024081210300F6A6002055
:1064900004510240145102400450024000E100E067
:1064A000024B03495868002227F0A6B9602D00204E
:1064B0005673050070B500221049054627F09CF977
:1064C00027F0D4FC0E4B0F4906460322586827F0EC
:1064D00093F9044630B10022B1B227F0D0F820463B
:1064E00025F024FE084B186824F04BFC00210446DC
:1064F000284610F075FE204670BD00BF1749050004
:10650000602D002024490500CCA6002010B5838A08
:10651000C3F30C0413F4604301D1204610BDB3F55E
:10652000005F02D106206043F8E71B0407D5002274
:106530000449006827F060F927F098FCF3E7002091
:10654000ECE700BFC551050008B540B2FFF78DFD6F
:1065500040F2EA71BDE8084012F0DCB938B50546F2
:1065600008460C4624F0AEFE002808BF0024224650
:106570000F49284627F0FCF80E4B4FF6FF7219889A
:1065800084B18A4206D1002040F63551BDE838403A
:1065900012F0C0B900221888114612F001FB082839
:1065A000F2D1F0E78A42EED0188812F0F7FAF6E757
:1065B00000490500BE2C0020014B188810F00ABFCE
:1065C000BE2C0020014B188810F004BFC02C002006
:1065D00008B5084B1A884FF6FF71914209D0188808
:1065E0001321FEF79BF94FF4F171BDE8084012F05A
:1065F00091B908BDC02C002007B50023084607222A
:1066000069460093CDF80330FAF73EF90A4B1A8831
:106610004FF6FF7191420BD018886A46012112F0A3
:10662000C1FA40F6DF3112F075F903B05DF804FBF2
:1066300043F20200F5E700BFBE2C002038B500226F
:106640000E49054627F0D8F80446A8B90C491EF0B3
:10665000EDFC0A4904460246284627F089F82A46F6
:106660000849204627F084F8002025F043FC06491D
:106670000246204627F093F8204638BDB74805006B
:10668000BC480500D6480500F6480500F8B50446A4
:1066900028B9244A136823F480431360F8BD2249C3
:1066A00025F0C2FF0028F4D1204624F031FE054633
:1066B000A0B11C4A1368204643F48043136028F0BD
:1066C0005DF853EC102B10EE100A194615F044FA41
:1066D00040F6E121BDE8F84012F01CB9204624F054
:1066E000D6FD0028DAD00F4A1049136843F48043DE
:1066F000136020462A4627F07FF828F02DFB2A4613
:1067000006460F4620460A4927F076F828F024FB73
:1067100002460B463046394615F01EFA40F6E72190
:10672000D8E700BFD0A60020994C05009E4C05007C
:10673000AA4C0500084B1A6818B142F400521A60BE
:10674000704722F400521A60044B1860044B012277
:106750001A7010F009BD00BFD0A60020FCA60020D2
:10676000F8A6002010B5044624F0ACFD094B0A49F8
:10677000002808BF00242246186826F0F9FF201CD4
:1067800018BF012011F04CF840F2CC71BDE8104068
:1067900012F0C0B8602D0020004905002DE9F74F28
:1067A000464B474907460322586827F025F8064616
:1067B00000283CD000224349DFF80881384627F002
:1067C0001BF83146814668461FF09AFC009CF4B1E4
:1067D000204626F0A1FD00224146054627F00CF890
:1067E0000123002249468246F9F724FF10BBB5F881
:1067F0000B3003F50073A5F80B302C4650462946A4
:1068000026F0EFFC68461FF06AFC002CDED00098F2
:1068100025F08CFC3946002C4CD001A81FF070FCF0
:10682000019D4DB932464946204626F0CDFC03B0C5
:10683000BDE8F08F0024E1E7B5F80B3003F50073F5
:10684000A5F80B30284626F067FD012229460746A9
:10685000204627F057F91C498046284625F0E4FEDB
:106860001A498246284625F0DFFEBAF1000F00D112
:1068700070B1404626F050FD8346B0B1BAF1000F2A
:106880000FD00122394627F00BFD584625F04EFC6B
:1068900040463A46294626F097FC01A81FF01FFC07
:1068A000BEE7394627F077F9EFE73946404626F04C
:1068B000D9FBEDE7304626F099FEB3E7602D0020C6
:1068C0004D4A0500A74B0500544A05005D4A0500E6
:1068D000F8B5054608460C4624F0D9FC0646D8B162
:1068E00000222B49204626F087FF27F0FBFC0022E0
:1068F00006462849204626F07FFF044698B124F03A
:10690000BDFC80B9204625F011FC22462249032017
:10691000BDE8F84020F0F8BB2CB122461F49032007
:1069200020F0F2FB3446284624F0CCFC40B33DB3C3
:1069300048F248011A4825F0C3FA074688B12246B2
:10694000002127F0EBF92A461649384626F010FFB9
:10695000154B164918683A4626F00AFF384625F0C6
:10696000E5FB281C314618BF012010F083FF40F2E0
:10697000DC6111F0CFFF2046BDE8F84025F0D6BB22
:10698000094B0A49186827F02BFB0025E9E700BFEF
:10699000C04C0500694B0500C74C0500FB4C0500C9
:1069A000F96E0200144D0500602D0020194D050000
:1069B0002DE9F84380460C4624F084FC30B92F4979
:1069C00042460120BDE8F84320F09EBB204624F05B
:1069D0009FFC05462046C5B127F0D0FE57EC106B52
:1069E000002432463B46304639462CF0B5FD30B9DE
:1069F0000022234B304639462CF086FDC8B1214990
:106A00000120BDE8F84320F07FBB24F040FC50B1EA
:106A10002A461D49204626F0EFFE40B128F09CF999
:106A200006460F46DDE714B122461849C9E7184F5C
:106A30000026184DD5F8049025F04CFA1649024668
:106A4000484626F0ACFE42461449686826F090FE9F
:106A50000821134825F034FA054628B12146FFF7EE
:106A600037FF284625F062FB32463B460D481BF0B7
:106A70005DFBBDE8F84325F059BB00BFE3490500C5
:106A800000002440344A05003C4A0500114A050034
:106A900000409F40602D00204D4A0500444A0500FB
:106AA0009D670200A96A020037B5144C0021084610
:106AB000FFF70EFF03221249606826F09DFE0022B8
:106AC00001901049606826F097FE0D490546606800
:106AD00027F086FA0B49606827F082FA019B33B1F0
:106AE0002DB1012301AA294600201BF037FB2946BE
:106AF000019826F076FB03B030BD00BF602D00206A
:106B00004D4A0500444A05001FB54FF08052D2F8A7
:106B1000A430D2F8A820D8B20290C3F30720019085
:106B2000C2F30721C3F3074000901B0ED2B241F01D
:106B3000C001034825F098FE05B05DF804FB00BFD6
:106B4000694A050038B525F0C8F91E4D0446286885
:106B500025F0D8F91C490246204626F020FE686838
:106B600025F0D0F919490246204626F018FEA868FB
:106B700025F0C8F916490246204626F010FEE868BE
:106B800025F0C0F913490246204626F008FE286980
:106B900025F0B8F910490246204626F000FE686943
:106BA00025F0B0F90D490246204626F0F8FD287E72
:106BB00025F0A0F90A490246204626F0F0FD2046BD
:106BC00038BD00BFDCA60020A7520500FB4F050022
:106BD000AA520500AE520500B2520500B652050099
:106BE000BA5205002DE9F04786B00D46014601A8CE
:106BF0001FF086FA019838B90446019825F096FAF4
:106C0000204606B0BDE8F08726F086FB00229949B1
:106C1000064626F0F1FD0746002800F0E18000223C
:106C20009449284626F0E8FD3946804602A81FF020
:106C300067FA01240298002840F0A18041463846B6
:106C400026F0CFFA00228C49304626F0D5FD0746C3
:106C5000E0B100228849284626F0CEFD804638461D
:106C600024F080FC002800F0BD80404624F07AFC2F
:106C7000002800F0B7804146384625F0D5FF0028AF
:106C80004146384608BF002426F0ABFA00227B4973
:106C9000304626F0B1FD074610B30022764928465B
:106CA00026F0AAFD8046384624F013FC98B14046F1
:106CB00024F00FFC78B1384625F09FFE814640460F
:106CC00025F09BFE814506D8012300224146384627
:106CD000F9F7B0FC00B100244146384626F081FAAD
:106CE00000226749304626F087FD074680B1002222
:106CF0006349284626F080FD01468046384625F047
:106D000093FF41460028384608BF002426F069FA60
:106D100000225C49304626F06FFD804670B124F0B9
:106D2000B6FA40B1414605A81FF0EAF9DFF85491E0
:106D3000059F002F62D1404625F0F8F90022524904
:106D4000304626F059FD804670B124F0A0FA40B1DB
:106D5000414605A81FF0D4F9DFF830A1059F002FA8
:106D60006CD1404625F0E2F9304625F0DFF901A864
:106D70001FF0B5F9002C3FF43DAF01243DE7B8F119
:106D8000000F10D026F0C8FA014603A813F04CF803
:106D9000414604A81FF0B4F94FF00009049838B92F
:106DA000B9F1000F00D1002402A81FF098F941E7C3
:106DB00026F0B2FA014605A813F036F89DF8162021
:106DC0009DF80E309A4207D1BDF81420BDF80C3062
:106DD0009A4208BF4FF0010904A81FF080F9DDE7CF
:106DE00001242FE7384624F0EDF88146404624F090
:106DF000E9F8A9EB00035842584140E7B7F80B30D7
:106E000003F50073A7F80B3000224946284626F008
:106E1000F3FC824680B10022394626F073FE00283A
:106E200008BF002425F082F93846514626F0D9F9EA
:106E300005A81FF054F97BE70446F5E7B7F80B30D7
:106E400003F50073A7F80B3000225146284626F0C0
:106E5000D3FC81460146384625F0E6FE4946002827
:106E6000384608BF002426F0BCF905A81FF037F902
:106E700074E700BF544A0500B5490500BA4905004A
:106E8000A74B05005D4A0500C5490500D649050028
:106E900073B505460E4624F0F1F938B915490320BB
:106EA00020F032F90024204602B070BD304624F0B4
:106EB000E5F90028F2D025F00DF804460028F2D0BC
:106EC000294601A81FF01CF901980028EBD026F0F4
:106ED00023FA054601463046FFF784FE18B12946DD
:106EE000204626F083FB284625F020F901A81FF054
:106EF000F6F8E9E78F4905002DE9F04F87B000AFBC
:106F0000C7E902011446002A6CD0914900201EF006
:106F10008DF80022054638618E49204626F06CFC2B
:106F20008C490246284626F03AFC00228A493D69EF
:106F3000204626F061FC88490246284626F02FFCB0
:106F400024F0C8FF804624F0C8FF0022824683490F
:106F5000204626F051FC8146E8B102467F49386957
:106F600026F006FC002307F1140148467B6125F05A
:106F70008FFD0446002844D1484623F0FDFA05461B
:106F800078611EF057FD05F5807383422ED9744950
:106F9000012020F0B9F8B8F1000F07D0D8F8003080
:106FA00023B142466F49386926F0E2FB504625F08E
:106FB00046FD20B152466C49386926F0D9FB52464D
:106FC0004146484626F000F9FB68002B40F0B780A8
:106FD00007F1100301220021B8681CF0E7FC3869B2
:106FE00025F0A4F81C37BD46BDE8F08FEB1D23F05B
:106FF0000703ADEB030D6C462A462146484623F0B5
:10700000DFFB7B69002BC6D0B8F1000FCED0BAF100
:10701000000FC0D0002514E0092A09D1A91C214481
:10702000701ED7F810B025F07BFF5049024619E0DA
:10703000911E012927D89B4602239E4216DA01366B
:1070400035447B69AB42A6D96319665D5A78082A34
:10705000E2D1A91C2144701ED7F810B025F060FFC2
:1070600043490246584626F09AFBE8E73BF8021FE0
:1070700040487B6025F0F8FB0146404626F0CFFAF9
:107080007B680233D9E7911F012908D8A81C204446
:1070900013F050F90146404626F0C1FACFE7162A10
:1070A0002BD0212A32D1A81C204413F043F91223FB
:1070B00083463B60BBF1000F1BD00122594650466E
:1070C00026F020FD3B6878605919701CC01A2144D5
:1070D00023F030FE7A6803463AB130B10146386099
:1070E000104625F0BFFFD7E900321946104626F0BA
:1070F00078F8584625F01AF8A1E759881D4825F078
:10710000B3FB28F02FF804238346D2E7FF2A96D159
:10711000D8789B78D7F810B043EA002024F0F2FE2C
:1071200015490246584626F03AFB291D2144F01E17
:10713000D7F810B023F0FEFD1049024692E7D7E9D8
:107140000301FFF74FFD00287FF442AF47E700BF80
:107150008A4D0500A74B050006490500BA530500F6
:1071600098530500544A05005D4A0500B5490500DD
:107170009A4D050013720500D6490500C549050062
:107180002DE9F04186B000AF00238846391D044642
:107190007B6025F07DFC0546002C38D0E0B9204608
:1071A00023F0EAF9064678601EF044FC06F5807389
:1071B000834206D9414901201FF0A6FF22464049DB
:1071C0003BE0F31D23F00703ADEB030D6D463246A4
:1071D0002946204623F0F4FA7B68002BEED0404687
:1071E00024F070F828B1374B37491868424626F02A
:1071F000BFFA364B1A6812F0400F1E460AD13449C6
:1072000001201FF081FF1837BD46BDE8F08100283E
:10721000E2D1D3E72F4A12884FF6FF71914201D194
:107220002D49EDE71A6812F0800201D02B49E7E7FB
:107230007C68102C05DD2A49102201201FF064FF14
:10724000E1E7284B93F800C0274BA4B2BCF1000F34
:1072500025D19A7C72B3B3F8760188422CD09B8AF0
:107260007C80C7F80AC0A7F80EC03B810123BB721F
:1072700007F10801BB1CC7E90435FCF751FB18B93D
:107280007B88A34218BF0C2040F6BB3111F042FBB3
:107290000028B8D1336843F080033360B3E7B3F814
:1072A0007601884208D07C80C7F80A20FA81B3F8BA
:1072B0004E31DAE70720E7E70820E5E798530500B5
:1072C000104C0500602D0020A04B0500D0A600202A
:1072D000AA4B0500C02C0020BE4B0500CD4B05007D
:1072E000E54B0500F7A6002048A200202DE9F04F4D
:1072F0009D4B91B01B681B0700AF044607D59B4907
:1073000001201FF001FF4437BD46BDE8F08F14F0A7
:107310009DFC204623F0BBFF0546002800F01A81A3
:10732000214607F114001EF0EBFEDFF864A2796934
:1073300089B10023BB61B1F80B3003F50073A1F8EC
:107340000B3007F1180012F06FFD024638B1884982
:1073500001201FF0D9FE786924F0E8FED3E7D7F8C2
:107360001480B8F1000F03D0404625F0D5FF8046C9
:10737000414607F11C001EF0C3FEF96985B179B1E1
:10738000B1F80B3003F50073A1F80B3007F12000C2
:1073900012F04AFD024670B1764901201FF0B4FE9A
:1073A000F86924F0C3FE404624F0C0FE07F1140043
:1073B0001EF095FEBBE707F128003C8C97F8226091
:1073C00013F0C0FC08B1FAF79DFB4FF00009002252
:1073D00007F13001388DC7F8309013F0B1FC052863
:1073E00010D043F2030290420CD0A8B93B8EA342C6
:1073F00014D197F83230B34210D1B7F82890B9F1D0
:10740000000F0FD1386A12F0ABFF5B490446024609
:1074100001201FF079FE3EE0FAF774FB3B8D01334B
:107420003B85D4E7FC691CB1204625F075FF044676
:1074300000225249204626F0DFF900225049064634
:10744000204626F0D9F926F04DFF0022B8604D49BC
:10745000204626F0D1F926F045FFF860C6B100239A
:1074600007F1240130467B6225F012FB834620BBE6
:10747000304623F081F8786278601EF0DBFA7A6893
:1074800002F5807383420ED93F4901201FF03CFE74
:10749000304624F04BFE204624F048FE07F11C0045
:1074A0001EF01DFE69E7D31D23F00703ADEB030DAE
:1074B000EB465946304623F083F97A6A002AE7D032
:1074C000002179853A85494607F12802BAF800007B
:1074D000C7F82CB0FEF730FC40F2915111F01AFAC7
:1074E000BB6880F00100C5B213B9FB68002BCFD098
:1074F000BAF800204FF6FF719142C9D0FB68BAF884
:107500000000A7F830900022002BC7F83220FA863E
:107510007A6A7A8214BF0222012287F8322007F1A8
:10752000300107F11202C7E90E2BFCF7F9F930F030
:107530000802ADD043F204029042A9D043F20142C6
:107540009042A5D040F2A65111F0E4F9002818BFEE
:1075500000259DE7002C3FF4D6AE22460B490320C0
:107560001FF0D2FDCFE600BFD0A600203A4E0500A6
:10757000624E05007B4E0500AB4E050056540500DB
:107580009B4E0500A24E050098530500CF4E050006
:10759000C02C00202DE9F04F9BB000AF0D460446F3
:1075A0003C22002107F12C00F7F7BCFF022387F8EB
:1075B0002C302846062387F82F3023F068FE002859
:1075C00079D000228449284626F016F938B126F0F1
:1075D00089FE002814BF0223002387F82C300022E4
:1075E0007E49284626F008F938B126F07BFE0028AF
:1075F00014BF0623052387F82F3000227849284638
:1076000026F0FAF88146D0B1002307F10C01FB60A7
:1076100025F03EFA064600283CD1484622F0ACFF51
:107620008046F8601EF006FA08F58073834225D97B
:107630006C4901201FF068FD484624F077FD28467C
:107640000022694926F0D8F8054640B13B6D6BB37E
:1076500025F078FE3B6D1880284624F067FD204613
:1076600023F00CFE80B3B4F80B3003F50073A4F8DC
:107670000B3020466C37BD46BDE8F08F08F107039C
:1076800023F00703ADEB030D6E46424631464846F4
:1076900023F096F8FA68002ACED084B06B464FF6F5
:1076A000FF713B6519809A809E60C5E74F490320B2
:1076B0001FF02AFDD0E7002DD1D04D492A460320E6
:1076C0001FF022FD0024D4E7204623F0BAFD054632
:1076D0000028C8D1204623F0DAFD002876D02046C5
:1076E00024F0F2FE0C235843073020F00700ADEBE6
:1076F000000D214607F108001EF002FDE846DFF804
:10770000E4A04446A946B868F8B987F85850C7F8C5
:1077100054801F2307F1080207F10C0107F12C0028
:107720003B81FDF7A3F918B1324B5B68002BC9D040
:1077300040F2F63111F0EEF80028C3D107F10C0148
:10774000388923F0F7FA044693E725F0E5FD07F1C1
:107750000C018346C7F80C9025F09AF90646BBF158
:10776000000F10D078B9584622F006FFF860786014
:107770001EF060F97A6802F5807383421BD9514686
:1077800001201FF0C1FC584624F0D0FCB86828B195
:10779000B0F80B3003F50073A0F80B3026F066FB51
:1077A000FB682080A380A66007F108001EF097FC0C
:1077B00001350C34A7E7D31D23F00703ADEB030D10
:1077C0006E463146584622F0FBFFDCE7002CA0D085
:1077D0002246094973E700BF874A0500904A050021
:1077E000C549050098530500D64905009D4A050086
:1077F000D14A0500602D0020074B050008B5064A58
:10780000136823F40073136012F018FB40F20B218D
:10781000BDE8084011F07EB8D0A6002008B5054AA2
:10782000136843F40073136010F04AFFBDE808408A
:10783000FEF7CEBED0A6002008B511F0F9F941EC54
:10784000100B08BD10B50F4B1B884FF6FF729BB293
:107850009342044603D10C4A1288934208D00B4845
:107860001AF0EAFC0A4A136843F00803136010BDDB
:1078700023F028FD002814BF20460020BDE810405A
:1078800010F024B8BE2C0020C02C0020714B050045
:10789000D0A6002010B5044623F0F9FC224630B9EA
:1078A0002CB10B490320BDE810401FF02DBC094B43
:1078B0000949586826F0A5FB11F040F8074B1B68F2
:1078C0001B0704D50020BDE81040FFF7BBBF10BD6B
:1078D000A44D0500602D0020CD4D0500D0A6002050
:1078E00038B5104C104900220546606825F084FF29
:1078F00026F0BCFAC3B285B143F0010098420FD024
:10790000646824F0FFFA08490246204625F047FF44
:107910000020BDE83840FFF795BF03F0FE00EDE71B
:1079200038BD00BF602D0020B64C05002DE9F041A8
:107930008CB00646884623F0AAFC40B93EB13246D8
:10794000474903201FF0E0FB0CB0BDE8F0810023A5
:1079500002930193434B039302AB0593424B06936F
:1079600003270B23ADF81C300DEB0703012208930E
:107970003E4B8DF8032009933A4601AB03A94046DC
:10798000ADF81070ADF828700B9326F069FF002851
:10799000DAD00298364D374C23F0C8FD48B1029A30
:1079A0003549686825F0E4FE236843F00803236046
:1079B00009E0029B002B37D12F49686826F010FBA5
:1079C00023685906F0D4029824F0B0FB9DF80330E8
:1079D000002B2ED02368294968689A065EBF236869
:1079E00043F00803236026F0FBFA32462449686816
:1079F00026F007FB42462349686826F002FB019AFD
:107A00001AB1236843F0080323601F49686826F011
:107A1000F8FA019824F08AFB236813F0180F1BD0A2
:107A20000020FFF70FFF8FE7184938461FF06CFB67
:107A3000C9E723686F689B0648BF23684FF00000C2
:107A400044BF43F00803236024F054FA0B49024674
:107A5000384625F0A4FEC8E730460FF035FD73E741
:107A6000CF4E0500A64B0500D54D0500DA4D0500AB
:107A7000602D0020D0A60020E44D0500134E050027
:107A80001C4E0500264E0500304E0500EE4D05004B
:107A900013B56946044612F0C1FB28B90749012015
:107AA0001FF032FB02B010BD054B06495868224654
:107AB00025F05EFE0020FFF7C5FEF3E7284C050029
:107AC000602D00205E4C050038B50A4C05462DB9E6
:107AD000094B002C08BF1C46204638BD3CB120464F
:107AE0002BF0EEFF013D01300444EDB2EFE7024C14
:107AF000F2E700BF0A480500FAB1050070B50D4C69
:107B0000064620780D4640B1FFF7DEFF0A490246DF
:107B100001201FF0F9FA002070BD09F057F8074B5B
:107B200026701860284623F02CF9054B18600120B8
:107B3000F2E700BFD4A6002094480500CCA60020A0
:107B4000D8A6002037B50546002105208DF806107F
:107B5000FFF7D4FF58B1074B186823F012F90199C9
:107B6000044628460FF0AAFB204603B030BD044669
:107B7000FAE700BFCCA6002037B505460C46052025
:107B80000021FFF7BBFFB8B1214601A812F0B6F8FB
:107B9000024638B1094901201FF0B6FA00242046F8
:107BA00003B030BD064B186823F0EBF8019904468A
:107BB00028460FF083FBF2E70446F0E7984E0500F5
:107BC000CCA6002013B5002104208DF80610FFF785
:107BD00095FF50B1064B186823F0D3F8044601987E
:107BE0000FF0B2FB204602B010BD0446FAE700BF1A
:107BF000CCA6002013B50C4604200021FFF77EFF21
:107C0000B0B1214601A812F079F8024638B109490D
:107C100001201FF079FA0024204602B010BD064B67
:107C2000186823F0AEF8044601980FF08DFBF3E7D7
:107C30000446F1E7984E0500CCA600202DE9FF414F
:107C4000002288462649064625F0D6FD0022254911
:107C5000074625F0D1FD6946054612F0DFFA0446D5
:107C600058B92946384625F0BCFA1F4903201FF0B1
:107C70004BFA204604B0BDE8F081384624F056FAAD
:107C800000221A49304625F0B7FD26F02BFB0746A7
:107C900020B1304608F0FAFF0446EAE731460220F8
:107CA000FFF72CFF20B90024284624F03FFAE0E734
:107CB00048210F4824F004F904460028F3D0014677
:107CC000022302AA3846CDE902581AF047FA2046A4
:107CD00024F02CFA074B186823F053F80446E3E726
:107CE000D6480500A74B05004B490500F64805009E
:107CF000B1B10200CCA6002070B504460E460020AB
:107D00000E491DF093F9054610B90025284670BDAF
:107D100022460B4925F02CFD2846FEF78FFC044631
:107D2000284624F003FA002CEFD031462046FFF716
:107D300085FF0546204624F0F9F9E7E78A4D05005E
:107D4000A74B050070B5064650B123F0A0FA0446D3
:107D500030B92849324603201FF0D6F9204670BDBD
:107D600000222549304625F047FD054623F086FAD6
:107D70000446284624B924F0D9F92A461F49EAE7DF
:107D800024F0D4F900221E49304625F035FD26F0B6
:107D9000E3FF02460B4604460D462BF0DDFB30B9EF
:107DA00000220023204629462BF0B8FB08B1154DD0
:107DB00000242B46224614481AF0B8F9054601461D
:107DC0000120FFF79BFE78B10821104824F078F8D5
:107DD000044628B13146FEF77BFD204624F0A6F983
:107DE0000B4B186822F0CDFF0446284624F09EF97C
:107DF000B4E700BF344B0500694B0500C74C0500D4
:107E00003C4A050000409F4059AE020005B3020005
:107E1000CCA6002029F06CB82DE9F04F2DED028B97
:107E2000A3B08B46154624F055F88246002800F092
:107E3000C080584623F07AFB002800F0BA8028461C
:107E400023F025FA002800F0908008AA1892804AB2
:107E5000199206AA1B927F4A7F4B1C9204AADFF854
:107E6000049216931E920A237C4AADF85C300026D9
:107E700000274FF00008ADF86830ADF874301F925D
:107E8000ADF88030042202AB16A92846CDE9086778
:107E9000CDE90667CDE90489CDE90267219326F093
:107EA000DFFC002800F085809DED028B32463B46CA
:107EB00051EC180B2BF01EFB002851D1B0EE480AF4
:107EC000F0EE680A28F024FF53EC102BB0EE480ABD
:107ED000F0EE680ACDE9002329F00AF8DDE9002375
:107EE00055EC104BDDE90467304639462BF09AF823
:107EF0003246804689463B46204605F10041CDE9A1
:107F00000A892BF08FF8DDE90823CDE90E01CDE9D0
:107F10001223304622462B4639462BF083F8DDE902
:107F20000623CDE90C01CDE91089CDE91423012206
:107F3000594616A81FF013FB16A81EF099F858B161
:107F400016A81EF025FA064616A80F461EF0ABF935
:107F500016A81EF08DF890BB16A81EF05DF828E05C
:107F600034463D4642464B46BCE7284623F0DEFAFF
:107F7000C8B1284624F063FD0628044613D12946DB
:107F8000012216A81FF0EBFA0AAD16A81EF000FA9F
:107F9000E5E8020116A81EF086F9013CF5D116A805
:107FA0001EF03AF8C3E72E4903201FF0ADF84FF05A
:107FB000000A504623B0BDEC028BBDE8F08F16A836
:107FC0001EF0E6F9044616A80D461EF06CF9DDE930
:107FD0000A23304639462BF025F8DDE90E2380468A
:107FE0008946204629462BF01DF802460B4640469E
:107FF00049462AF061FEDDE912232AF05DFE41ECDC
:10800000100B23F06DFF0146504625F008FBDDE91B
:108010000C23304639462BF005F8DDE910230646DF
:108020000F46204629462AF0FDFF02460B46304601
:1080300039462AF041FEDDE914232AF03DFE41ECE9
:10804000100B23F04DFF0146504625F0E8FA73E788
:1080500087770500005305005D770500065305008E
:108060000D5305000000F03F2DE9F04F93B00C4692
:10807000164623F02FFF0546002800F08480002CD0
:1080800000F081802368062B7DD12146012207A8BC
:108090001FF065FA01AF002407A81EF0CEF90134E5
:1080A00047F8040B07A81EF0FEF8062CF4D107A829
:1080B0001DF0B2FF304623F0EAF830B10022354916
:1080C000304625F099FB25F0D1FEDDF80480059EB1
:1080D000DDF80890069FB8EB060448BFA6EB08043D
:1080E000B9EB070348BFA7EB09039C42A8BF1C4696
:1080F000002C08BF01244FF4A04393FBF4F4B4F523
:10810000805F44DA40F299139C42B8BF1C460028B5
:10811000C8BF4FF480544A46C8BF94FBF0F44146B0
:10812000284625F086FAC4F5805BA2460BFB0BFCC3
:108130000AFB0BF04FEA2C3C049A40F3D3200CFBD3
:1081400009F302FB0032039B0AFB0AF10CFB08FC5B
:1081500003FB00C3091301FB072201FB063102F5F3
:10816000006201F50061121309132846A24425F0AC
:1081700060FABAF5805FABEB040BD7DD3A463146C7
:10818000284625F056FA284613B0BDE8F08F40F295
:108190005554BCE7FB5105002DE9F04F9BB001465B
:1081A00009A813F081F828B90023039303981BB0A2
:1081B000BDE8F08FBDF829309DF82F40DB06A4F113
:1081C000020347BFBDF82D70BDF82B60BDF82B70C2
:1081D000BDF82D60012B70D9082CB8BF082407FB0F
:1081E00004F31F33082C4FEA6313D8BF4FF0010983
:1081F0004FEA83030093D4BF09FA04F94FF0000952
:10820000009B09EB490505F11A0803FB068A504655
:1082100023F040FD03900028C6D023F09FF84223AE
:1082200003704D2343700C2383733B1280F802A02C
:10823000C3744FEA2A2A33124FF0010E082C80F83B
:1082400003A080F80A8087740675437580F816E0ED
:10825000047634DD0123A340013B0693009A0823F2
:10826000B3FBF4F30193E3100593731E02FB035574
:10827000431902934FF00008B04597DA08F1010363
:108280000493029B072C03F11A0547DD4FF0000908
:10829000B94549DA4246494609A812F0B6FF2A46CE
:1082A000002308339C4202F8010B4FEA1020F8DC4F
:1082B000059B09F101091D44EAE704248FE79DF8B5
:1082C0002F30032B00F11A0315D000219DF82F2029
:1082D0000EFA02FC8C4503F10303BBDDC1EB012266
:1082E00092FBFCF2D2B203F8032C03F8022C03F841
:1082F000012C0131EAE700224A4503F10303A9D02A
:1083000042F3000103F8031C42F3400103F8021C8E
:1083100042F3800103F8011C0132EDE7DDF804B0FF
:108320004FF0000ABA451CDB029B009ADDF8108072
:108330009B1A0293A0E74B1C424609A8079312F030
:1083400064FF069B1840079B09FA04F940EA0909F3
:1083500019465945EFD1019B05F8019B9A449B446E
:10836000E0E751464FF00009F3E7000038B5FFF7AA
:1083700013FF054610B90025284638BD0BF03EFB1B
:108380000446284623F0D2FE002CF4D021460448AF
:1083900024F06AFA0546204623F0C8FEECE700BF49
:1083A0000B4F050010B5FFF7E1FF044608B11BF0C5
:1083B00075FA204623F0BAFE0248BDE810401AF0D4
:1083C000A5BD00BF8184050000B593B0014601A89A
:1083D00012F06AFF10B101A8FEF798F813B05DF82B
:1083E00004FB000000B593B0014601A812F05CFF49
:1083F000D8B1BDF8180010F460430AD0B3F5005F9F
:108400000D4918BF00211B0405D429B923F07AFDBA
:108410000BE00A49F7E70A4941F6FE73184207D014
:10842000C0F30C02074824F01FFA13B05DF804FBF8
:10843000084624F0CDFDF8E7BB510500B451050016
:10844000F4510500BF51050030B593B00C4601460C
:1084500001A8154612F028FF20B12A46214601A89E
:1084600012F0D3FE13B030BD00B593B0014601A8A1
:1084700012F01AFF08B19DF80F0013B05DF804FB6D
:108480002DE9F041B2B00546884601460CA812F02D
:108490000BFF002800F0D4800BAA1F92694A20929B
:1084A0000AAA2292684A694B239209AA1D9325922F
:1084B0000923674AADF87830ADF88430ADF89030D4
:1084C0002692ADF89C3008AAADF8A830ADF8B430CB
:1084D00006AB28922E935F4A5F4B29922F9307AAEF
:1084E0000B2300242B92ADF8C0305C4ABDF83770E6
:1084F000BDF839608DF817400DF117034046CDE9FE
:108500000A44CDE90844CDE906442C92319322F087
:10851000BEFE40B9524901201EF0F6FD0025284656
:1085200032B0BDE8F08107221DA9404626F098F937
:108530000028EFD00B99099A00290A4404DA079B16
:1085400009925B1A07930B940A98089B002803442E
:1085500005DA06990893091A069100210A91D21B9F
:10856000002AC8BF09990B98C8BF8A1AA3EB060353
:10857000C8BF0992002BC8BF089A0A99C4BFD31A72
:108580000893079B099A002B1A4404DAC31A0B9329
:108590000023099207930698089B0028034404DAF5
:1085A000091A0A91002108930691D71B002FC8BF12
:1085B000099A07990698C8BFD71BA3EB0603C8BF43
:1085C0000997002BC2BF089AD31A0893DDE9082344
:1085D000002B01DC002A2CDDCDE901100092DDF832
:1085E0006B40DDE90A210CA8A0479DF8173003B3C2
:1085F000DDE90610BDF95340099A089BA0420244E8
:10860000B8BFADF85300BDF957008242C8BFADF8FE
:108610005720BDF955209142BDF95920B8BFADF89A
:1086200055100B4493420CA8C8BFADF8593012F056
:1086300017FEB5F80B3003F50073A5F80B306EE7A5
:1086400005466CE7274F050011670500244F05001C
:10865000C26405002A4F0500304F05002D4F05006C
:108660003C4F050030B593B00D46014601A812F00D
:108670001BFE00284CD0BDF92720BDF92B309A42B3
:1086800044DC23F02AFC044618B3BDF9270023F08C
:1086900039FC20490246204625F081F8BDF9290021
:1086A00023F030FC1C490246204625F078F8BDF93D
:1086B0002B0023F027FC19490246204625F06FF8CD
:1086C000BDF92D0023F01EFC15490246204625F079
:1086D00066F8C5B100226FF07F038DF82B208DF86E
:1086E0002C308DF82D208DF82E304FF0FF327F2367
:1086F00001A88DF827208DF828308DF829208DF8D5
:108700002A3012F0ADFD204613B030BD0024E0E762
:108710000446F8E7244F0500274F05002A4F0500BF
:108720002D4F050070B592B004460D46014601A8D4
:10873000164612F0B9FD58B3BDF80930022D23F0EA
:1087400070039BB21ED0032D1FD0012D08BF43F034
:108750003003ADF809304EB1BDF80930DA064CBF30
:1087600083F0400383F02003ADF8093001A812F034
:1087700077FDB4F80B3003F50073A4F80B302046F6
:1087800012B070BD43F06003E3E743F05003E0E74D
:108790000446F4E770B592B004460E46014601A8BF
:1087A000154612F081FD78B101A8ADF81A60ADF858
:1087B0001C5012F055FDB4F80B3003F50073A4F80B
:1087C0000B30204612B070BD0446FAE7F0B593B006
:1087D00004460E46014601A815461F4612F064FDE8
:1087E00008B3012E9DF81E10A8BF0126012DA8BFB9
:1087F000012546EAE67666F3010145EAE57565F38B
:10880000830187F3020767F3051101A88DF81E1095
:1088100012F026FDB4F80B3003F50073A4F80B300A
:10882000204613B0F0BD0446FAE7F0B593B0044615
:108830000F46014601A816461D4612F035FDA0B1AF
:10884000189BADF8253001A8ADF81F70ADF8216078
:10885000ADF8235012F004FDB4F80B3003F50073AB
:10886000A4F80B30204613B0F0BD0446FAE72DE91A
:10887000F0419AB007460D46014609A8144612F089
:1088800013FD4FF000080646002800F09D8006AA60
:1088900005A909A8CDE90754CDE9058812F022FC05
:1088A00008AA07A909A812F01DFC059B079D089CB2
:1088B000BDF84120BDF84310BDF845000791ED1A01
:1088C000069B0890E41ABDF82B3006929D42C8BF63
:1088D0001D46C3F10003C8BF4646AB42C8BF1D4694
:1088E000BDF82D30C8BF00269C42C8BF1C46C3F14E
:1088F0000003C8BF0026A342C4BF1C460026BDF823
:108900003F30059346B1CDE901100092DDF8636078
:108910002246294609A8B047DDE90512BDF947609E
:10892000DDE90730B142BDF94B60B8BFADF8471083
:10893000B342BDF94960C8BFADF84B30B242BDF992
:108940004D60B8BFADF84920B042C8BFADF84D008A
:10895000002D23DD6B180D9DDDF85760CDE9000576
:10896000013B09A8B047002C23DD069A0D9B01931B
:108970001444013CDDF85750079B0094059909A861
:10898000A84709A812F06CFCB7F80B3003F5007388
:10899000A7F80B3038461AB0BDE8F081E3D00D9946
:1089A000DDF8576003F1010CCDE900010CEB050186
:1089B000D7E7E6D0089B0D99DDF857505A1CCDE952
:1089C00000312244079BD9E70746E3E70000000097
:1089D0002DE9F04FCDB005460E46014617A81746C3
:1089E0000293569C12F060FC002800F06783382246
:1089F000002109A8F6F796FD304622F048FC002831
:108A000054D0B049304624F015FF00284ED03146EE
:108A100028A812F049FC002800F0A8809DF8A48046
:108A2000B8F1000F40F0A280BDF8A7300993BDF85F
:108A3000A930A5490A9342469DF8AB300B933046C6
:108A400024F0DAFE064623F00FFE0E90304623F0A7
:108A50006DFBCDF83C809DF8303013B94FF0FF33FB
:108A60000D93109B5BB90B9B012B08D11B9AADF8A2
:108A700054201A9AADF8562015AACDE910230E9865
:108A800022F027FD064648B10999002906DD0A9B18
:108A9000002B03DD0B9B202B40F32C818B49012005
:108AA0001EF032FB0E9823F041FB5FE0304622F0CF
:108AB000EEFB002872D000228549304624F09CFE4F
:108AC00025F0D4F9002283490990304624F094FE21
:108AD00025F0CCF9002280490A90304624F08CFE23
:108AE00025F0C4F90028CCBF0B9001234FF0000201
:108AF0007A49D8BF0B93304624F07EFE031C18BF82
:108B000001238DF8303025F0B1F900220D90744921
:108B1000304624F071FE804688B322F092FB50B3B9
:108B2000B8F80430022B26D1002328A94046289308
:108B300023F0AEFF1090404623F0F8FA289B102B4C
:108B400005D9B3F5807F06D00023109305E0654A70
:108B5000DA40D107F8D5013B1193DDF84080B8F138
:108B6000000F0CD1604901201EF0CEFA00252846E6
:108B70004DB0BDE8F08F404623F0D8FAEDE7002273
:108B80005149304624F038FE064623F06DFD0E9024
:108B9000304623F0CBFA00230F935CE7304622F0F7
:108BA00098FC58B1304622F04CFB70B9B6F80B3047
:108BB0000E9603F50073A6F80B300AE0304622F05B
:108BC00040FB0028EED14949CDE7304623F04CFD6B
:108BD0000E9000210E9823F0F2FD012109900E98CD
:108BE00023F0EDFD02210A900E9823F0E8FD020625
:108BF0000B902CD500F07F0001230B9003210E98E1
:108C00008DF8303023F0DBFD04230D900B9E0F9385
:108C100073067FF520AF06F03F064FF0010808FA13
:108C200006F808F1FF39022E0B96CDF8449028DCA7
:108C3000DDF83C9015AB4FF0000AD04509DC15ABD0
:108C40001093022303FA06F60F9B3344A4E7032391
:108C5000DCE749460E98039323F0B1FD09F10202C7
:108C6000834609F101010E98009223F0A8FD039BB1
:108C7000009A4BEA002023F8020B0AF1010A914600
:108C8000DBE7082E16DC002328A90E982893DDF8D0
:108C90003C8023F0FDFE0B9B082B0BDC50B1022324
:108CA000B340289A434493423FBF0F9BCDF8449072
:108CB000C0181090DDF84080B8F1000FC1D10C4908
:108CC00051E700BFA55005001D570500855105005F
:108CD000AE500500B4500500BB500500BF50050064
:108CE000CB50050014010100D35005005051050080
:108CF0001E51050001229A40013A072B1292DCBF57
:108D0000082292FBF3F203FB01F3D4BF02F1FF321E
:108D1000002207331392DB10DDE90E1204A814932E
:108D20001DF0DBFD002C40F08C80BDF8613013F0AD
:108D3000700F1AD0DFF89CA3029E4FF00008444643
:108D40000A9B029A1344B34279DC079823F0EEF9A8
:108D50000E9823F0EBF917A812F082FAB5F80B3051
:108D600003F50073A5F80B3001E7BDF87700BDF8F7
:108D70007910029B099ABDF87DC08742B4BF344682
:108D800038463A448B42BDF87B30A8BF029902F1C5
:108D9000FF3EB8BF34469E45C8BF9E460A9A029B16
:108DA000134403F1FF33C8BF34466345C8BF63466D
:108DB000BDF97FC0BDF98120C8BF34468445C8BF16
:108DC000ADF87F00BDF98300C8BF34467045BCBF15
:108DD0003446ADF883E08A42BDF98520C4BFADF8C2
:108DE000811034469A4202DAADF88530A2E7002CB1
:108DF000A0D1DDF88BA09FE704A81DF067FC083424
:108E000040EA08280B9BA342F6DC129AE41A28FADF
:108E100004F313400D9A9A4209D0109A1AB111998D
:108E20000B4032F813303246494617A8D04709F1B3
:108E30000109099B3B444B45E4DC013680E7B94618
:108E4000F7E7204622F023FA00283FF47EAF002205
:108E50009D49204624F0D0FC25F07EFF824621F07B
:108E600000498B464FF0FF32984B504649462AF056
:108E700073FB70B94FF0FF32944B504649462AF0CD
:108E800061FB30B900220023504659462AF046FBC8
:108E900018B1DFF844B24FF0000A00228C49204696
:108EA00024F0AAFC25F058FFCDE90001DDE900839C
:108EB00023F000494FF0FF32844B404649464FF0C3
:108EC00001042AF049FB40B94FF0FF327F4B404686
:108ED00049462AF037FB00B9044684F001044FF0FC
:108EE000FF327A4B40464946E4B22AF035FB38B9A6
:108EF0004FF0FF32754B404649462AF023FB18B12C
:108F00009FED6F7B8DED007B029B299309AE0FCE09
:108F1000289731AF0FC70FCE0FC70FCE0FC796E8F8
:108F2000030004AE87E803000FCE3FAF0FC79DEDEF
:108F3000007B33683B6028A80023CDE92EAB8DED84
:108F40002C7B8DF8C0408DF8C130F8F71BFBBDF8C5
:108F50007780289BBDF879402A9F2B9E9845B8BF03
:108F60009846299B9C42B8BF1C46BDF87B30013F08
:108F70009F42A8BF1F46BDF87D30013E9E42A8BF5C
:108F80001E46BDF97F309845BDF98330B8BFADF8B6
:108F90007F809F42BDF98130C8BFADF88370A34286
:108FA000BDF98530C8BFADF881402246B342414685
:108FB00028A8B8BFADF88560FDF78BF8BDF8613023
:108FC00013F0700F0CBFDDF88BA0DFF808A1B442DE
:108FD00006DD3FAE0FCE04AC0FC433682360B4E6A9
:108FE00028A8FDF76DF8C146B94504DD28A8FDF7AE
:108FF0003EF80134EBE74A9A7F322BD44B9B13F1B6
:109000007F0B27D4449B9A4224DA459B9B4521DA67
:109010004FEA222C339A082A4FEA2B2BDDE936102F
:1090200023D13C9A0CEB000302FB0B323FA821F04A
:1090300091F9439B0BB13F9A9B5C359A9A4209D0B8
:10904000389A1AB139990B4032F813302246494602
:1090500017A8D0474A9B469A13444A93479A4B9B7A
:109060009B1A4B9309F10109BEE7319B03FB0BCB24
:109070000BFB02F200EBE2023FA821F06BF9439BED
:109080000BB13F9A9B5C08213398814207DB3B9AE6
:1090900022EA0B0250433A9AC3401340CDE73FA85F
:1090A000009102931DF0BFF8029B439A00991B02A6
:1090B0000AB13F98125C13430831E5E7054656E5CF
:1090C000000000000000000000530500FFFFEF7FDC
:1090D0000653050043B203000000F03F70B594B0A2
:1090E00004460E46014603A8154612F0DDF8C0B14D
:1090F0003346BDF92420BDF92210009503A812F0D3
:109100000FF803A8ADF82260ADF8245012F0A8F8CB
:10911000B4F80B3003F50073A4F80B30204614B0FC
:1091200070BD0446FAE7F0B595B004460D46014619
:1091300003A816461F4612F0B7F898B11A9B009381
:1091400032463B46294603A811F0EAFF03A812F075
:1091500087F8B4F80B3003F50073A4F80B30204601
:1091600015B0F0BD0446FAE72DE9F04F99B0064678
:109170008946014607A812F097F8B0B3BDF8304011
:1091800004F460480FFA88FABAF1000FC4F30C0433
:109190002EDA00223049304624F02EFB00222F49DF
:1091A0000546304624F028FB24F060FE074648467A
:1091B00025F0F0F800220146814602A81DF08DFB43
:1091C0000026A3000093B346DDE902218A4212D3B0
:1091D000059822F0ABFF284622F0A8FF484622F06F
:1091E000A5FFB3455846B8BF304619B0BDE8F08F6B
:1091F00000273D46DBE7069939B1895C0A2904D18D
:109200005E45B8BF5E464FF0000BB8F1000F07D1C6
:109210002046F8F76BF8834402A81DF004F8D3E762
:10922000B8F5005F02D1009B9B44F5E7BAF1000F4F
:10923000F2DA2846019122F04CF948B10199B9427D
:10924000EADBC91B284623F0BAFA00FB04BBE3E7BC
:10925000284624F077F8F8E79D520500A252050051
:10926000F8B506460F46154622F033F9044698B184
:10927000284622F04DF888B1284624F063F80446C9
:10928000384625F087F8054623F0B7FB241A09D5A0
:109290000024284622F04AFF2046F8BD304623F03D
:1092A000ACFBECE7284623F0A8FB0719304623F077
:1092B000A4FB8742ECDC2246012329463046F7F71F
:1092C000B9F9B0FA80F46409E3E7F8B507460E4649
:1092D000154622F0FEF8044648B1304625F05AF80B
:1092E000002D064605DA0024304622F01FFF2046F6
:1092F000F8BD23F082FB4419384623F07EFB8442FC
:10930000F1DC01232A4631463846F7F793F9B0FAE3
:1093100080F46409E8E7F0B595B004460D460146CF
:1093200003A816461F4611F0BFFFA8B1079B019383
:109330001A9B009332463B46294603A811F04DFF85
:1093400003A811F08DFFB4F80B3003F50073A4F8F7
:109350000B30204615B0F0BD0446FAE7F0B595B0E5
:1093600004460D46014603A816461F4611F09CFF11
:10937000A8B1069B01931A9B009332463B462946AF
:1093800003A811F02AFF03A811F06AFFB4F80B300C
:1093900003F50073A4F80B30204615B0F0BD044669
:1093A000FAE700002DE9F04FE1B00D4602901C46AF
:1093B00001469DF8A831159324A8924611F074FF38
:1093C000002800F0A582BDF8A43024A803F4604270
:1093D000C3F30C090592FDF799F8BDF914300C9010
:1093E000002B119380F29380059BB3F5204F00F082
:1093F0008C80B3F5404F14BF012304230022B049F1
:109400000298039324F0F8F900220E90AD490298D7
:1094100024F0F2F900220690AB49029824F0ECF90E
:1094200024F024FD04909DF8AA20BDF89530ADF8F5
:10943000583002F03002102A9BB270D183F0300312
:10944000BDF89720ADF895300AF10103A246D41A71
:109450009DF8AA3003F00303012B0DD8294602988A
:10946000FFF782FE9DF8AA3003F0030303FB000020
:1094700000EBD070AAEB600A9DF8AA30C3F3810319
:10948000012B9FBF0C9A03FB022303EBD373A4EBC6
:109490006304BDF8AB300A93BDF8AD300993BDF855
:1094A000AF300893BDF8B1300793BDF89530DB06B7
:1094B00042BFDDE90923CDE90932DDE9073228465B
:1094C00048BFCDE9072324F065FF00221290014632
:1094D0001FA81DF002FA039A01239340013B189341
:1094E0004FEA89031793C2F1080356461D93DDE93D
:1094F0001F239A4245D21FA81DF0E8F80A28054606
:109500002BD10C9B56461C44F1E7022376E701233E
:109510000022CDE90332002306930E9383E7202A2D
:109520000ED183F06003BDF89720ADF895300AF1B5
:109530000103A2EB030ABDF8993001341C1B87E735
:10954000302A85D183F05003BDF89920ADF89530CD
:10955000631C5446A2EB030A7AE7059B002B40F0FC
:1095600092800146BDF8A400F7F7C0FE0A9B0B905D
:109570001B1AB34222DB0B9B1E441CF053FA00283B
:10958000B5D0229822F0D2FD129822F0CFFD069994
:109590000E9823F026FEBDF85830ADF8953024A87B
:1095A00011F05EFE029B029AB3F80B3003F50073D4
:1095B000A2F80B30029861B0BDE8F08F089B9E4284
:1095C000D9DABDF8A480099BA3EB0803A342D2DA41
:1095D000079B9C42CFDA202DCDD93C49059AA5F1B5
:1095E00021033B4DDBB20846D7B29F422AD3C75C6A
:1095F000002DC0D03301083B0D932301083B0F938E
:109600002F444FF00D0BBD42B5D015F8012BC82AE1
:1096100022D8304B30499B5C14932E4B00205FFACC
:1096200080FE964513D3149B0DF1D40C01EB030E71
:109630008E450CF1040C11D135AA149924A811F00F
:10964000D3FBE0E711F8017B01323D44CCE713F88E
:1096500001EB01307144E2E70021E4E711F8012B4E
:10966000B2FBFBF00BFB10220D9BD2B212FB08F2F7
:109670001A4402380F9B2CF8042C10FB08F01844F5
:109680002CF8020CD4E7059BB3F5005F26D10A9BAA
:10969000033BB34212DC089B9E420FDA099B053B59
:1096A000A3420BDC079B9C4208DA159B2246CDE9BE
:1096B00000933146034624A811F0D2FE179B5BE7C6
:1096C000AF5105009D520500A25205009B3D0500CB
:1096D0007A3E0500D53F05009E400500119B002BFA
:1096E000BFF64BAF069821F0F4FE00285ED0049B35
:1096F000AB4200F30A810DF1D408002206994046DE
:109700001DF0EBF8049B0027ED1ADDE935239A42A2
:1097100003D2379B1344AB4241DB399B002B43D030
:1097200013F80280389822F001FD0A9BA3EB08038E
:10973000B34245DA089B9E4242DA099B0C9A9B1A77
:10974000A3423DDA079B9C423ADA92FBF9F3039A73
:10975000139353435F43FA100E9935A81DF0BDF8DB
:10976000399D07F007070DB1359BED5C039B7B43EB
:109770009D4006EB09030D9300230F930F9B434578
:1097800080F2BF800D9BA3EB09031B930D9B013B54
:109790001C9304EB09030B930023109377E04046DE
:1097A0001CF094FF0744B0E79846BBE7069823F007
:1097B000C9FD049BEF1AAB42804600FB07F7B4DDFE
:1097C00008FB0966D9E61D9BE8B21841159B0BB949
:1097D000002851D00B9B9DF89BC0A3EB09031A9363
:1097E0000B9B013B19930002189BB0FBF3F0B0F503
:1097F000807F0146A8BF4FF48071BCF1080FDDE9FE
:10980000273223D9BCF1100F4CD1C3F34510C1F559
:10981000807EC2F3451C4843C3F3C42B0EFB0C0CE3
:1098200001FB0BFBC2F3C4200EFB00B0000A03F0E7
:109830001F034B434FEA1C2CC00202F01F0240EAF8
:109840004C1C0EFB02324CEA12230CE04FF48A7ED1
:109850002EFA0CFC1CF0010F46D0C1F580704B4372
:1098600002FB00331B0A0193199B0093DDE91A21C7
:109870001C9B24A811F0B1FC039B1F44072F37DC6D
:109880009D40109B013310930B9B4B440B93109BFB
:10989000139A934297DB0F9B01330F930D9B4B441D
:1098A0000D936BE7BCF1180F1ED1C3F30720C1F570
:1098B000807EC2F3072C48435FFA83FBC3F3074360
:1098C0000EFB0C0C01FB0BFBD0B24B43C2F3074267
:1098D0002CF0FF0C0EFB00B00EFB02334CEA102004
:1098E0001B0A40EA0343BEE77F28D8BF1346BAE706
:1098F00035A81CF098FC399D0DB1359BED5C002717
:10990000BFE7389822F012FC5AE74FF0000857E7FB
:1099100002904FE630B595B00546014603A811F018
:10992000C3FCA0B122F0D6FA044668B1094823F07E
:109930004FFB0146204623F072FE01220094064BA5
:109940001146284607F02EFC204615B030BD0446CF
:10995000FAE700BFBB5105005D99020038B5054626
:1099600008460C4623F049F8072824D90122124959
:10997000204622F051FEF0B11049204622F054FE5C
:10998000C8B90F49204622F04FFEA0B90D49204624
:1099900022F04AFE78B96FF000420721204622F0FB
:1099A00052FF04460146284623F020FE2046BDE82B
:1099B000384022F0BBBB38BDCA510500D25105006A
:1099C000E0510500ED5105002DE9F04792B0044645
:1099D0008A46014601A8914698461A9F11F064FCF8
:1099E000002859D0504621F074FD40B92B49012080
:1099F0001DF08AFB0024204612B0BDE8F087B9F1C3
:109A0000FF0F01D92649F2E7404621F062FD28B94F
:109A1000404621F033FE08B92249E8E7C7F307269C
:109A2000002E4FEA274308BF0126012B05DD022B3C
:109A30002CD0042B2DD01C49D9E74FF400455246B9
:109A40001A49204623F094FE42461949204623F045
:109A50008FFEF8B222F056FA16490246204623F04D
:109A60009EFE484622F04EFA13490246204623F055
:109A700096FE354401A8ADF8185011F0F1FBB4F88A
:109A80000B3003F50073A4F80B30B4E74FF4204516
:109A9000D5E74FF44045D2E70446ACE71B5205003A
:109AA00038520500555205007F520500AF510500A0
:109AB0009D520500C5510500A2520500000000009E
:109AC0002DE9F04F97B090460191014605A81F4639
:109AD00011F0EAFB002856D0019821F0FAFC00288A
:109AE00079D00023092202A901988DF81030CDE920
:109AF000023324F0CFFD9DF80C609DF809009DF81D
:109B00000A909DF80B70002E40D11CF0B1F929F09D
:109B10001FFA0022904B29F0AFFB044648460D4641
:109B20001CF0A6F929F014FA00228B4B29F0A4FBB3
:109B3000824638468B461CF09BF929F009FA864B81
:109B4000002229F099FB002206460F4600232046FA
:109B5000294629F0D9FC88B90022002350465946ED
:109B600029F0D2FC50B9002200233046394629F0B2
:109B7000CBFC18B99DF80F30002B3BD00120774962
:109B80001DF0C2FA002017B0BDE8F08F49461CF066
:109B900084F929F0DDF96EA3D3E9002329F06CFBE9
:109BA00004460D46384631461CF077F929F0D0F9C5
:109BB00067A3D3E9002329F05FFB82468B469DF81B
:109BC0000D009DF80E101CF068F929F0C1F960A392
:109BD000D3E90023B5E7019824F0D0FD404655ECC9
:109BE000104B24F0CBFD38465BEC10AB24F0C6FDE7
:109BF00057EC106B25F000494FF0FF32584B2046D0
:109C0000494629F0A9FC002840F09E804FF0FF3221
:109C1000534B2046494629F095FC002840F094809B
:109C20002BF000494FF0FF324D4B5046494629F08A
:109C300093FC002840F088804FF0FF32484B50469C
:109C4000494629F07FFC00287ED127F000494FF0DB
:109C5000FF32434B3046494629F07EFC002873D141
:109C60004FF0FF323E4B3046494629F06BFC00284E
:109C70006AD100223B4B2046294629F0D3F929F02E
:109C800081FC0022374B04465946504629F0CAF958
:109C900029F078FC0022334B05463946304629F03E
:109CA000C1F929F06FFCBDF8191011F4607184F34B
:109CB000080385F3080280F3080008D0B1F5C07FDF
:109CC00019D010D880291AD0B1F5807F1CD09DF80A
:109CD0001F1010291FD19110DA10D20242EA41124E
:109CE00042EAE0004FE7B1F5007F11D0B1F5207FE7
:109CF000EDD1114601E019461346024606E0194629
:109D0000034610460A46E2E7194603460846DEE7E0
:109D100019461346F6E7202906D11B0443EA02231D
:109D2000034343F07F402EE7182904D11B0443EA84
:109D30000223184327E713440344B3F5C07F4FF0D1
:109D4000FF30B8BF00201EE7019823F0FBFA1AE7A6
:109D50000000000000E06F4000002E40BF520500F0
:109D6000FFFFEF7F0000704070B5044608460D46C7
:109D700021F08DFA002875D000223E49284623F0B4
:109D80003BFD064650B100231A4601462046FFF728
:109D900097FE394B1860304622F0C8F90022374947
:109DA000284623F029FD064650B100231A460146F5
:109DB0002046FFF785FE304B5860304622F0B6F95A
:109DC00000222F49284623F017FD064650B10023F4
:109DD0001A4601462046FFF773FE274B986030462F
:109DE00022F0A4F900222749284623F005FD064663
:109DF00050B100231A4601462046FFF761FE1E4B74
:109E0000D860304622F092F900221F49284623F0FC
:109E1000F3FC064650B100231A4601462046FFF7E0
:109E20004FFE154B1861304622F080F90022174989
:109E3000284623F0E1FC064650B100231A460146AD
:109E40002046FFF73DFE0C4B5861304622F06EF97C
:109E500000220F49284623F0CFFC18B124F042FA23
:109E6000054B1876B4F80B3003F50073A4F80B30EB
:109E7000204670BDA7520500DCA60020FB4F050060
:109E8000AA520500AE520500B2520500B6520500B6
:109E9000BA520500F0B593B004460E46014601A83B
:109EA00015461F4611F000FAF0B1AFB9049B2A46DF
:109EB000314601A811F0C5F901A8ADF81A60ADF856
:109EC0001C5011F0CDF9B4F80B3003F50073A4F871
:109ED0000B30204613B0F0BD00231A463946204609
:109EE000FFF7EEFD0346E2E70446F2E72DE9F04F07
:109EF0009DB00BAD80460F460146284616461C46CF
:109F000011F0D2F90290002800F09B80269B0A9362
:109F100008AA07A92846CDE90776099411F0E2F8C6
:109F20000AAA09A9284611F0DDF80798099B0899A3
:109F30000A9CC21802EBD27252101B1A009203EB59
:109F4000D3730A19641A5B1004EBD474641005937C
:109F50005B43039302EBD27204FB04F352100493AD
:109F60000192DDE903326600013E03FB162600275D
:109F7000009B03EB070B019B03EB040A52460E9B6D
:109F80005946284611F01CF8009BA3EB07095246DE
:109F90000E9B4946284611F013F8019BA3EB040AD7
:109FA00052460E9B5946284611F00AF828460E9B49
:109FB0005246494611F004F8049A7B0003FB022242
:109FC00071009142BFBF049A0298033302FB0366FB
:109FD0004FEA440C039BCCF1010203FB02F2B4BF35
:109FE00001370020914208DD039AACF10303013CE4
:109FF00002FB1366002CBBDA01E00028FAD1059BB6
:10A00000BB4207F101040CDC284611F029F9B8F82D
:10A010000B3003F50073A8F80B3040461DB0BDE8C7
:10A02000F08FDDE900120E9B2144284610F0C8FF96
:10A03000DDE900120E9B091B284610F0C1FF2746E0
:10A04000DDE7DDF80880E8E713B51C46134400930C
:10A05000121B0B19091BFFF749FF02B010BD2DE9B8
:10A06000F04F9FB00DF1340A80460E46014650462F
:10A0700015461C4611F018F90390002800F089805D
:10A08000289B0C930AAA09A95046CDE909650B94AF
:10A0900011F028F80CAA0BA9504611F023F80999E1
:10A0A0000B9B0C9CCDF818A0CA1802EBD272521070
:10A0B00002920A9A1519A41A5B1A04EBD47464105C
:10A0C00003EBD3735B10660005EBD575059304FBBA
:10A0D00004F95B43013E6D10049303FB16960027C1
:10A0E0007B0003FB099271009142BCBF033309FB63
:10A0F00003660498B8BF039A4FEA44030793C3F179
:10A10000010300FB03F3B4BF0137002299421FDDB6
:10A11000029B069803EB070AA3EB070B109B2A1977
:10A12000CDE9002351465B4610F00EFE109B0698C9
:10A130002A1BCDE9002351465B4610F005FE079B24
:10A14000049A033B013C02FB1366002CC8DA01E0D1
:10A15000002AFAD1059BBB4207F101040CDC0DA8D3
:10A1600011F07EF8B8F80B3003F50073A8F80B3047
:10A1700040461FB0BDE8F08F109B0299CDE9005317
:10A18000029B2A461B1B21440DA810F0DDFD27462B
:10A19000E0E7DDF80C80EBE713B51C4613440093B1
:10A1A000121B0B19091BFFF75AFF02B010BDF0B5C7
:10A1B00099B004460F46014607A816461D4611F001
:10A1C00073F8002840D01E9B069304AA03A907A891
:10A1D000CDE90376059510F085FF06AA05A907A825
:10A1E00010F080FF049A0A9B0399CDE9002307A889
:10A1F000059B10F0A9FD0A9B0193069B0093DDE9E6
:10A20000042307A8194610F09FFD069A0A9B03999C
:10A21000CDE9002307A8059B10F096FD0A9B01934A
:10A22000049B0093039B069A194607A810F08CFD27
:10A2300007A811F015F8B4F80B3003F50073A4F873
:10A240000B30204619B0F0BD0446FAE72DE9F0477F
:10A250008AB0804621F03DF9044638B948490320C8
:10A260001CF052FF20460AB0BDE8F08700224146AC
:10A2700068461CF032FB00273D463E463C464FF008
:10A280000009DDE900329A4225D8039821F04EFFFB
:10A2900021F023FE04460028E4D0304621F032FEAF
:10A2A00038490246204623F07AFA284621F02AFE51
:10A2B00035490246204623F072FA05FB06F00730C6
:10A2C0000021C01022F02CFE0546C0B9204621F026
:10A2D0002DFF2C46C6E768461CF0F8F90A2805D180
:10A2E00059EA040308BF01270134C8E7AC4209F169
:10A2F0000109A8BF651C4E45B8BF4E46C1E73A46A6
:10A30000414668461CF0E9FA4FF0000847464FF016
:10A310008009DDE900239A4208D3039821F006FF63
:10A320002A461A49204623F03AFA9BE768461CF071
:10A33000CDF90A2803D108F101080027E9E7202810
:10A340001CD0284621F0C5F8C0B106FB087A294682
:10A350004FEADA0205A81CF0C0FA099909B1059B79
:10A36000C95C0AF0070A49FA0AFA41EA0A0105A893
:10A37000C9B21CF00FF9089821F0D8FE0137C8E7E0
:10A3800092500500AE500500B45005001D57050061
:10A390002DE9F04390461D46421E47F6FE739A4251
:10A3A00093B006460F4602D84A1E9A4208D932494F
:10A3B00001201CF0A9FE0024204613B0BDE8F08364
:10A3C0004046FBF79FFE044620B92C4901201CF0B3
:10A3D0009BFEF1E7284620F05AFFD8B10022284919
:10A3E000284623F009FA002204462649284623F08D
:10A3F00003FA25468146284620F064FF044688B9C2
:10A400002A46214901201CF07FFE4946284622F0B9
:10A41000E8FED1E7B5F80B3003F50073A5F80B3073
:10A420008146E8E7B9F1000F06D0484620F04AFF20
:10A43000044608B94A46E4E7144900201AF0F6FD3C
:10A4400004460028B8D001238DF808303A46434628
:10A45000314601A810F0B4FF2A460D490194204668
:10A4600023F086F94A460B49019823F081F901A8A7
:10A4700010F0F6FEC9E700BF1F5005002C50050084
:10A4800038500500415005004A500500A550050010
:10A490007E500500885005002DE9F04391461D4689
:10A4A000421E47F6FE739A4293B00746884602D88A
:10A4B0004A1E9A4205D9674901201CF025FE002456
:10A4C00008E04846FBF71EFE044638B96249012001
:10A4D0001CF01AFE204613B0BDE8F0835F4900204F
:10A4E0001AF0A4FD04460028F4D0002601A84B462B
:10A4F000424639468DF8086010F062FF28468DF814
:10A5000009608DF80A60019420F0C1FE00285CD03B
:10A5100032465349284623F06FF923F0E3FE28B171
:10A52000BDF8093043F00103ADF8093000224D4970
:10A53000284623F061F923F0D5FE28B1BDF8093093
:10A5400043F00403ADF8093000224749284623F0C0
:10A5500053F923F0C7FE28B1BDF8093043F00803D2
:10A56000ADF8093000224149284623F045F923F08F
:10A57000B9FE88B19DF80F0001280BD1BDF8093054
:10A5800043F00203ADF80930BDF80D305B0703D08E
:10A59000374992E737498FE728460022364923F0AA
:10A5A0002BF9054688B1354922F03EF850B93449B7
:10A5B000284622F039F808BBBDF8093043F0800383
:10A5C000ADF80930284621F0B1FDBDF80D00BDF809
:10A5D0000B3043439DF80F0058430730C0080AF082
:10A5E00095FB284A05460146019823F04DF9294676
:10A5F00022F0F7FD01A810F033FE6BE72249284650
:10A6000022F012F820B9BDF8093043F48073D7E77F
:10A610001E49284622F008F820B9BDF8093043F455
:10A62000C073CDE71A49284621F0FEFF20B9BDF8D6
:10A63000093043F40073C3E71649284621F0F4FFBC
:10A6400020B9BDF8093043F42073B9E712481CF073
:10A650001BFCB7E71F5005002C500500A550050056
:10A660004C4F0500534F0500574F0500634F050041
:10A67000A14F0500714F0500DA4F0500E64F0500B8
:10A68000EA4F05001D570500EE4F0500F24F05008B
:10A69000F64F0500FA4F0500FE4F050000000000D0
:10A6A00008B500222DED028BB0EE408AF0EE608AF4
:10A6B000002351EC100B28F03BFF98B1B0EE480A94
:10A6C000F0EE680A26F0FCFC0B4B51EC100B00225C
:10A6D00028F0A8FCBDEC028B41EC100BBDE8084053
:10A6E00026F06ABCBDEC028B9FED010B08BD00BFDC
:10A6F000000000000000F87F0000E03F00000000C4
:10A70000F8B555EC104B25F000474FF0FF32284BC1
:10A710002046394628F020FF60B94FF0FF32244B25
:10A720002046394628F00EFF20B9B5F1004F08BF8A
:10A73000002C05D145EC104BBDE8F84021F0D0BB12
:10A74000002200232046294628F0DEFEC8B912A1C7
:10A75000D1E900012B46224628F0AEFA06460F4604
:10A7600028F0C0FF04460D4654EA05030DD100222F
:10A7700000233046394628F0C7FE30B19FED080B64
:10A78000DAE709A1D1E90001E4E720462946BDE85E
:10A79000F84021F0CCBB00BF2083E4FFFFFFDF3F88
:10A7A00000000000000000802083E4FFFFFFDFBF07
:10A7B000FFFFEF7F26F0FCBB26F07EB838B555ECE6
:10A7C000104B10EE102A2B4610EE100A294628F0E6
:10A7D00029FC02460B460020094928F06BFA41EC9F
:10A7E000100BFFF75DFF204653EC102B294628F095
:10A7F00043FDBDE8384041EC100B26F05DB800BFCA
:10A800000000F03F30B591B0054620F08FFE0446C1
:10A8100038B92A461F4903201CF076FC204611B0A7
:10A8200030BD0122294605A81CF099FE00231A46D6
:10A8300005A9194810F0C2FE044605A81BF0ECFB60
:10A840002046002122F06CFB044618B913481CF086
:10A850003BFBE3E72946012205A81CF080FE2146C8
:10A86000002268461CF039F86B460D4A0A4805A9D3
:10A8700010F0A4FE039821F059FC05A81BF0CCFBB6
:10A880000021204622F043F90546204621F04EFCE7
:10A890002C46C3E756530500938603007B530500FF
:10A8A000B586030030B591B0054620F03FFE044662
:10A8B00038B92A461F4903201CF026FC204611B057
:10A8C00030BD0122294605A81CF049FE00231A4686
:10A8D00005A9194810F066FF044605A81BF09CFB6B
:10A8E0002046002122F01CFB044618B913481CF036
:10A8F000EBFAE3E72946012205A81CF030FE2146C9
:10A90000002268461BF0E9FF6B460D4A0A4805A97C
:10A9100010F048FF039821F009FC05A81BF07CFB10
:10A920000021204622F0F3F80546204621F0FEFBE8
:10A930002C46C3E756530500938603007B5305005E
:10A94000B5860300F8B5051E0C4606DC2949012032
:10A950001CF0DAFB00242046F8BD084620F097FCE6
:10A960000646A8B100222449204622F045FF23F0E4
:10A97000B9FC002221490646204622F03DFF23F083
:10A9800075FA30F0080309D0102809D01C49DEE719
:10A9900024B122461B4901201CF0B6FB012400E033
:10A9A00002242946204621F0D0FB07469EB12946C5
:10A9B000204621F0CAFB0546134900201AF036FB59
:10A9C000044610B10FB146B13DB92A46394620467A
:10A9D00022F0FAFBBEE73546EEE73A460B49204641
:10A9E00022F0DDFE002DB6D02A460949204622F08D
:10A9F000D6FEB0E77354050092540500B15405002B
:10AA00009F540500B6540500ED5405001D57050080
:10AA1000F6540500F8B506460D460AB3104622F076
:10AA200091FC002D044603DA304621F0E6FF054490
:10AA3000002C03DA304621F0E0FF04441B2021F013
:10AA4000D1F925EAE57524EAE474074630B1A54258
:10AA500004DA631B2A46314621F0C8FE3846F8BDA9
:10AA600000296FF00044E9DADEE7F8B505460C4648
:10AA7000C2B1104622F066FC20EAE076002C05DA2E
:10AA8000284621F0BAFF044424EAE4741B2021F094
:10AA9000A9F9074620B133462246294621F0A6FEF1
:10AAA0003846F8BD6FF00046E8E7F8B507460C46B3
:10AAB000CAB1104622F046FC20EAE07524EAE474AC
:10AAC000A542B8BF23464FF01B00BCBF2C461D4615
:10AAD00021F088F9064620B12B1B2246394621F089
:10AAE00085FE3046F8BD6FF00040E5E770B50D1EFD
:10AAF000064606DA0B4901201CF006FB002420461E
:10AB000070BD1B2021F06EF9044615F1FF35F6D318
:10AB10001AF088FF0028F2D13146204621F08EFE3F
:10AB2000F3E700BF485405002DE9F04186B023F05B
:10AB300031FC0546E0B10146002201A81BF0CDFE24
:10AB40004FF0FF340026DDE90183984514D30498C3
:10AB500021F0ECFAA642DABFA21B013200223146F4
:10AB6000284621F070FE0446284621F0DFFA2546EB
:10AB7000284606B0BDE8F08101A8039F1BF0A6FDA2
:10AB80001BF0A8F90028DED107EB080336EA2406FB
:10AB900028BF1E461C46D6E72DE9F84F04460D4651
:10ABA00020F097FC20B94FF000084046BDE8F88F30
:10ABB00021F090F980460028F5D01DB9214622F0F9
:10ABC00015FDF2E75149284622F034FE00285FD0F7
:10ABD000002021F097F94E490246284622F0DFFD79
:10ABE0002146284603F0F4FB0027064626B13046EE
:10ABF00020F00EFB8146D0B1304621F097FA0020BC
:10AC000021F080F942490246284622F0C8FD20463C
:10AC100021F0F3FEB842C8DB39466FF0004220460F
:10AC200021F011FE0146404622F0F9FCBDE74946FD
:10AC3000304622F07FFB4A4636498246304622F0B3
:10AC4000DBFD23F013F98146504621F0D6FE834602
:10AC5000504621F06BFAA9EB07023946204621F055
:10AC6000F2FD0146404622F0DAFC0BEB09073046C4
:10AC700021F05CFA384621F045F92549024628467C
:10AC800022F08DFD2146284603F0A2FB0646ADE7E3
:10AC9000284623F07FFB814688B121F0AEFE0746AF
:10ACA000204621F0AAFE002600F1010BABEB070ABB
:10ACB0003546554522DC7FB925BB0135F9E7074606
:10ACC000EEE75D4612E00146404622F08FFC30463A
:10ACD00021F02CFAEE19F0E75545F2D001232A466F
:10ACE00049462046F5F7A6FC0028E6D1AA1B3146C6
:10ACF000204621F0A8FD06460028E4D1484621F070
:10AD000015FA52E75545F1D1F8E700BF5C5405004C
:10AD1000635405006D540500BFF34F8F0549064B82
:10AD2000CA6802F4E0621343CB60BFF34F8F00BFE9
:10AD3000FDE700BF00ED00E00400FA05024B034907
:10AD40005868002222F058BD602D00208A48050076
:10AD500070B5174B1C7884420DD0FCF7B5FE054644
:10AD60002046FCF7B1FE2A46034612490420BDE8FE
:10AD700070401CF0C9B9104C00201870206840B118
:10AD800089B1114603F022FC206821F0CFF900239D
:10AD900023600A4C206821F0C9F900232360084B86
:10ADA00001221A7070BD114603F058FDECE700BF98
:10ADB000D4A6002059480500CCA60020D8A6002023
:10ADC000F5A6002010B50A460C460021FFF7C0FF8B
:10ADD0002046BDE8104021F0A9B9000038B5194D52
:10ADE0002A884FF6FF719142044613D00146032092
:10ADF000FCF784FE18B1144B18681FF0C2FF04461C
:10AE000013212888F9F78AFD40F66B410DF082FD89
:10AE1000204638BD0D4B1D78022D0DD10C4822F077
:10AE2000D7F801462846FFF7CDFFFBF71CF920466F
:10AE3000BDE8384005F02ABF064901201CF064F93E
:10AE4000F5E700BFBE2C0020CCA60020D4A6002031
:10AE5000DD480500F248050010B5094B1C78012CAF
:10AE60000CD100210846FBF733FD064822F0B0F86C
:10AE700001462046BDE81040FFF7A4BF10BD00BF4B
:10AE8000D4A60020504B05000A460021FFF760BF02
:10AE9000F7B500223449044622F0AEFC22F0E6FF6A
:10AEA000324B334906460322586822F0A5FC05467A
:10AEB00030B12246B1B222F0E2FB284621F036F949
:10AEC00000222C49204622F097FC0746002839D161
:10AED00021460820FCF712FE18B90025284603B0C9
:10AEE000F0BD254B254E18681FF04BFF33884FF6F9
:10AEF000FF729A42054607D1214822F069F80146BF
:10AF00000820FFF75FFFE9E73A461749204622F09D
:10AF100073FC22F0ABFF013080B2ADF80400ADF855
:10AF2000060001A930880DF02DFE0DF08FFC0446BF
:10AF30000028D3D001460820FFF7A6FF204621F0C5
:10AF4000F5F8CBE721F0F2F800210920FCF7D6FD57
:10AF50000028C2D0084B18681FF013FF01210546D6
:10AF600020460CF03DF9B9E717490500602D002097
:10AF7000244905000B490500CCA60020BE2C00206A
:10AF8000F248050070B5014606460720FCF7B6FDFD
:10AF900068B3184B184D18681FF0F3FE2B884FF656
:10AFA000FF729A42044608D1144822F011F8014673
:10AFB0000720FFF707FF204670BD002210493046EA
:10AFC00022F01AFC22F052FF2B8881B20022184690
:10AFD0000DF0D6FD0DF03AFC05460028EBD00146F9
:10AFE0000720FFF751FF284621F0A0F8E3E70446C9
:10AFF000E1E700BFCCA60020BE2C0020F2480500EF
:10B00000174905002DE9F04F85B00D4600AF00232C
:10B010008046394628463B6021F03AFD0446002D23
:10B0200039D0F8B928461FF0A7FA064638601AF05A
:10B0300001FD06F58073834209D9374901201CF0D0
:10B0400063F8002630461437BD46BDE8F08FF31D87
:10B0500023F00703ADEB030D6C463246214628462C
:10B060001FF0AEFB00210620FCF748FD0028E8D0C9
:10B070002A4B2B4D18681FF084FE2B884FF6FF7269
:10B080009A4206460AD1274821F0A2FF014606202F
:10B09000FFF798FED6E70028E4D1D2E70022224944
:10B0A000D7F80090404622F0A7FB22F0DFFE0022F6
:10B0B0001FFA80FA1D49404622F09EFB834640B3AA
:10B0C00000221B4922F098FB23F00CF980465846D9
:10B0D00021F02CF8002398453B8114BF0223012363
:10B0E0003B71391D012328887B71FC60A7F806A0FD
:10B0F000A7F80A900DF042FD0DF0A8FB04460028C9
:10B10000A0D001460620FFF7BFFE204621F00EF832
:10B1100098E78046DEE700BF98530500CCA60020E4
:10B12000BE2C0020F2480500174905002B490500F8
:10B130003649050038B50D4601460A20FCF7DEFC0D
:10B1400060B3174B18681FF01CFE164B1A884FF699
:10B15000FF719142044608D1134821F039FF01469E
:10B160000A20FFF72FFE204638BD18880F4B1B78AA
:10B1700080B28BB100232A461946F9F797F90DF0F2
:10B1800065FB05460028EED001460A20FFF77CFE4D
:10B19000284620F0CBFFE6E70820F0E70446E2E788
:10B1A000CCA60020BE2C0020F2480500C8A3002039
:10B1B000F0B58BB06D460C4629460FF02FF80028ED
:10B1C00000F084800022012395E80300ADF81820E8
:10B1D0008DF81830A023ADF81A303F4BADF80C10A5
:10B1E000CDE907323D4B0290090C58688DF80E10DE
:10B1F0003B49099222F000FB22F038FEC3074CBF06
:10B20000384B394B089320464FF0C873099320F010
:10B210003EF8002841D000223449204622F0ECFAC2
:10B2200023F09AFD02460B4606460F4628F094F995
:10B2300090B900222E4B3046394627F0F3FE24A366
:10B24000D3E9002328F018F800222A4B27F034FD18
:10B2500028F0C0F9ADF8200000222749204622F04E
:10B26000CBFA23F079FD02460B4604460D4628F042
:10B2700073F990B900221E4B2046294627F0D2FED2
:10B2800013A3D3E9002327F0F7FF0022194B27F07F
:10B2900013FD28F09FF9ADF8220002AB93E80300FC
:10B2A000ADF81410090C04908DF8161008AA06A920
:10B2B00004A80DF06DFC0DF0C9FA044630B101464A
:10B2C0000220FFF7E1FD204620F030FF0BB0F0BD7B
:10B2D000000000000088934090000400602D0020D2
:10B2E000B64C0500900120031000A0009E4C050004
:10B2F00000408F400000E03FAA4C05000A460121B3
:10B30000FFF726BD70B50D4B1C78012C054613D1F7
:10B3100000210846FBF7DCFA2146094822F09CF997
:10B32000064608F015F8304620F000FF2946204672
:10B33000BDE87040FFF7E2BF70BD00BFD4A600209B
:10B34000D8A600207CDF70472DE9F04F964C85B0E1
:10B35000236800AF054603F0040308460E463B6031
:10B360001FF095FF002800F0AB8000228F49304687
:10B3700022F042FAB0B122F079FD4FF47A735843CB
:10B3800040F2712390FBF3F080B2B0F5804F884B10
:10B3900028BF4FF4804020281A8838BF20208242DE
:10B3A00018BF188000228349304622F025FA38B1B0
:10B3B00022F098FF2368002862D023F40063236002
:10B3C00000227D49304622F017FA38B122F08AFF78
:10B3D0002368002857D023F4805323600022774944
:10B3E000304622F009FA8146002873D0002307F185
:10B3F0000C01FB6021F04CFB8046002852D14846EE
:10B400001FF0BAF88246F8601AF014FB0AF5807350
:10B4100083423BD96A4901201BF076FE484620F062
:10B4200085FE28461FF033FF814608B9002D54D110
:10B4300031462846FCF7AEF8002D40F0B2800025DA
:10B44000604C614960682A4622F0DBFD32465F4964
:10B45000606822F0D6FD284620F068FE3B680BB1FC
:10B460000DF02EF94FF45B7140460DF053FA3B6836
:10B4700063B30EF0E3FC40F26E310DF04BFA25E0C1
:10B4800043F400639BE743F48053A6E70AF1070304
:10B4900023F00703ADEB030DE8465246414648460C
:10B4A0001FF08EF911234146BA893B7207F108005B
:10B4B000FFF748FF40F22D3180460DF02BFAADE743
:10B4C00046B13246424903201BF01EFE1437BD46EA
:10B4D000BDE8F08F4FF00008A3E728461FF0CEFE2E
:10B4E000786000284BD0B5F80B3003F50073A5F851
:10B4F0000B30236823F07F7323F40033294607F1D0
:10B500000C0023601AF0FCFDCB46F86850B9B9F185
:10B51000000F95D0BBF1010F92DD236843F4003397
:10B5200023608DE721F0F8FE82461FF0B0FE10B9CF
:10B53000BAF1000F0FD131465046FCF72BF8814687
:10B54000F86810B1494621F08DFD484620F0EEFD27
:10B55000D7F8049009E050461FF090FE0028F7D17C
:10B5600050461FF06EFE0028F2D1504620F0DEFD5E
:10B5700007F10C000BF1010B1AF0B1FDC5E72846ED
:10B580001FF05FFE00283FF45AAFB5F80B3003F50B
:10B590000073A5F80B30236823F07F7323F4003386
:10B5A000BEE705464CE700BFD0A60020664C05006C
:10B5B000BC2C00206F4C05007B4C0500B5490500F4
:10B5C00098530500602D0020854C05008F4C050028
:10B5D000D14A050072DF7047F0B5284B284983B087
:10B5E000044600AF0246586822F00BFD20461FF0CB
:10B5F00045FE48B10023391D20467B6021F048FA02
:10B6000005466CB970BB1BE020461FF01AFE0028EF
:10B61000F0D1CCB122461B4903201BF075FD13E08D
:10B6200000BB20461EF0A8FF064678601AF002FA1A
:10B6300006F5807383420AD9134901201BF064FD8B
:10B64000124903201BF060FD0C37BD46F0BDF31D11
:10B6500023F00703ADEB030D6D4632462946204625
:10B660001FF0AEF800213B792A460846FFF7B2FFEB
:10B6700040F225410DF04EF9E6E700BF602D0020B5
:10B68000244D0500594D0500985305002D4D05002A
:10B6900070B5294C29492068002222F0ADF80546F2
:10B6A00018B1002101200CF0E5F8284620F03EFDFD
:10B6B00000222349206822F09FF8054610B101209E
:10B6C0000CF0AEF8284620F031FD00221D496068DC
:10B6D00022F092F8002205461B49606822F08CF89F
:10B6E000014606462846FFF72FFE2846314621F040
:10B6F00078FD00221549606822F07EF805460BF0BF
:10B70000E3FE284620F012FD60681149002222F075
:10B7100073F8044608B1FFF75FFF204620F006FDEE
:10B720000DF00CF90B4B1B689B0503D5BDE8704071
:10B73000FCF764B870BD00BF602D0020194D0500F6
:10B7400000490500854C05008F4C05001C4E050086
:10B75000244D0500D0A6002070B592B004460D46D9
:10B76000014601A816460FF09FFD60B33EB140F2BE
:10B77000FF339D42A8BF1D46012DB8BF0125BDF96D
:10B780001830002B11DA2B040FD41049204622F078
:10B7900027FC0F49204622F023FC0E49204622F0C8
:10B7A0001FFC0D49204622F01BFC01A8ADF81850E3
:10B7B0000FF056FDB4F80B3003F50073A4F80B300E
:10B7C000204612B070BD0446FAE700BFAF51050035
:10B7D0009D520500C5510500A25205002DE9F84310
:10B7E000074608460D4614461FF073FE002800F079
:10B7F000848001224249284620F00EFF0646C8B345
:10B80000284621F0FAF8062894BF4FF0FF384FF091
:10B8100006083A21284620F0AFFF00282DDB00F172
:10B82000010841466FF00042284621F00CF822F052
:10B830001DFBB8F1010FB8BF4FF00108044608F135
:10B84000FF322846002120F0FEFF054641F6FF7337
:10B850009C42A8BF1C46012CB8BF0124BEB1A4B2B3
:10B86000284620F063FC324621463846BDE8F843BE
:10B87000FFF772BF4FF0FF38CBE7B8F1FF3FD0D1F1
:10B88000B5F80B3003F50073A5F80B30DEE715B9FA
:10B8900004F50054E3E7284621F0AFF80028F7D07C
:10B8A0001849284620F0C0FE0028F1D12946164844
:10B8B00020F0DAFF32460146804638461BF02AFD6A
:10B8C0008146B8B133463246394618F06FF820F059
:10B8D0002DFCA4F50044A4B24146484621F081FC69
:10B8E0004FF6FF739C42BBD12A46084901201BF04A
:10B8F0000BFCB5E74FF6FF74EEE7BDE8F88300BF39
:10B90000B4510500BB510500015205000B52050062
:10B9100070B592B00546014601A80FF0C5FC68B3AA
:10B920009DF80830012B83BF154B1A6804924FF025
:10B93000FF338EBF5B68049300230593BDF80B3083
:10B94000013BADF82330BDF80D30013BADF825309B
:10B95000079B03F44003002442F2010643F47023E2
:10B9600001A806960793ADF820408DF822400FF00D
:10B9700077FC224631462846FFF7EEFE12B070BD36
:10B98000DCA6002010B5044694B019B1FFF7C0FF43
:10B9900020F0CCFB214603A80FF086FCC8B1079A23
:10B9A0000192BDF81520BDF81330013A0092002233
:10B9B000013B114603A80FF0C7F903A80FF050FC94
:10B9C000B4F80B3003F50073A4F80B30204614B024
:10B9D00010BD0446FAE710B592B00C46014601A826
:10B9E0000FF062FC60B1BDF8093003F010031CB128
:10B9F00023B1BDF80B0003E0002BFAD0BDF80D0019
:10BA000012B010BD2DE9F04F99B006460D46014623
:10BA100007A80FF049FC044620B90024204619B0BD
:10BA2000BDE8F08F8DB15C49284620F0FDFD8046D1
:10BA300058B95A49284620F0F7FD044630B92A463D
:10BA4000574901201BF060FBE8E7A0460021304683
:10BA5000FFF7C1FF012183463046FFF7BCFF9DF889
:10BA6000277000FB0BF47C4307340646E410B8F162
:10BA7000000F35D020F031FA05460028CDD05846C9
:10BA800020F040FA47490246284621F088FE304619
:10BA900020F038FA44490246284621F080FE012F62
:10BAA00007D0384620F02EFA40490246284621F0B9
:10BAB00076FE9DF82030ABB9082F05D0BDF82130B7
:10BAC00003F00F03042B0DD100223949079821F010
:10BAD00093FE02463649284621F061FE2C469DE73A
:10BAE000033445462046002121F01AFA044618B9CD
:10BAF000284620F01BFB91E70146002202A81AF01D
:10BB0000ECFEB8F1000F0CD15FFA8BF102A81AF02D
:10BB10000CFDF1B202A81AF008FD394602A81AF08D
:10BB200004FD0026B1463346B24627E01A46514688
:10BB300007A800930FF069FB0AF1010A09FA07F957
:10BB4000D34549EA000907EB0602009B02DC0133FA
:10BB50004FF0000A16460AE0083E29FA06F1C9B27B
:10BB600002A8CDE900321AF0E0FCDDE90032072E30
:10BB7000F2D8D6086FF0070101FB0626DDE90212B4
:10BB80009142D3D3059820F0D1FAB8F1000F3FF4D9
:10BB900045AF22469EE700BF64660500EA5B0500EC
:10BBA000F54E0500AE500500B4500500BB50050031
:10BBB0001D5705002DE9F74F21F00045894616462F
:10BBC0001F464FF0FF32414B29468046044627F07E
:10BBD000C3FC002876D14FF0FF323C4B404629464B
:10BBE00027F0B0FC00286DD132463B46304639463E
:10BBF00027F0B2FC002865D10022002340464946C8
:10BC000027F082FC28B309F10045002200233046CA
:10BC1000394627F079FC10B107F100431F46002296
:10BC200000233046394627F065FC78B94FF0FF32E3
:10BC3000264B3046394627F071FC38B14FF0FF32C1
:10BC4000224B2046294627F069FCE8B9002400254C
:10BC500022E04D46D9E700221D4B2046294627F019
:10BC6000E1F9CDE90001B246BB4652465B46DDE94B
:10BC7000000127F05DFC52465B46E0B920462946AC
:10BC800027F018F804460D4622462B463046394622
:10BC900027F044FC0028DED100220023404649461C
:10BCA00027F032FC10B105F100431D46204629461D
:10BCB00003B0BDE8F08F1046194626F0FDFF82461E
:10BCC0008B46D2E70024034DF0E700BFFFFFEF7F74
:10BCD0000000E03F0000F87F2DE9F84355EC114BE0
:10BCE00011EE100A294657EC106B27F04BFC09287F
:10BCF000804619D827F02CF922462B4627F0FAFB6C
:10BD000090B1B8F1000F63D030463946B8F1010F59
:10BD100003D141EC100BBDE8F88332463B4627F0D7
:10BD200081F908F1FF38F1E7002200233046394657
:10BD300027F0EAFB0022D8B3284B20462946FFF71C
:10BD400039FF0022002327F0D5FBF0B300224FF08B
:10BD5000804320462946FFF72DFF0022002327F0CD
:10BD6000C9FBB04607F1004949EC108B68B125F0DA
:10BD7000A7F922462B4651EC100B27F053F9BDE8EA
:10BD8000F84341EC100B25F017B925F099F922463C
:10BD90002B4651EC100B27F045F941EC100B25F028
:10BDA0000BF953EC102B10EE100A03F10041B0E731
:10BDB00000233046394627F09DFB30B10022002396
:10BDC0002046294627F0AAFB28B147EC106BCEE7A6
:10BDD000002002499DE7002000219AE70000F03F83
:10BDE00038B5114C114B1546002291420CBF21462B
:10BDF000194621F001FD0446A0B15DB100232B706E
:10BE00001FF01FFA30B1A38803F00F03022B04BF09
:10BE100001232B70204620F027FC0546204620F009
:10BE200085F92C46204638BD1D570500F6540500FF
:10BE30002DE9F04F8DB0CDE900230D4600228A494F
:10BE4000DDF858A09DF85CB0044621F0D5FC22F046
:10BE500049FA30B1854901201BF056F90DB0BDE813
:10BE6000F08F284616F044FB08B98149F3E7DDE975
:10BE7000006323F000474FF0FF327E4B30463946D7
:10BE800027F06AFB80B94FF0FF327A4B30463946D3
:10BE900027F058FB40B972A3D3E90023DDE9000184
:10BEA00027F032FB074608B17349D4E70DF062F979
:10BEB000039050461FF0EBF9064600287BD03A4627
:10BEC0006E49504621F098FC22F046FF21F00049CF
:10BED0000F464FF0FF32674B4946064627F03CFBC2
:10BEE000F8B94FF0FF32634B3046494627F02AFB42
:10BEF000B8B9002200233046394627F023FB80B131
:10BF000000225F4B3046394627F08CF800225D4B0B
:10BF100027F088F800225A4B27F0AEF927F0E2FB11
:10BF2000039000225849504621F066FC22F0DAF9CD
:10BF3000064600270DF11302394620468DF813708E
:10BF4000FFF74EFF3A46804601212046FFF748FFA3
:10BF50009DF813308146002B36D0BB4514BF052712
:10BF60000627DDE900230020454927F085F9002256
:10BF7000444B27F057F80022414B27F07DF927F07A
:10BF8000B1FB26B1B9F1000F14BF4E464646039BE4
:10BF90000690032F184405908DF82C7001D0052FC2
:10BFA00018D13A4B33F81530ADF82A30FBB9384880
:10BFB0001AF06AFF2EE0BAF1000FBAD052463549A6
:10BFC00001201BF0A1F8B4E7BBF1000F14BF032759
:10BFD0000427C6E707F00507042FE8D12E4B05EB31
:10BFE000450213449B78002BE1D08DF82A5040463F
:10BFF0001EF0E8FFADF8200030460EB11EF0E2FF63
:10C00000ADF8220005A815F07FFE05A815F0C6FCC6
:10C010000028CCD04946404621F0E3F801201FF02B
:10C0200069FF11490246204621F0B9FB9DED000B46
:10C030001FF056FF19490246204621F0B0FB184B6D
:10C0400018495868032221F0D7FB054600283FF421
:10C0500005AF214621F0CAFA284620F067F8FDE630
:10C06000FCA9F1D24D62503FA455050020550500B2
:10C070003C550500FFFFEF7F485505001A5F05009E
:10C0800000408F40000030416855050000A70020A7
:10C090006F550500B6540500CC3C05008A550500D7
:10C0A000602D00208F5505002DE9F3410546084617
:10C0B0000C46904657EC106B0DF092FB00220023CB
:10C0C00051EC100B27F020FA38B9CDE90080324648
:10C0D0003B4621462846FFF7ABFE02B0BDE8F081A3
:10C0E00007B50123CDE9002353EC102BFFF7A0FE89
:10C0F00003B05DF804FB00002DE9F04F484B4949BF
:10C1000058688DB0002221F077FB064660B10146E9
:10C1100003A819F0F5FFDFF82491DFF824A10398B4
:10C1200030B9304620F002F800200DB0BDE8F08FA5
:10C1300021F0F2F800224946044621F05DFB22F08E
:10C14000D1F8054658B3002211462046FFF748FEB5
:10C1500083461EF037FF05AAADF81000074604A974
:10C16000314815F04BFB054618BB02462F492046C7
:10C1700021F042FB04AA2E4904900123204616F028
:10C1800025F804981FF0D2FF28461FF0B3FE494659
:10C190000246204621F003FB58461FF0C7FF204609
:10C1A0001FF0C4FF002D37D1314603A819F082FFDC
:10C1B000B5E7BDF82230002BEED0BDF82080434516
:10C1C000EAD0B8EB070318BF0123092251462046E5
:10C1D000019321F011FB21F049FE019B8342DBD04A
:10C1E00018461FF08FFE51460246204621F0D7FA2E
:10C1F0000E4B10490022B84518BF1946204621F0C1
:10C20000FBFA0123049004AA20460B4915F0DEFF37
:10C2100004981FF08BFFBFE703A819F060FF7EE7CB
:10C22000602D00208F550500D3F703001D57050032
:10C23000FE540500F654050016550500A4550500EA
:10C240000855050013B500221349044621F0D4FA1D
:10C2500022F048F828B9114901201AF055FF02B020
:10C2600010BD002211462046FFF7BAFD04461EF01D
:10C27000A9FE0DF10601ADF80600094815F002FB14
:10C2800018B9084901201AF03FFF20461FF04EFF61
:10C29000FFF732FFE3E700BFA45505009455050002
:10C2A000D3F70300AC5505002DE9F84304460D46CD
:10C2B000174698461FF00DF948B9B4F80B3003F54E
:10C2C0000073A4F80B3026463046BDE8F8832046BC
:10C2D00020F093FBA842F0DA204620F08EFB2D1AC6
:10C2E000B8F1000F1AD01B201FF07CFD0646002875
:10C2F000EAD0D7B1384622F04DF8074620F07DFB52
:10C300008146002D15DCB8F1000F03D021463046E0
:10C3100020F094FA38461FF009FFD5E76FF000428D
:10C320004146204620F08FFAE0E7084820F050FE12
:10C33000E3E7A9454B464FF00002A8BF2B4639461C
:10C34000304620F053FAA5EB0905DAE7A57F050092
:10C3500070B505468AB01B200E461FF043FD04460B
:10C36000D0B1284622F016F800220146054605A85D
:10C370001AF0B3FA0022214668461AF0AEFADDE957
:10C3800005239A420BD308981FF0D0FE03981FF0A4
:10C39000CDFE28461FF0CAFE20460AB070BD05A893
:10C3A0001AF094F901465EB1A0F16103DBB2192BDA
:10C3B00002D8A0F12001C9B2684619F0ADFEDEE74F
:10C3C000A0F14103DBB2192BF6D82031F3E710B40A
:10C3D00013460A4653F8044B0021A4465DF8044B6B
:10C3E00060472DE9F84388469146054618B1077A1B
:10C3F0000024A74201D8BDE8F8832B68686833F8A9
:10C400003430184420F0E4FD014606464846C04753
:10C4100030461FF08BFE0134EBE721F011BE000027
:10C42000002201491AF0FCBF795B050008B508B18C
:10C43000036823B91B20BDE808401FF0D3BC0021CE
:10C4400020F078FFBDE8084022F0A3B8024B034972
:10C450005868052221F0D0B9602D00209C590500B4
:10C4600070B5002286B00E46114921F0C5F9054687
:10C470001FF02FF8044660B10022294601A81AF0E7
:10C480002CFA0024DDE901239A4208D304981FF016
:10C490004DFE28461FF04AFE204606B070BD01A89A
:10C4A0001AF014F9B04208BF44F00104E4B2E9E71D
:10C4B000BE5F050010B5044618B9002000F0010069
:10C4C00010BD1EF0A5FE0028F7D120461EF020FF6B
:10C4D00080F00100C0B2F1E708B520F070F908BDA6
:10C4E00070B5054686B01B200E461FF07BFC044647
:10C4F000E0B128461EF0EDFFC0B1002E16DB32463B
:10C50000294601A81AF0E9F9DDE901239A420AD285
:10C51000059B03B19B5C8DF8033001220DF10301F3
:10C52000204620F0E3F904981FF000FE204606B0F4
:10C5300070BD37B505461B201FF054FC044628B1DA
:10C54000294601A819F0DCFD019810B9204603B076
:10C5500030BD20F0E1FE21F089FC01228DF80300BE
:10C560000DF10301204620F0C1F901A819F0B7FD33
:10C57000EAE70000F8B507460E461EF088FE88B3CD
:10C5800000221949384621F037F905461EF0A1FF6F
:10C5900018B3284620F031FA002E01DD86420AD376
:10C5A0001149384621F01CFD2C46002528461FF075
:10C5B000BDFD2046F8BD32460021284620F043F953
:10C5C000314604466FF00042284620F03CF9064907
:10C5D0000246384621F0E3F8E8E71B201FF002FC92
:10C5E0000446E3E70446E4E79F3C050038B504460B
:10C5F0001EF04DFE88B100220949204621F0FCF8CA
:10C6000005461EF066FF10B1284620F0F6F90446F4
:10C6100028461FF08BFD204638BD0446FBE700BFCF
:10C620009F3C050070B504461EF031FE30B9002471
:10C63000254620461FF07AFD284670BD0022144989
:10C64000204621F0D9F805461EF021FE044618B90F
:10C6500028461FF06BFDEBE7002DE8D000220D49C6
:10C66000284621F0C9F804461EF02CFE50B1284699
:10C670001FF05CFD002CDBD0074D2368EB1A5D42F8
:10C680005D41D6E72946204620F0ABFDCFE700BF4D
:10C69000795B050058670500F10B03002DE9F041B7
:10C6A000CB1D23F0070300AFADEB030D134614467B
:10C6B0006E460D4653F8048B0A463146C047A369BF
:10C6C0002B44A36163692B44636135441C34AE423F
:10C6D00002D1BD46BDE8F081204616F8011B19F0D5
:10C6E00060FF204619F0C5FDF1E7000010B50446D3
:10C6F00030B90246064903201AF006FD204610BD57
:10C70000B0F80B3003F50073A0F80B30F6E700BF6C
:10C71000FC5C05002DE9F04F93B000AF0E461546C6
:10C72000814615F0AFFD4FF0010A044607F11701ED
:10C73000304687F817A0F4F701FF002D804606DC8D
:10C740004FF0000840464C37BD46BDE8F08F19F069
:10C7500071F905F58073834204D9604950461AF097
:10C76000D3FCEDE7EB1D23F00703ADEB030D122C1B
:10C770006E463BD15A4B1B78CBB1002307F1200208
:10C780004FF040215748C7F82230C7F826307B8544
:10C7900087F820A087F8218087F822507E62F8F77A
:10C7A000C7FB024618B1504904201AF0ADFC2946D7
:10C7B00001201FF0CAFC80460028C1D0014600229B
:10C7C00007F120001AF09CFE354416F8011B07F112
:10C7D000200019F0E6FE07F1200019F04AFDB542ED
:10C7E000F3D107F1200019F011FCABE7002CA7D121
:10C7F0003E492246484620F0FFFF8246014607F1A7
:10C80000180014F0BDFF00285CD022463849484685
:10C8100020F0F2FF21F066FD3B7FB877FF2B51D06F
:10C820007A7FFF2A4ED087F8212087F82030BA6916
:10C83000304B93FBF2F37B62FB7FF97D87F822009C
:10C84000002B07F120002C4BF96008BF0023BB62CE
:10C8500014F05CFF4FEA480101F4FF7141F001015F
:10C8600007F1200014F00AFF60B305F1FF38A8EBD0
:10C8700004035942594108224FF0000B07F12000F0
:10C88000C7E9011214F09AFEBA6879684FEA4B0BB7
:10C89000013A40EA0B0BF1D107F1200014F0BEFE83
:10C8A00097F8210014F07AFE06F804B00134A5428E
:10C8B000DDD1FB681BB107F1200014F0F1FE97F801
:10C8C0002230BB77B87F1FF015FB09490246484666
:10C8D00020F04EFF514620F084FC68E72C580500FC
:10C8E000C4A600209CA000206158050074580500D3
:10C8F0007D58050090D00300A08601002DE9F04F7F
:10C9000089B000AF0D469046064615F0BBFC4FF0CF
:10C91000010AF91D0446284687F807A0F4F70EFE21
:10C920000023834607F108014046BB6020F0B0F8C1
:10C930000546B8F1000F43D0F0B940461DF01CFE8B
:10C940008146B86019F076F809F58073834207D9FB
:10C95000494950461AF0D8FB2437BD46BDE8F08F50
:10C9600009F1070323F00703ADEB030D6D464A46BB
:10C97000294640461DF024FFBB68002BECD0122C4A
:10C9800021D13E4A1278002AE6D0F9793C48BD61AF
:10C99000002291427A61FA61BB754FF0402114BFC9
:10C9A0001346202307F1140287F815B0F8F7C0FAF0
:10C9B00002460028D0D0334904201AF0A5FBCBE76B
:10C9C0000028C9D0D8E7002CC6D12F4922463046CE
:10C9D00020F012FF8046014607F10C0014F0D0FE53
:10C9E00060B322462949304620F006FF21F07AFC48
:10C9F0003B7CB874FF2B21D07A7CFF2A1ED07A753D
:10CA00003B75FA68224B93FBF2F3BB61FB7CB87574
:10CA1000002B07F114001F4BD7F808A097F80790D8
:10CA200008BF0023FB6114F071FE4FEA4B0101F4D3
:10CA3000FF7107F1140014F021FE88B9B87C1FF0D3
:10CA400059FA12490246304620F092FE414620F043
:10CA5000C8FB81E7295D07F1140014F00FFE0134D3
:10CA6000A245F7DCB9F1000F03D007F1140014F070
:10CA700017FEBB7DBB74E1E798530500C4A60020F8
:10CA80009CA00020D1580500745805007D58050071
:10CA900090D00300A08601002DE9F74F0D46032139
:10CAA0000446CDE900230CF03BFE4FF0000B4FF0A5
:10CAB000010A4FF08008D94615F1FF3502D203B0C4
:10CAC000BDE8F08F009B0AEA0306019B0BEA03070F
:10CAD00056EA070316D088F31188002120460CF08F
:10CAE0002FFB0A20F4F784FE012120460CF028FBDE
:10CAF00089F311883720F4F77BFE1AEB0A0A4BEB17
:10CB00000B0BD9E788F31188002120460CF018FBA5
:10CB10004120F4F76DFE012120460CF011FB89F352
:10CB200011880520E7E710B40C7802460023204660
:10CB300008215DF8044BFFF7AFBF00002DE9F04F6F
:10CB400089B08946009015F09DFB4946044602A82D
:10CB500014F016FE28B3122C40F0FF809DF80C4014
:10CB6000204615F0C5FC9DF80D5018B1284615F06B
:10CB7000BFFCC8B92246294689481AF0A5F9B9F17F
:10CB8000000F00F0078101228649009820F096FDF1
:10CB9000034618B1494620F065FA034618461FF0CF
:10CBA000C5FA09B0BDE8F08F7F49029E7F4B04EBC8
:10CBB000440405EB45050C440D449E4294F8018065
:10CBC0006F7858DD7A4B9E42D4BF4FF080664FF0AD
:10CBD000CD66784A784C13785BB323681BB1774BEA
:10CBE0001021C3F880104FF040234FF0FF31C3F8FD
:10CBF0000813D3F800120021C3F80012C3F800157F
:10CC0000012184F8221094F8271079B9D3F8081577
:10CC10004FF0A04001F5E07140F2023540F821509C
:10CC2000D3F80C3503F5E07340F82350002384F863
:10CC3000223094F8223001251570FBB1082260499A
:10CC400004201AF061FA9DF80C40204615F050FCC3
:10CC500020B14FF4207120460CF0E2FB9DF80D400E
:10CC6000204615F045FC002889D04FF49451204609
:10CC70000CF0D6FB83E74FF0CC76AAE79DF81E2098
:10CC800084F827209DF81D20A360C4E9003384F8B0
:10CC9000253084F8243072B34FEA8800B90000F1DF
:10CCA000A04001F1A04140F20C624FF0A04BC0F84F
:10CCB000002705FA08FAC1F80027BD4040F20D62CE
:10CCC0000193CBF808A5CBF80855C0F80027C1F8A8
:10CCD00000270420F4F748FD019BDBF810150D42F6
:10CCE0002BD043B14FF0A04A0420CAF80C55F4F7FA
:10CCF0003BFDCAF808554FF0A04308F5E07140F23B
:10CD00000C6243F8212007F5E07143F821204FF031
:10CD100040231D46C3F80885C3F80C75C3F8246585
:10CD200022681AB106210420F8F7DEFA0523C5F8B7
:10CD30000035022384F8223085E701930420CBF8E4
:10CD40000CA5F4F711FDCBF808A50420F4F70CFDB1
:10CD5000019B0133092BC0D1C4E7002C7FF40FAF36
:10CD60009DF80C00FF2807D001210CF0E9F9032100
:10CD70009DF80C000CF0D4FC9DF80D00FF283FF44A
:10CD8000FEAE01210CF0DCF903219DF80D000CF042
:10CD9000C7FCF4E60349009821F022F901E700BF3F
:10CDA0008558050074580500CC3C050097AB02007F
:10CDB00087F50400C4A600209CA0002000E100E04C
:10CDC000B45805000149002018F030B92858050072
:10CDD0000149002018F02AB92F61050001490020FF
:10CDE00018F024B94660050070B506460D461EF0E1
:10CDF00070FB044630B93246134903201AF084F917
:10CE0000204670BD1149002018F010F93246104933
:10CE1000044620F0ADFC45B128461EF05AFB68B927
:10CE20003246094903201AF06FF900201FF06AF812
:10CE300008490246204620F0B2FCE1E72A460649AE
:10CE4000204620F095FCF0E78C5F05005C5405005F
:10CE5000B75F050063540500BE5F050038B50022CA
:10CE60000849054620F0C8FC044640B9064918F0B8
:10CE7000DDF8044904460246284620F079FC2046A5
:10CE800038BD00BF238205007F5F0500F0B58DB07F
:10CE90000D4616461C4615F0F5F911289DF8487008
:10CEA00005D02F4901201AF02FF90DB0F0BD16B9A9
:10CEB0000CB90F2403262B4B1B78F6B2E4B25BB9F6
:10CEC0002949ADF810306FF0FF02CDE9011201A839
:10CED000264A03920CF0C2FAFF2F03D000213846F5
:10CEE00015F064FF28461EF013FA80B1284620F0A2
:10CEF00029FA22463146C0B2F4F7C2F9F4F770F8C5
:10CF0000FF2FD2D00121384615F050FFCDE728463B
:10CF10001EF00CFBE8B1802383F31188012229461F
:10CF200001A81AF01CFB01A819F0A2F8054601A8F7
:10CF300025B919F071F885F31188DFE719F07DFA4A
:10CF400022463146C0B2F4F79BF901A819F0ABF9BB
:10CF5000E9E72A46064901201AF0D6F8CEE700BFD5
:10CF600033610500A8A60020A0860100000108008A
:10CF70005B610500F0B58DB00D4616461C4615F0F8
:10CF800081F911289DF8487005D0304901201AF028
:10CF9000BBF80DB0F0BD16B90CB9032401262C4B1B
:10CFA0001B7806F00F0604F00F045BB92949ADF8B1
:10CFB00010306FF0FF02CDE9011201A8264A03925A
:10CFC0000CF04CFAFF2F03D00021384615F0EEFE8E
:10CFD00028461EF09DF980B1284620F0B3F922467C
:10CFE0003146C0B2F4F70CF9F3F7FAFFFF2FD0D0B7
:10CFF0000121384615F0DAFECBE728461EF096FAF6
:10D00000E8B1802383F311880122294601A81AF090
:10D01000A6FA01A819F02CF8054601A825B918F0C0
:10D02000FBFF85F31188DFE719F007FA2246314646
:10D03000C0B2F4F7E5F801A819F035F9E9E72A4696
:10D04000064901201AF060F8CEE700BF0B61050029
:10D05000A8A60020A0860100000108005B61050071
:10D0600010B50C4615F0CCF92146BDE8104015F07E
:10D070009DBE08B515F0C4F90021BDE8084015F0C3
:10D0800095BE08B515F0BCF90121BDE8084015F0C2
:10D090008DBE0000F0B58BB004460D4615F0F2F8D9
:10D0A00001AE074632466946204615F0F9F898B3B6
:10D0B000009B059396E80F0006AC07C423807DB360
:10D0C000296800292CDD0139284620F033F906466D
:10D0D0001EF0F8FA10B3304615F092F904462846CF
:10D0E00020F048FF1FF022F830461FF01FF8FF2CF9
:10D0F00003D00021204615F059FE05AA094928460B
:10D100001DF040F9112F01D1F3F76AFFFF2C03D076
:10D110000121204615F04AFE0BB0F0BDFF24E3E7E5
:10D12000FF24EAE7CFC302002DE9F041B8B00D4675
:10D13000164607A908AA15F0B3F8002877D0FF2EE5
:10D1400003D00021304615F031FE28461EF0E0F8ED
:10D1500080462846B8F1000F18D020F0F3F818A93F
:10D160008DF8600008AB08460122079CA0479DF897
:10D1700060001EF0C7FE0446FF2E03D0012130469A
:10D1800015F014FE204638B0BDE8F0811EF0A1F97C
:10D190000746002831D01B201EF024FE42460446DC
:10D1A000294602A819F099FBDDE902239A4203D32C
:10D1B00005981EF0BBFFDFE718F034FC0028F7D11C
:10D1C00001AA694602A819F005F8019D002DEBD0CF
:10D1D000802D28BF802508AB2A4618A90098079FF4
:10D1E000B8472A4618A920461FF080FB019B5B1B0D
:10D1F0000193009B1D440095E7E728461DF0BCF90C
:10D20000014601201EF0A1FF04460028B4D03A4692
:10D2100001460EA8CDE90C771AF072F907AA054964
:10D2200028461DF0AFF80EA818F0F0FEA4E704465B
:10D23000A8E700BF9DC602007FB50C46054615F065
:10D2400021F821460646684613F090FF98B1112E4A
:10D2500013D168460CF002F93CB301221549284667
:10D2600020F02CFA034618B121461FF0FBFE0346BE
:10D2700018461EF05BFF04B070BD002EFBD19DF878
:10D280000500FF2802D001210CF04AFA9DF80600A3
:10D29000FF2802D004210CF043FA9DF80700FF2874
:10D2A000DAD001210CF03CFAD6E70249284620F0FA
:10D2B00097FEE0E7745805002DE9F04300228DB099
:10D2C0002449064620F098FA05AD0146284622F08A
:10D2D000CDFA1B22541E295D09B1144602E02246F4
:10D2E000002CF7D10CAB4FF001081C440DF12409C0
:10D2F00004F81C8C99E807008DE8070095E80F00FA
:10D3000022F005F908F1010807460028F0D10120B4
:10D310001EF0F8FD10490246304620F040FA38462B
:10D320001EF0F0FD0D490246304620F038FA38462E
:10D330001EF0E8FD0A490246304620F030FA384631
:10D340001EF0E0FD0749024630460DB0BDE8F0434F
:10D3500020F025BAB5490500AC610500B2610500B1
:10D36000B9610500796F05002DE9F04F00229BB0EF
:10D370000C469B49054620F03FFA20F077FDC0B2ED
:10D38000772808D0612806D09649012019F0BCFE04
:10D390001BB0BDE8F08F204620F0FCFF07460028B8
:10D3A000F6D01FF02AFB81460028F1D000228E49DA
:10D3B000284620F021FA20F059FD00228B498246B0
:10D3C000284620F019FA20F051FD002288498346B2
:10D3D000284620F011FA20F049FD002285498046B8
:10D3E000284620F009FA0BAC0146204622F03EFA0E
:10D3F0001B22531EE15C09B1134602E01A46002BC2
:10D40000F7D11AAA1A44CDE9082302F83C8C7A49CC
:10D410000022284620F0F0F920F028FD06460028DA
:10D4200045D0099BA0F120020DF1480E106851680B
:10D43000F446ACE803000832B242E646F6D15A1C84
:10D44000214613A826F0F4FAA8B112AB03930FAB50
:10D4500093E807008DE8070094E80F0021F065FFCE
:10D46000064608B9654990E71EF04CFD6249024640
:10D47000284620F094F9ABEB0A0BD94556444FDB14
:10D480005A46002138461FF0DEF93146824606F042
:10D49000B5FD50461EF04AFEB8F1FF0F4BD158497A
:10D4A000012019F031FE38461EF040FE70E74FF4BF
:10D4B0007E63CDE905034023CDE903730FAE96E803
:10D4C00007008DE8070094E80F0022F061F80028BB
:10D4D000E9D012AB039396E807008DE8070094E8C3
:10D4E0000F0021F022FF0646129820F07F444846A4
:10D4F0001EF008FD3C490246284620F050F920461F
:10D500001EF000FD39490246284620F048F9304611
:10D510001EF0F8FC38490246284620F040F9C2E7E0
:10D520003846314606F06AFD09EB0A001EF0EAFCB7
:10D530002D490246F0E7089B08F1010003F83C0C76
:10D540001EF0E0FC2A490246284620F028F96FF038
:10D550000042594638461FF076F900234FF47E62A8
:10D56000CDE905324023CDE903030FAE804696E8AE
:10D5700007008DE8070094E80F0022F009F8002862
:10D5800091D012AB039396E807008DE8070094E86A
:10D590000F0021F0CAFE0646129820F07F4448464C
:10D5A0001EF0B0FC10490246284620F0F8F820464C
:10D5B0001EF0A8FC0D490246284620F0F0F830463F
:10D5C0001EF0A0FC0C490246284620F0E8F8404630
:10D5D0001FF013FA044640461EF0A8FD2046A5E7BA
:10D5E000796F0500D6610500B2610500EF610500A5
:10D5F000AC610500B5490500B9610500F36105009E
:10D600000F6205002DE9F04F0022A1B00E466E49D1
:10D61000054620F0F1F820F029FCC0B2722808D0AD
:10D620006A49012019F070FD0027384621B0BDE895
:10D63000F08F00226649284620F0DEF820F016FC24
:10D640008046002800F0BD8000226249284620F074
:10D65000D3F820F00BFC00225F498146284620F0D9
:10D66000CBF820F003FC00225C498246284620F0DB
:10D67000C3F820F0FBFB002259498346284620F0DE
:10D68000BBF8014609A822F0F1F81B22531E09A994
:10D69000C95C09B1134602E01A46002BF6D120AA54
:10D6A000D318069303F85CBCF30F059318BF20262C
:10D6B00000273EBB7CE04FF0000846E012F8011B5B
:10D6C000FF291CD00598013300286CD00A296AD1A3
:10D6D00000221C46059237B91B2007931EF082FBDF
:10D6E000079B074630B1224610A9384607931FF022
:10D6F000FDF8079B059AA1441AB91E1BD9E71C46E1
:10D7000054E02026AAEB0904002C3DDCBBF1FF0FFE
:10D71000D1D0069B0BF1010B03F85CBC18AB039353
:10D720000DAB93E807008DE8070009AB0FCB21F0A4
:10D73000FCFD189B23F07F4A804650461EF0E2FB1A
:10D7400025490246284620F02AF840461EF0DAFB1A
:10D750001F490246284620F022F800201EF0D2FB86
:10D760001C490246284620F01AF858461EF0CAFB0B
:10D770001A490246284620F012F8B8F1000F3FF48B
:10D7800054AF54464FF00009202E3346A8BF202343
:10D790009C42A8BF1C46224609EB080110A826F0AF
:10D7A00055F910AA0023A34288DB3346002C92D1FE
:10D7B00048461EF0A7FB0749024628461FF0EFFF28
:10D7C00033E7074631E700BF796F0500BE6105000A
:10D7D000B9610500B2610500EF610500AC610500AB
:10D7E000B54905004FF0FF31FFF70CBF21EAE171A9
:10D7F000FFF708BF2DE9F04F0022A5B03B491FF00D
:10D80000FBFF05AC01460546204622F015F82846E8
:10D810001EF08CFC1B235E1EA25D0AB11E4602E0B8
:10D820003346002EF7D124AB1E444FF001080CAF55
:10D8300006F87C8C0DF1240B03979BE807008DE81C
:10D84000070094E80F0021F070FD0546002847D03E
:10D850000C9B23F07F4303444FF0000913F8013C75
:10D860000C9AFF2B22F07F4A02D0B8F1FF0F1ED195
:10D870000024AAEB0406002E14DD412E28BF40260A
:10D880003246611914A826F0E1F814AA002312F810
:10D89000011BFF2922D001339E42F8D100221C44F3
:10D8A000002AE6D004EB090025B0BDE8F08F08F1AE
:10D8B000010806F87C8C03979BE807008DE80700B9
:10D8C00094E80F0021F031FDD144054658B10C9B7E
:10D8D00023F07F43034413F8013CC1E70122DEE754
:10D8E00081460446DEE70446DCE700BFB549050093
:10D8F00010B58CB005AC0146204621F09DFF0CAB65
:10D9000013E907008DE8070094E80F0021F0FFFD00
:10D910000CB010BD2DE9F04F0C46A7B00646674984
:10D9200020461EF081FE98B9654920461EF07CFE17
:10D9300050BB644920461EF077FE054638BB2246A0
:10D940006149012019F0E0FB284627B0BDE8F08FBF
:10D950004FF0720A5D49002017F068FB0546002869
:10D96000F2D01C22002130461EF06DFF0DF11C0884
:10D9700001460646404621F05FFF1B214B1E18F86A
:10D9800003203AB10B4608E04FF0770AE2E74FF088
:10D99000610ADFE71946002BF0D126AAD3184C49BB
:10D9A00005933246284601240EAE03F87C4C0DF157
:10D9B0002C091FF0F4FE039699E807008DE8070094
:10D9C00098E80F0021F0B1FC0E9BBAF1770F0746E3
:10D9D00023F07F4B09D100286ED02846FFF76CFC5E
:10D9E0004FF0000B5F46002629E0BAF1610FFAD133
:10D9F000002F61D007EB0B0313F8013CFF2B01D084
:10DA0000FF2C45D10026ABEB0608B8F1000F16DD60
:10DA1000B8F1400FA8BF4FF040084246F11916A8D0
:10DA200026F014F816AA002312F8011BFF2941D092
:10DA300001334345F8D100221E44002AE3D020469A
:10DA40001EF060FA2349024628461FF0A8FE304621
:10DA50001EF058FA2049024628461FF0A0FE38461C
:10DA60001EF050FA1D49024628461FF098FE5846FF
:10DA70001EF048FA1A49024628461FF090FE50460A
:10DA80001EF040FA1749024628461FF088FE5BE761
:10DA9000059B013403F87C4C039699E807008DE858
:10DAA000070098E80F0021F040FC0E9B074623F08A
:10DAB0007F4B9DE70122BFE73E46C0E72DAF050043
:10DAC000116705006E7C050090610500A0610500EE
:10DAD000B5490500AC610500B2610500B9610500FA
:10DAE000EF610500796F0500F3F762B821F09ABB8A
:10DAF00030B58FB007AC01460025204621F09CFED2
:10DB0000CDE903550EAB13E907008DE8070094E853
:10DB10000F0021F051FC044638B129461EF0F7FFF2
:10DB2000054620461EF002FB2C4620460FB030BDB5
:10DB300070B58EB007AC16460D460146204621F062
:10DB40007BFECDE903560EAB13E907008DE8070015
:10DB500094E80F0021F030FC0EB070BD4FF4D820D7
:10DB600021F036BE13B50C4614F08CFB8DF807007F
:10DB70000938042805D80DF10702034920461CF096
:10DB800009FD02B010BD00BF8DDB02000B78C1B2F1
:10DB9000184614F0CBB900002DE9F04389B098463F
:10DBA00005460E46174614F06DFBA0F10903DBB2E3
:10DBB000042B04462ED80D280FD1274BDB7863B9F0
:10DBC0004FF0FF324FF41651CDE9041204A8234A56
:10DBD00006928DF81C30F7F7ADFB8DF80040204C15
:10DBE0001FB1304620F0D6FB06466A462146304635
:10DBF0001CF0D0FC17B130461EF098FAB8F1000FB7
:10DC000005D069460D20A04769460A20A04709B003
:10DC1000BDE8F0830028FAD10246124928461FF0D9
:10DC2000EBFD22468146104928461FF0E5FD04AD74
:10DC3000024649460446284613F0BCFB20461EF027
:10DC400075FA48461EF072FA95E80F006C4607C454
:10DC50002370064CC4E700BFC5A6002008000100E1
:10DC6000F12E04006F5605007458050011250400BC
:10DC700000231A46FFF790BF01231A46FFF78CBF17
:10DC800000230122FFF788BF2DE9FF47044614F067
:10DC9000F9FA00220546404920461FF0ADFD00225A
:10DCA00007463E4920461FF0A7FDA5F1090682461A
:10DCB000002F4CD001463A46684613F07BFB9DF896
:10DCC0000600FF2802D000210BF02AFD9DF8070076
:10DCD000FF2802D000210BF023FD9DF80400FF284F
:10DCE00002D000210BF01CFD9DF80500FF2802D09A
:10DCF00000210BF015FDF3B2042B28D9002228498E
:10DD000020461FF079FD10B320F0B0F85FFA80F8DC
:10DD1000002140460BF002F9002013F0DFFA8146A3
:10DD2000A8B141461EF0CAFA804618B101464846DD
:10DD300020F0A6F848461EF0C7FB20B9194B1A4937
:10DD4000586820F04DF9494640461FF04AFA5146BE
:10DD500038461FF046FA1149204620F041F9F6B244
:10DD60000D49204620F03CF9042E11D80D2D0AD182
:10DD70000E4BDB780BB10AF02BFFFF220021284667
:10DD800014F046FC04E0A5F10C03DBB2012BF4D93E
:10DD900004B0BDE8F08700BF745805006F56050059
:10DDA000FD600500602D002002610500C5A6002071
:10DDB000F0B585B005460F46144614F063FA0646E2
:10DDC00084B92246524928461FF016FD04462246D1
:10DDD0003946684613F0EEFA58B920461EF0A6F907
:10DDE00005B0F0BDB4F80B3003F50073A4F80B30A8
:10DDF000EDE700981EF086F84649024628461FF0D7
:10DE0000CEFC7CB12246424928461FF0C8FCA6F150
:10DE10000903DBB2042B0AD80D2EE1D16846F7F7CF
:10DE200089FADDE73A49284620F0DAF8EFE7002ED4
:10DE3000D6D19DF80500FF2807D001210BF070FC1A
:10DE400001219DF8050014F0B1FF9DF80400FF28A2
:10DE50000BD005210BF064FC60201DF01BFF044675
:10DE600060B92D49012019F04FF99DF80630FF2BBC
:10DE7000B6D02A49012019F047F9B1E702462849EE
:10DE800028461FF08CFC20461DF068FA002680F81A
:10DE9000406004460BF06EF9009B9DF80A2084F860
:10DEA0005860C4E914369DF8083013449DF80920E1
:10DEB000B24218BF0133C4E9120184F8593001217C
:10DEC0009DF804000BF02AF80446C8B11EF01AF8B9
:10DED0001449024628461FF062FC012013F0FEF9A7
:10DEE00006460028C1D02A4621461FF0C8FB30460E
:10DEF0001EF01CF9013C0C4B0C4A43F82420B4E7FB
:10DF00009DF804200A49012019F0FEF8ADE700BF92
:10DF1000745805006F56050078600500D56005004F
:10DF20009E600500FD60050040A70020F912040076
:10DF3000A660050010B50C4614F0A4F9A0F1090381
:10DF4000DBB2042B04D82146BDE8104015F0C2B95D
:10DF500002490120BDE8104019F0D6B84D60050017
:10DF60002DE9F74F9846012313600D6907468A464D
:10DF700016460DB10B68ED5C38782E2800F0FA805B
:10DF80005B2836D1012388F8093097F801B0BBF13E
:10DF90005E0F02D13368013333604FF0000907E0B0
:10DFA0002E2C19D12E2D08BF49F001090133336001
:10DFB0003368FC5CF818002C00F0DE805D2CEFD19B
:10DFC00001333360002388F80930BBF15E0F14BFC2
:10DFD000484689F0010019E0434601AA5146FFF77F
:10DFE000BFFF3368019A49EA00095FFA89F91344CF
:10DFF000DDE75C286CD1022333607878642808D18F
:10E00000A5F1300009288CBF0020012003B0BDE835
:10E01000F08F442806D1A5F13000092894BF0020D4
:10E020000120F3E766286ED062286ED06E286ED08D
:10E0300072286ED0732805D1284603B0BDE8F04F92
:10E0400017F048BF532806D1284617F043FF80F049
:10E050000100C0B2DAE774285DD076285DD0772859
:10E060000ED1A5F13003092B40F28480284617F029
:10E0700025FF00287ED15F2D14BF00200120C5E7B9
:10E0800057280CD1A5F13003092B12D9284617F0D7
:10E0900015FF70B9B5F15F0018BF0120B6E7302851
:10E0A0003DD0A0F13103082B05D83649012019F0E5
:10E0B0002BF80020AAE778280AD1BB7843B1FB7877
:10E0C00033B104233360F978B87817F0E6FEC0B2B4
:10E0D00098F809302BB33368FA5C2D2A21D13B44E0
:10E0E0005B785D2B1DD0A8F80A00306801303060E5
:10E0F000434601AA51463844FFF732FF3368019A7C
:10E100001344336082E70C20E2E70820E0E70A20AE
:10E11000DEE70D20DCE70920DAE70B20D8E7002056
:10E12000D6E798F8082062B1A5F14103192B98BFF2
:10E130002035A0F1410398BFEDB2192B9CBF2030D0
:10E14000C0B2B8F90A30B3F5807F11D0DBB22AB182
:10E15000A3F14102192A9CBF2033DBB24FF4807235
:10E160009D42A8F80A20A4D38542A2D8984255E738
:10E17000854281E7012049E70120034918F0C4FFE7
:10E18000204643E71D6205003A62050082B02DE992
:10E19000F047ACB00C4634A9054681E80C0017F0F6
:10E1A00041FC30B1002630462CB0BDE8F04702B04B
:10E1B00070472B780BB17C2B43D1582234A90DEB3F
:10E1C000020025F043FCDDE93457DDF8DC901DF05A
:10E1D00081FE2368A2681A440646D21B39462846A7
:10E1E0001EF031FB00210446024630461FF047FA7C
:10E1F00020461DF09BFF0DF1680800244C450DDB07
:10E2000038461DF07FFE7049024630461FF0C7FABF
:10E210002A466E4930461FF0ABFAC4E758F8041B93
:10E22000D8F820202846521A1EF00DFB01348246F1
:10E230000246214630461FF022FA50461DF076FF76
:10E24000DCE75E2B09D12368A268D342AAD119F07A
:10E250001DF90028A6D0013507E0242B1DD1D4E9F3
:10E2600000329A4205F101050CD8502236A96846C1
:10E2700025F0ECFB34AB0CCB21462846FFF786FF9C
:10E28000064690E74C2237A9684625F0DFFB34AB01
:10E290000ECB284600F066F9F2E7282B0FD1379B0A
:10E2A0002168A26834A80A44191D082B40F82120CF
:10E2B00000EB83014A63CADC01333793C7E7292B9C
:10E2C0000AD1379B002BC2DD34AA02EB83032168FD
:10E2D000A2680A441A63BAE734AB15AA2146284655
:10E2E000FFF73EFE159FEB5DA3F12A02012A80464F
:10E2F00005EB07064ED801372F4450B92B2B08D118
:10E300004C2237A9684625F0A1FB34AB0ECB38462A
:10E31000C0E7214616A818F00CFA502236A9684624
:10E3200025F094FB34AB0CCB16A93846FFF72EFF33
:10E33000064619981DF0FAFED4E900239A42BFF46C
:10E3400032AFB8F1000F3FF42EAF204617F06BFF4D
:10E3500034AB15AA21462846FFF702FE2146804627
:10E3600016A818F0E6F9502236A9684625F06EFB8B
:10E3700034AB0CCB16A93846FFF708FF8146199835
:10E380001DF0D4FEB9F1000FD6D030461DF0CEFE00
:10E390004E46D1E7D4E900239A420BD250B1204631
:10E3A00017F041FF19F072F800283FF4FBAE159BFF
:10E3B0001D445AE74C2237A9684625F047FB34AB89
:10E3C0000ECB304666E700BF6D5405005C62050069
:10E3D0002DE9F047B4B00646084614AF1FF0DAFF47
:10E3E00000225449804630461FF006FA1FF03EFDD9
:10E3F00000220546504930461FF0FEF904461DF044
:10E4000068F848B9214640461EF0EBFE002420463D
:10E410008037BD46BDE8F08740461EF0EEFAA842C0
:10E42000F0D320461EF0E9FA00F1080323F00703B9
:10E43000ADEB030D0DF1500A421C5146204620F071
:10E4400029F920461DF072FE69213046FEF708F8D2
:10E450004FF48072002387F830007A8641462A46BE
:10E46000384687F831307B63C7F8288018F035FAD2
:10E47000394607F1140018F05CF9502207F1300119
:10E480006846FD6225F0E2FA07F1280999E80C00D8
:10E4900007F114015046FFF779FE0446386A1DF073
:10E4A00045FE384617F0BFFE2CB9D7E900239A4243
:10E4B00005F1010514D3F8681DF038FE40461DF043
:10E4C00035FED4B902201DF08DFC002504462846F7
:10E4D0001DF018FD1749024630461FF060F996E717
:10E4E000394607F1140018F024F9502207F13001E1
:10E4F0006846FD6225F0AAFAC8E767213046FDF7B5
:10E50000AFFFA0B1002120461EF014FF002280467C
:10E510000A4920461FF070F91FF0A8FC0546404646
:10E520001EF06BFA054440461DF000FECFE705469D
:10E53000CDE700BF63540500B75F05006D540500CB
:10E5400038B5FFF745FF054650B11CF061FE80F07D
:10E550000100C4B228461DF0E9FD04F0010038BDF9
:10E560000446F7E784B0F0B59BB021AE054686E8D7
:10E570000E0018F08BFF68B9044620461BB0BDE8BA
:10E58000F04004B070475C2C03D16C78002CF4D0C0
:10E590003D4601352C78002CEFD07C2C05F101078D
:10E5A000F1D1DDE9211215A818F097F923A950221D
:10E5B000684625F04BFA96E80C0015A93846FFF797
:10E5C000E5FD044618981DF0B1FDD6E737B50546C0
:10E5D00001910B4848F208011DF072FC044660B13D
:10E5E0002A4608491FF0C4F82846012301AA2146FB
:10E5F00013F0B4FD20461DF099FD03B030BD00BFFF
:10E60000B3EA0200144D05002DE9F743054608461C
:10E610000F4690461CF056FE38B93A46254903206D
:10E6200018F072FD03B0BDE8F083B8F1000F0BD015
:10E630000022214928461FF041F80446E8B11EF0A7
:10E640006FFE04461D4E01E01D4E44460022314639
:10E6500028461FF0D1F8814688B93A463146284607
:10E660001FF086F8B8F1000FDCD028462146FFF7EE
:10E67000ADFF20461DF05AFDD4E78046E2E71CF0CE
:10E68000FDFD38B1394648461EF0B0FF48461DF042
:10E690004DFDE7E702216846CDE900971EF0DCFF5B
:10E6A00031460746024628461FF062F838461DF0FC
:10E6B0003DFDEBE7225605004656050018560500BD
:10E6C0001D56050010B500220446FFF79DFF2046A9
:10E6D000BDE81040FEF7C2BB38B51546012204461E
:10E6E000FFF792FF25B1002229462046FFF78CFF55
:10E6F0002046BDE83840FEF7B1BB00002DE9F74FDA
:10E7000005461CF013FF044640B92A46344903204D
:10E7100018F0FAFC204603B0BDE8F08F3149002024
:10E7200016F084FC04460028F4D048F208012E4874
:10E730001DF0C6FB8146D8B122462C491FF018F8BF
:10E740001DF0C8FB2946824601A817F0D9FC002617
:10E750003546019880B9A81B1DF0D4FB2449024618
:10E7600020461FF01CF85246224920461FF017F899
:10E7700048461DF0DBFCCDE71EF0CEFD8046FDF7E0
:10E7800051FF30B348F260011B481DF099FB07466A
:10E7900028461DF0B7FB00210246834638461FF08D
:10E7A000BDFA58461DF0C2FC2246104938461EF0FC
:10E7B000DFFF39464A464046FFF78EFF39461EF0D6
:10E7C00010FD40461DF0B2FC01A8013517F087FC92
:10E7D000BFE74246294650461EF051FF0136F0E79A
:10E7E000565305007F5F050099E80200144D0500AF
:10E7F000745F05007A5F0500FDE702002DE9F04136
:10E800000F4690461349002205461EF0F5FF1FF003
:10E810002DFB00220446104928461EF0EDFF064657
:10E82000B0B142463946013C1EF029FF20461DF09A
:10E8300069FB0849024628461EF0B1FF1CB9314663
:10E840002846FFF7C3FE3046BDE8F0411DF06EBC20
:10E85000BDE8F081745F05007A5F050037B50546B5
:10E8600001910B4848F208011DF02AFB044660B1F3
:10E870002A4608491EF07CFF2846012301AA2146AA
:10E8800013F06CFC20461DF051FC03B030BD00BFFE
:10E89000ADEA0200144D050038B500220D460949C5
:10E8A00004461EF0A9FF58B11DF040FC2046054962
:10E8B0001FF096FB29462046BDE83840FFF7CEBF43
:10E8C00038BD00BF7A5F05002DE9F04385B00646EC
:10E8D0000191414914461FF083FB404930461FF027
:10E8E0007FFB00223E4930461EF086FF3C4905462C
:10E8F00030461FF075FB20461CF0C0FC074660B395
:10E90000214603A817F0FCFB0024039878B916F001
:10E91000A9FF804658B301462846FFF79FFF2A46C5
:10E92000214640461EF050FC05B0BDE8F0831EF0C5
:10E93000F3FC01AB01223146814615F037F88046E1
:10E9400017B91DF0F3FBA04648461DF0EFFB03A8E6
:10E9500017F0C5FB00274446D7E7002CD7D0204648
:10E9600001AB0122314615F021F80446CFE74DB343
:10E970002046FDF757FE50B348F2080119481DF034
:10E980009FFA48F20801064617481DF099FA074613
:10E99000A6B198B12A46154930461EF0E9FE2A462E
:10E9A000124938461EF0E4FE012231462046FFF7A8
:10E9B0002BFE424639462046FFF726FE39463046B2
:10E9C0001EF00FFC294620461EF00BFCACE721464A
:10E9D0002846FFF7FBFDF5E7185605001D56050014
:10E9E00023820500CDE502005DE80200144D05001C
:10E9F000294B2DE9F047B2F10009284E08BF1E4609
:10EA00000D460022314680461EF0F6FE044670BBDD
:10EA100002462349DFF888A040461EF0EDFE04467A
:10EA20004CB9B9F1000F25D12A461E490120BDE895
:10EA3000F04718F069BB0022314620461EF0DCFE8C
:10EA40000746024648B129462046FFF73DFF2146CA
:10EA50003846BDE8F0471EF0C4BB514620461EF0C4
:10EA6000CBFE074620461DF061FB3C46D8E7B9F1D6
:10EA7000000F05D02A460C4940461EF079FE4CB1E5
:10EA8000404622462946FFF71FFF2046BDE8F047D3
:10EA90001DF04CBBBDE8F0871D560500185605005B
:10EAA000238205004F560500465605000022FFF759
:10EAB0009FBF0122FFF79CBF70B505460E461CF0B4
:10EAC000E6FB58B928461CF0A3FB044630B92A4699
:10EAD0000E49032018F018FB204670BD30461CF08C
:10EAE000D6FB18B10A49012018F00EFB1DF0F5F90C
:10EAF00004460028F0D028461CF0C9FB0028EBD0C3
:10EB00002A46044920461EF033FEE5E7005A050078
:10EB1000335A0500795B0500F7B513F071FC054623
:10EB200013F0E6FC18B90024204603B0F0BD1DF038
:10EB3000D4F904460028F6D005EB4505224B5E19B2
:10EB40005B5D40338DF8043001A800238DF805305B
:10EB50001EF03EFA1D49024620461EF020FE707847
:10EB60001DF0D0F91A49024620461EF018FEB5786D
:10EB700085B11DF0B2F9074660B11DF0ABF906464C
:10EB800090B905F01F001DF0BDF91249024620465C
:10EB90001EF005FE1DF0A1F902460028C4D00E4962
:10EBA00020461EF0FCFDBFE7AB0606D501201DF098
:10EBB000A9F9014630461EF032FD32460749384673
:10EBC0001EF0EDFDDDE700BFCC3C0500425D050019
:10EBD000475D0500505D0500585D05004B5D050073
:10EBE0002DE9F74F0AF0C6FA894607461CF014FED5
:10EBF00083460AF0BFFA80468A461DF06EF9044645
:10EC0000002800F0A680564B5649586800221EF096
:10EC1000F3FD0546002800F0A0801DF031FC0646FB
:10EC200028461DF083FA002501230D214E485A1E67
:10EC300001FB0202B2F80B0080060FD010460193D0
:10EC400000921CF081FB0135019B0D2130B1009A2F
:10EC500012680C32B2FBF1F213441544013340F652
:10EC6000CA029342E2D9B018AB1B401B00931DF0BF
:10EC700049F93E49024620461EF091FD009B184688
:10EC80001DF040F93A49024620461EF088FD40F644
:10EC9000CA001DF037F93749024620461EF07FFDB5
:10ECA00030461DF02FF92F49024620461EF077FD11
:10ECB00058461DF027F93049024620461EF06FFDE8
:10ECC000B8EB07006AEB090124F07EF900222B4B18
:10ECD00024F0A8F92A4B002224F0A4F941EC100BEF
:10ECE0001DF0FEF82749024620461EF058FD0D2073
:10ECF0001DF008F92449024620461EF050FD234825
:10ED00001DF000F92249024620461EF048FD002071
:10ED10001DF0F8F81F49024620461EF040FD1E482F
:10ED20001DF0F0F81D49024620461EF038FD4FF454
:10ED3000D8201DF0E7F81A49024620461EF02FFDA4
:10ED40004FF400201DF0DEF81649024620461EF062
:10ED500026FD204603B0BDE8F08F064663E700BFFE
:10ED6000602D0020FC5E05007C2D0020045F050066
:10ED7000095F05000F5F0500155F050000408F402B
:10ED80000000B03E185F05001F5F0500A8B300201B
:10ED9000295F0500395F0500BCB70500455F050028
:10EDA000565F0500675F050010B51DF096F8044634
:10EDB00029481EF00DF92949024620461EF0EFFCB5
:10EDC00027481EF005F92749024620461EF0E7FCB9
:10EDD00025481EF0FDF82549024620461EF0DFFCBE
:10EDE0004FF400201DF08EF82149024620461EF007
:10EDF000D6FC4FF420401DF085F81E4902462046FF
:10EE00001EF0CDFC4FF480301DF07CF81A4902460C
:10EE100020461EF0C4FC04F06DFB18490246204653
:10EE20001EF0BDFC04F052FB1549024620461EF0C0
:10EE3000B6FC14481EF0CCF81349024620461EF0DA
:10EE4000AEFC12481DF05EF81149024620461EF045
:10EE5000A6FC204610BD00BF7B5E0500835E05005A
:10EE60008B5E0500945E05009F5E0500A95E0500AF
:10EE7000AF5E0500B55E050044770500BD5E050088
:10EE8000C45E0500CC5E0500EE5E0500C42C0020CB
:10EE9000F65E050038B508490546002016F0C6F8AC
:10EEA000044638B128461DF035F80449024620468C
:10EEB0001EF075FC204638BD185D05004455050060
:10EEC00010B513F09DFA044613F012FB20B1204652
:10EED000BDE810401DF01EB810BD2DE9F8430D46E9
:10EEE000032107460AF01CFC002401264FF080088D
:10EEF000A14615F1FF3502D22046BDE8F88388F31C
:10EF00001188002138460AF01BF90320F2F770FC43
:10EF1000012138460AF014F90A20F2F769FC384654
:10EF20000AF0FAF800B1344389F311883520F2F77A
:10EF30005FFC7600DDE710B5032104460AF0F0FB24
:10EF4000002120460AF0FCF84FF4FA70F2F750FC6A
:10EF5000012120460AF0F4F85020F2F749FC20463F
:10EF60000AF0DAF804464FF4D270F2F741FC84F06C
:10EF70000100C0B210BD000008B5002203491EF018
:10EF80003BFCBDE8084013F091BA00BF44550500B2
:10EF90002DE9F04F8BB00C46FFF7EEFF064613F05D
:10EFA000A7FA28B94FF0000840460BB0BDE8F08F33
:10EFB0001CF090FF80460028F4D0631EFF2B28BF72
:10EFC000F0242246E317CDE900234FF00009304634
:10EFD000FFF7B1FF0028E7D0DDE900230821304624
:10EFE000FDF75AFD01240025AA4627460121304697
:10EFF000FFF773FF01215FFA80FB3046FFF76DFFDB
:10F00000BBF1010FC0B22BD101283AD1402FCBDD8B
:10F010009DF80C30002BC7D005AC0DF10C09002574
:10F02000A34619F8017B380916F00EFD207007F091
:10F030000F0016F009FD0135082D607004F102047F
:10F04000EFD1002358468DF824301DF0C1FF014652
:10F0500040461EF0E4FAD146BAF1000FA4D0B6E75C
:10F060000AAB2B44834513F81C3C2DD14F4524DAC1
:10F070001C4214BF4FF0010B4FF0000BBBF1000F0F
:10F0800021D00AAB2B444FF0010B13F81C3C234357
:10F090000AAA2A44012102F81C3C30465A460023A1
:10F0A0006400FDF7F9FC14F0FF0404BF01350124EE
:10F0B000072D07F1010799DDA8E70CBF4FF0010B01
:10F0C0004FF0000BDAE7BA4623EA0403E0E770B535
:10F0D0008AB00C46FFF750FF064613F009FA68B3F2
:10F0E00020461CF015F918B320461EF02BF90146F6
:10F0F000054601201DF029F8044650B101460022C2
:10F10000684618F0FDF915F1FF3505D2684616F08E
:10F110007DFF20460AB070BD08213046FFF7DDFEB6
:10F12000C1B2684617F03DFA684617F0A2F8EAE760
:10F1300008213046FFF7D1FE1CF0E4FE0446E8E764
:10F1400037B50D461446FFF717FF8DF8070013F08B
:10F15000CFF980B10DF107020C4928461BF01AFACD
:10F160009DF807004CB1012109F0EAFF01219DF84B
:10F1700007000AF0D5FA03B030BD04210AF0D0FA36
:10F1800001219DF8070009F0DBFFF4E727CB02001F
:10F1900010B5FFF7F1FE044613F0AAF938B1204686
:10F1A000CC2200230821BDE81040FDF775BC10BD3E
:10F1B0002DE9F04186B00C46FFF7DEFE054613F060
:10F1C00097F940B120461CF084F938B92246264907
:10F1D000032017F099FF06B0BDE8F08120461DF02E
:10F1E0000CFC1028F2D12846FFF7A5FE214600228C
:10F1F00001A817F072FB002427462646A04601A866
:10F2000017F064FA8DF8000001A817F05FFA0023E8
:10F210001A468DF80100102168468DF8028016F01C
:10F2200064FEA4F12002C4F12003A14000FA02F21E
:10F2300020FA03F31143A04008341943402C47EA55
:10F24000000746EA0106DAD104981CF06FFF284651
:10F25000552200230821FDF71FFC3A46334621467C
:10F260002846FDF719FCB6E7205D050010B5FFF74D
:10F2700083FE044613F03CF920B12046BDE810405F
:10F28000FFF759BE10BD73B51CF024FE054660B1F2
:10F29000FDF7DCF8064640B1014601A816F030FF44
:10F2A000019C2CB930461CF041FF284602B070BDCD
:10F2B000B4F80B30002203F500731146A4F80B30AC
:10F2C00020461EF0ACFC014628461EF0A8F9204658
:10F2D0001CF02CFF01A816F002FFE1E710B101219C
:10F2E0001EF0E3BA704700002DE9F74305460F46CC
:10F2F00091461BF0E7FF044640B92A4657490320D0
:10F3000017F002FF204603B0BDE8F08328461BF04B
:10F3100088FF60B3A98828681CF0D2FD0446002845
:10F32000F0D02946684616F0EBFE009D7DB3B5F897
:10F330000B3003F50073A5F80B3028461DF0ECFFE9
:10F34000804628461CF01BF9D8B1B8F1000F2AD02E
:10F35000012128461EF0A9FA064630B10146204692
:10F360001EF066F830461CF0E1FE01260AE0284651
:10F370001BF09EFF002814BF082007201CF032FD60
:10F38000CCE70646414628461DF02BFF6EB9B9F181
:10F39000000F0ED1009D002D45D13A463049204640
:10F3A0001EF0E6F9AEE74646ECE7684616F097FE33
:10F3B000BBE7494601A816F0A3FE01980028E9D052
:10F3C0001DF0AAFF009D064665B1B5F80B3003F5A8
:10F3D0000073A5F80B3028461CF0D1F840B9284638
:10F3E0001CF0A4FE3246002120461EF097FC13E0DC
:10F3F0000122002128461EF012FC314680461DF0F5
:10F4000031FE414620461EF013F8284641461DF0C5
:10F41000E8FE684616F063FE30461CF087FE01A841
:10F4200016F05DFEC9E7B5F80B30012203F5007355
:10F43000A5F80B30114628461EF0F1FB064630B108
:10F44000014620461DF0F4FF30461CF06FFE2846B2
:10F450001CF06CFE684616F042FE9BE7CE57050096
:10F46000144D05002DE9F04F8FB0814602AF1046D4
:10F470008A4616461CF05AF80446002856D03046F4
:10F480001DF0DDFAB0F5807F044680460AD90246B9
:10F490002B49012017F038FE002420463437BD46A2
:10F4A000BDE8F08F8300DA1D22F00702ADEB020DFC
:10F4B00002AD2A462B440021934219D10122314644
:10F4C000381D18F04CF8381D16F0D2FD98B9381DCB
:10F4D00016F0A2FD00231946CDE9008552464846A4
:10F4E0001AF0A4F82946044640461DF050FED4E721
:10F4F00042F8041BE0E7381D16F063FD06461CF0D9
:10F50000EBF860B130461DF01DFFB0F1000B06DBDB
:10F510005C4504DD381D17F09CF945F82B0030469A
:10F520001CF004FE381D16F0BEFECCE72EB13246AC
:10F530000449012017F0E8FDAFE7B0463546C9E7BA
:10F540004A570500935705002DE9F34704460D4639
:10F550001BF0B8FE30B94449032017F0D5FD02B0C6
:10F56000BDE8F08728461BF0ADFE0028F3D020460A
:10F570001BF057FE064628461BF053FE86420AD073
:10F5800028461BF04EFEB4F80B30002842D043F062
:10F590004003A4F80B3020461BF08AFE064628469E
:10F5A0001BF086FE86420BD028461BF081FEB4F885
:10F5B0000B3023F03F0380B343F00803A4F80B3073
:10F5C00000222A49DFF8A490DFF8A4A020461EF00C
:10F5D00075F800222649074620461EF06FF80646B9
:10F5E00020461EF018FD294601A816F089FD019D50
:10F5F000B5B91FB1394620461DF01AFF38461CF038
:10F6000095FD1EB1314620461DF012FF30461CF01C
:10F610008DFDA4E723F04003BBE743F00703CDE7EC
:10F62000B5F80B3003F5007301A8A5F80B3016F000
:10F6300056FD494628461CF0F7FF88B95146284632
:10F640001CF0F2FF60B9012128461EF02EF9804619
:10F6500030B1014620461DF0EBFE40461CF066FD31
:10F6600028461CF063FDC2E7055805002358050035
:10F670006A7E050010B5FCF7E9FE044630B11EF0C5
:10F68000CAFC2046BDE810401CF050BD10BD000073
:10F6900070B506461BF01DFF28B911490120BDE8D1
:10F6A000704017F031BDFCF7D1FE0546B8B100221D
:10F6B00031461EF027FA044648B93246094901206E
:10F6C00017F022FD2846BDE870401CF02FBD014612
:10F6D00028461EF0D5FB20461CF028FDF2E770BD41
:10F6E000A4590500D25905002DE9F74305460F46F8
:10F6F00014461CF011F830B93549032017F004FD09
:10F7000003B0BDE8F08338461BF0E3FE08B9314989
:10F71000F3E720461BF0D6FD28B920461BF0D9FEA2
:10F7200008B92D49E9E739462C481DF09DF8804677
:10F730000028E5D00146012228461EF0E3F90646DE
:10F7400040461CF0F3FC30461DF0E6FD804620BB31
:10F75000214630461DF086FC314640461DF041FDF5
:10F760001F4938461CF060FF0028C9D000221D49FF
:10F7700028461EF041F801901BF0ABFE48B11A4933
:10F780002846012301AA12F021FD164928461EF041
:10F7900027FC01981CF0CAFCB2E71BF06FFD20B1FA
:10F7A000214640461DF022FFD6E71CF093FB414660
:10F7B00081461DF01BFF214648461DF017FF4946B4
:10F7C00030461DF04FFC48461CF0B0FCC4E700BFBB
:10F7D000835B0500BA5B0500F15B0500495C050031
:10F7E000BA5305009F3C0500633C0500F8B506468A
:10F7F000084614461F461DF0EBFB394605462046D9
:10F800001CF05EFB2946044602463046FFF76CFFBB
:10F8100029462046BDE8F8401DF0E3BC73B5054617
:10F820000C461BF079FF20B92149032017F06CFC2E
:10F830001AE020461BF04DFEC0B121461D481DF0C8
:10F8400013F8064680B10146012228461EF05AF9F7
:10F85000044630461CF06AFC34B1284621461EF0AE
:10F860000FFB20461CF062FC02B070BDF4B92946C3
:10F8700001A816F045FC104E019C002CF4D0B4F801
:10F880000B3003F5007301A8A4F80B3016F027FC29
:10F890000122314620461CF0BFFE18B12146284601
:10F8A0001EF0EEFA20461CF041FCE5E70349BCE7F8
:10F8B000835B0500495C05004F5C0500535C050057
:10F8C00038B5054608461DF083FB044640B10146A5
:10F8D0002846FFF7A3FF2046BDE838401CF026BCB1
:10F8E00038BD0000F8B507460C4616461BF014FF5D
:10F8F00028B921490320BDE8F84017F005BC20468F
:10F900001BF0E7FDA8B321461C481CF0ADFF0446E0
:10F9100088B30146012238461EF0F4F80546204619
:10F920001CF004FC28461DF0F7FC044640B186425A
:10F930000BD1294638461EF0A3FA20461CF0F6FBF0
:10F940002846BDE8F8401CF0F1BB1BF097FC0028EE
:10F95000F3D03146012220461EF089FC06460028DD
:10F96000EBD0014620461EF08BFA30461CF0DEFB41
:10F97000E3E70349BEE7F8BD835B0500495C05008A
:10F98000A85C05002DE9F04786B000AF81460C4623
:10F990001546E8461BF0C0FE40B92649032017F083
:10F9A000B3FB1837C546BD46BDE8F08720461BF0BF
:10F9B00090FD08B92049F1E7214620481CF054FF8A
:10F9C00082460028EDD02946381D16F099FB002408
:10F9D00007F10805786830B1042C21D12246184976
:10F9E000032017F091FB78681CF0A0FB0022514621
:10F9F00048461EF087F81DF093FC064650461CF062
:10FA000095FB2EB123462A463146484612F0A6FB06
:10FA100030461CF08BFB294620461DF0B8FBC0E7A2
:10FA20001DF07AFC45F82400381D16F058FB01340F
:10FA3000D0E700BF835B0500065B0500495C05005D
:10FA40003F5B0500F7B5014601A816F059FB1A4FB8
:10FA500000260198C8B11DF05FFC044648B31BF0B6
:10FA6000D7FB054628BB20461BF011FC98B922465F
:10FA70003946032017F048FB012520461CF056FBB1
:10FA800001A816F02CFB002DE3D001981CF04EFBD2
:10FA9000304603B0F0BD3EB9B4F80B3003F5007347
:10FAA000A4F80B302646E8E7214630461EF073F8EE
:10FAB000E3E70025E1E700BFE659050070B505461C
:10FAC0000E461BF0FFFBA8B10122104928461DF08D
:10FAD000F5FD04461BF033FB90B922460C49032088
:10FAE00017F012FB20461CF021FB2846BDE87040B1
:10FAF0001BF047B928461BF0CAFB0028E4D1E8E711
:10FB0000314620461DF0AEFAECE700BF795B0500F8
:10FB1000EB5C05002DE9F84304460F4616461BF042
:10FB2000B6FB054640B929492246012017F0ECFAF8
:10FB30002C462046BDE8F88330461BF0A8FB05465E
:10FB400010B932462249F0E738461FF089FA002200
:10FB50002049814630461DF04FFE002207461E49CF
:10FB600030461DF049FE8046B7B9A8B900221B49AE
:10FB700030461DF041FE05462A46494620461DF006
:10FB8000F3FF294648461DF02CFBB4F80B3003F573
:10FB90000073A4F80B30CCE706201CF023F90546CF
:10FBA00060B11FB13A460B491DF0E2FDB8F1000FFC
:10FBB00004D04246084928461DF0DAFD4146384641
:10FBC0001DF00FFB002DD7D1D0E700BFAE5A0500C6
:10FBD000D75A0500C0750500F763050056540500A7
:10FBE00073B504460D461BF052FB064640B91A4950
:10FBF0002246012017F088FA3446204602B070BD34
:10FC000028461BF044FB064610B92A461349F0E784
:10FC1000294601A816F074FA019D35B9B4F80B30E5
:10FC200003F50073A4F80B30E7E7B5F80B3003F5E4
:10FC30000073A5F80B3028461DF06EFB29460646DA
:10FC400002462046FFF766FF324629461DF0BCFA01
:10FC500001A816F044FADFE7595A0500835A050057
:10FC600070B5044688B008461FF0FAF906462046EB
:10FC70001BF052FD054640B10022314620461DF0E2
:10FC800041FF10B11CF052FA04E020461BF0FFFACD
:10FC900030B1002530461CF049FA284608B070BD46
:10FCA000204611F02BF805460028F2D020226946A4
:10FCB00030461EF0EFFC28466A46214611F008F94E
:10FCC000051C18BF0125DDE7F8B507460C46FFF710
:10FCD000C7FF10B900242046F8BD20461FF0C0F928
:10FCE000012204460146384617F014FB054620461B
:10FCF0001CF01CFA002DEDD01CF0EFF8044628464D
:10FD000014B91CF013FAE6E71BF041FA0646384630
:10FD10001BF0EAFA074601201CF0ECF823490246E2
:10FD200020461DF03CFD002F37D02846B84780F014
:10FD30000100C0B200F001001CF0DCF81C490246D2
:10FD400020461DF02CFD86F00100C0B21CF0D2F858
:10FD50001849024620461DF022FD28461EF00FF8E5
:10FD600006461BF0C9F9D0B10022134930461DF0F8
:10FD700043FD1149024620461DF011FD00220F49A6
:10FD800030461DF039FD0D49024620461DF007FDA5
:10FD900030461CF0CBF92846B3E70120CAE72846D5
:10FDA0001DF0BAFA06490246EFE700BF585B0500AE
:10FDB000615B05006C5B0500C0750500F76305001D
:10FDC0005654050010B5142994B0A8BF14210C4650
:10FDD0001EF0D4FC24EAE4740A2351EC100B0093C7
:10FDE00002AA4623019415F057FE02A81DF0F0F870
:10FDF00014B010BD30B5044695B008460D461BF052
:10FE00003DFC48B320461BF083FA28B328461DF07A
:10FE100099FA831E222B05461ED820461BF02EFC85
:10FE200060B120461DF08EFA2B46012202A915F082
:10FE300012FE02A81DF0CCF815B030BD20461EF011
:10FE40009DFC4FF0FF33CDE9005302AA462351EC4D
:10FE5000100B15F021FEECE720461EF09BFAEBE7B5
:10FE600010B504461BF00AFA30B104B124682046EC
:10FE7000BDE810401CF046B820461BF0E2F908B17E
:10FE80006488F4E720461BF024FB20B120461CF0D8
:10FE9000B4FD0446EBE720461BF014FA48B12046B7
:10FEA0001EF0F6FF18B104681CF040F9DFE70446C5
:10FEB000FAE710BD7FB503901BF0E9F948B1039C48
:10FEC000B4F80B3003F50073A4F80B30204604B0EF
:10FED00070BD03981BF0D2F90028F0D103981BF0F5
:10FEE000F1F904460028EAD1039810F03BFC18B958
:10FEF0001BF0F3FF0446E9E715F03AFD054600283C
:10FF0000F6D01DF009FA03AB0193012300932246BA
:10FF100023462946064619F089FB31460446284601
:10FF20001DF05FF9D2E7000070B508B1036823B98E
:10FF30000020BDE870401BF0E5BF00211DF0FAF97C
:10FF400004461BF09BF990B30CB1236823B9002041
:10FF50001BF0D8FF054602E0012B0AD00025204601
:10FF60001CF0E4F8BDBB9FED1E0BBDE870401BF01C
:10FF7000B7BF002120461DF0DDF906461BF0A9FAA7
:10FF800058B130461BF0C4FA38B100201BF0BAFF5C
:10FF9000054630461CF0CAF8E1E730461BF00EFB80
:10FFA00018B930461EF0E8FEF2E70025F1E7002C14
:10FFB000D4D020461BF06BF90028CFD120461BF08F
:10FFC00088FA20B120461BF0A3FA0028BFD12046B2
:10FFD0001EF0D2FEBEE7284670BD00BFAFF3008022
:10FFE000000000000000F87F38B512F009FA05465D
:10FFF00012F07EFA044650B1284609F033F880F03A
:020000023000CC
:100000001000C0F300142146284612F0CFFE20460F
:1000100038BD10B50C4612F0F3F921460022BDE8B8
:10002000104002F0E9BB08B512F0EAF9BDE808405B
:1000300002F0C2BB1FB50C468DED000B12F0E0F9CB
:100040009DED000B8DF80F00002251EC100B0A4BB8
:1000500022F0E8FF0022094B22F0E4FF0022064BC9
:1000600023F00AF923F03EFB23460DF10F02F0F7CF
:1000700085FF04B010BD00BF00408F40000030413C
:1000800008B512F0BDF9BDE8084013F073BC0000DC
:1000900070B506460D461BF01CFA28B9154901201B
:1000A000BDE8704017F030B828461BF012FA20B9AE
:1000B00028461BF007F90028F0D0FCF7C7F90446E2
:1000C000B8B1284614F052FE054648B932460A49EE
:1000D000012017F019F82046BDE870401CF026B842
:1000E0000246314620461DF03FFD28461CF01EF812
:1000F000F1E770BD535905008359050070B5AEB0E6
:1001000005461BF0E6F9044628B93D492A46032076
:1001100016F0FAFF0BE080220EA928461EF0BAFA6C
:100120007F2807D93749032016F0EEFF0024204628
:100130002EB070BDFCF78AF90546002858D0002281
:100140000EA91DF0BBFA1DF0EBF8044628461BF083
:10015000EDFF002CEBD12C490EA823F09FFC0028CA
:1001600034D02A490EA823F099FC002842D028490F
:100170000EA823F093FC00283ED026490EA823F0B9
:100180008DFC00283AD00EA823F09AFC1C2819D820
:1001900007AD0EA928461FF073FB0023CDE90333FA
:1001A0000BAB93E807008DE8070095E80F001FF000
:1001B00003F9064630B114F0D9FD054630461BF070
:1001C000B5FF55B90EAA14490120A1E71348002133
:1001D0001BF076FE05460028D5D0FCF737F904461B
:1001E00018B12A460EA91DF0C3FA20461BF09EFF47
:1001F0002C469CE70A48EAE70A48E8E70A48E6E7A7
:10020000C45F0500F45F0500196005001F6005006C
:1002100027600500E55E050032600500F1F503008A
:10022000D9F50300D5F50300B5F50300F8B515467B
:1002300004460F46084A194628461E4616F016FD83
:10024000240B14F1FF3400D2F8BD3A46314628465B
:1002500016F00CFDF5E700BF818405002DE9F041A3
:10026000774D2B68B3F90240822C8AB02E465FD0BE
:1002700021DC5B2C6CD00CDC2D2C3FD002A920465D
:1002800020221FF0D9FB02AA6E49022016F03CFF83
:100290003BE07B2C00F09080812CEFD11FF048FDDB
:1002A00015F08AFE04460D461FF0C4FD204629467F
:1002B0001BF03DFE19E0B42C12D007DC832CDDD1FD
:1002C0001FF096FB04461FF0B5FD0FE0B52C11D0D2
:1002D000B62CD3D11FF0AEFD02201BF083FD04E04D
:1002E0001FF0A8FD01201BF005FE044620460AB0C1
:1002F000BDE8F0811FF09EFD0020F4E71FF09AFD9D
:100300002B685B88813B012B01D90024EEE7FFF7C6
:10031000A5FF054600201BF0F5FD224629460646AE
:100320001AF05EFA3146044628461CF05AFFDDE713
:100330001FF0FEFC0021F0F7BFF9CDE900011FF02E
:1003400079FDDDE9000141EC100B1BF0C9FDCCE7A4
:100350001BF0C0FD04460028D7D01FF06BFD3A4FBC
:100360003368B3F902305D2B03D03B8A03F070038E
:1003700043B15D2020F0F6F90028B7D120461BF0EC
:10038000D5FEC2E7FFF76AFF054640B13368B3F90F
:1003900002305D2B08D02C2020F0E4F920B9214652
:1003A00028461CF01EFFB0E7294620461DF01EF926
:1003B00028461BF0BBFED3E71BF08FFD0446002848
:1003C000A3D01FF037FDDFF880803368B3F9023027
:1003D000832B04D1B8F8103003F070030BB17D20EB
:1003E000C8E71FF005FB1EF0BDFE07461FF022FD0B
:1003F0003A2020F0B7F930B9002522462946384680
:100400001CF0E2FE81E7FFF729FF05460028F3D044
:100410003368B3F902307D2B04D02C2020F0A2F9F0
:100420000028EAD0294638461CF070FC01462046D8
:100430001CF0FEFF394628461CF0D3FEC5E700BF7E
:10044000C09F002033590500602D002070B59CB07E
:100450001DF0A0FF094C01AB05462668236020F083
:10046000E9F928461BF062FEFFF7F8FE05461FF08B
:1004700089FC284626601CB070BD00BFC09F0020CC
:1004800070B58EB007AC0E46014620461FF0D4F979
:100490000023CDE903330EAB13E907008DE8070015
:1004A00094E80F001EF088FF054668B1FFF7CEFF05
:1004B000044628461BF03AFE1EB115F0D3F91BF096
:1004C00035FE20460EB070BD0446FAE72DE9F34133
:1004D00008B103688BBB3A4B3A4D18883A4E1AF074
:1004E0005FFD0146044601A815F00AFE019830B9E7
:1004F00020461DF090FD20461BF018FE26E01CF063
:100500000BFF0022294680461DF076F9074611F0C0
:1005100077FFC0F3471200F01F0356F82210D940AE
:1005200011F0010101D108F0F9FC384641461CF0F8
:1005300058FE01A815F0D3FDD8E700211CF0FAFE03
:10054000044630B92149012016F0DEFD02B0BDE8B5
:10055000F0811B4F38881AF023FD00222146064601
:100560001DF0D0FA054630461BF0E0FD15B32846D5
:100570001CF0D2FE0022134980461DF03DF911F017
:1005800095FF064640461BF0D1FD38881AF008FD5D
:10059000294607461DF074FC394628461CF021FE0A
:1005A000304611F045FF01460028A4D1304608F03E
:1005B000B5FCA0E722460649012016F0A5FD9AE702
:1005C00064A700204455050060A70020E5580500F9
:1005D000225905002DE9F84380460C4617469946F6
:1005E0001AF077FF18B900242046BDE8F8832046AA
:1005F0001DF0D0FE06460028F5D040461CF0FDF95F
:10060000044630461CF0F9F9844205DA30461BF006
:100610008DFD4FF0FF34E7E7241AB9F1000F0DD13B
:100620003846651C1AF074FE38B338461CF08AFE52
:10063000041E22DBA542E9DB012710E038461AF050
:1006400067FE38B138461CF07DFE002818DB844276
:10065000A8BF04464FF0FF352F4600E03C44AC42B3
:10066000D4D00123224631464046EFF7E3FF00286D
:10067000F4D130461BF05AFDB6E701270024EEE71F
:100680004FF0FF352F46F9E72DE9F04F9BB0884634
:10069000154681461DF07EFEA949064640461DF0DE
:1006A000C9F804462846002C00F018811AF00AFE0A
:1006B000002848D0B5F80B3003F50073A5F80B30CF
:1006C00000201BF01FFC9F49024640461DF067F8C2
:1006D00067214046FBF7C4FE04901B201BF082FB01
:1006E00000220146059008A816F0F7F8314640466A
:1006F000FDF76EFE4FF0000904463CB120461AF0AB
:1007000087FD18B915F08EF9074630B36FF0004336
:100710004A46314608A816F073FF0B981BF006FDF9
:100720003246294620461CF04FFD049B3BB1002079
:100730001BF0E8FB8349024640461DF030F805985F
:100740001BB0BDE8F08F28461AF0C3FE0028B1D1D7
:1007500028461DF01FFE0546B2E7394620461CF02C
:10076000E9FD3A467849039020461DF045F81DF012
:100770007DFB069003981CF040F9069B079008AF9C
:100780004A46A3EB09033146384616F039FF28469E
:100790001AF098FD0DF1340A0246002866D0039B3A
:1007A000039AB3F80B3003F50073A2F80B3001275E
:1007B0000D92394620461CF0BDFD07F1010B814624
:1007C00000284FD10246604920461DF015F81AABAB
:1007D00003EB87034A4643F8340C5C4920461DF07E
:1007E0000BF81AAB03EB8B0B02374BF8340C0DF103
:1007F000340B4B464A464946CDE9007B284618F063
:1008000015FF1DF0C6FE5946824638461CF0BFFC57
:1008100008A86FF000434A46514616F0F1FE5046D4
:100820001BF084FCDDE906320398134499461BF063
:100830007DFC20461BF07AFC049B002B4CD0079BD0
:10084000002B14BF484609F101001BF05BFB3D493A
:10085000024640461CF0A3FF31464046FDF7B8FD76
:1008600004464AE74AF827905F46A2E729465046E1
:1008700016F033F8DDE90D239A4201D31098CFE743
:10088000504615F023FF2428014623D1504615F089
:100890001DFFA0F13102D2B2082A834611D8A0F17F
:1008A000300120461CF046FD814650B101466FF0F4
:1008B000004308A8002216F0A3FE48461BF036FCB1
:1008C000D8E72421384615F027FC5946384615F05C
:1008D00023FCCFE708A8FAE7049C17E71DF05AFDB0
:1008E000074640461DF056FD234601460546224672
:1008F0004846FFF76FFEB0F100091ADB4A46214671
:1009000030461BF0A0FF6FF0004322463946804678
:100910001BF06CFF28461CF070F8314609EB000212
:100920006FF0004340461BF061FF30461BF0FEFBBA
:100930004646394628461CF054FC0596FFE600BFA3
:100940005C540500635405006D5405005C620500AD
:100950002DE9F84F06460D461AF0BBFD18B90024E4
:100960002046BDE8F88F002DF9D0464928461CF0F6
:1009700061FF0446002858D000201BF0C3FA42490A
:10098000024628461CF00BFF31462846FDF720FDA5
:10099000672104462846FBF763FD0028E0D01BF0E2
:1009A00099FA07460028DAD0DFF8DCB024B12046F7
:1009B0001AF02EFC804660B120461BF0B7FB0020E9
:1009C0001BF0A0FA3049024628461CF0E8FE3C46DF
:1009D000C6E7414620461CF0ADFC42462B49814605
:1009E00020461CF009FF1DF041FA804648461CF0E5
:1009F00004F849468246804438461CF010FE2046E2
:100A00001BF094FBBAF1000F14BF404608F101003F
:100A10001BF078FA5946024628461CF0C0FE3146C3
:100A20002846FDF7D5FC0446C0E728461DF0B2FC79
:100A300023460146054622463046FFF7CBFD061EFB
:100A400018DB1BF047FA044618B928461BF06EFB6A
:100A500086E729461CF0CAFD30461BF053FA0B49C5
:100A6000024620461CF09BFE2A46094920461CF0FF
:100A700096FE75E728461BF059FB0220BDE8F84FAB
:100A80001BF0B0B95C540500635405006D540500BB
:100A90005C6205002DE9F04F814699B008460C468E
:100AA0001AF0F5FB002863D14FF0000846461BF012
:100AB00011FA0746002857D04FF4D82420220021ED
:100AC00010A80094EEF72EFD012210A920461EF07A
:100AD00071FB002848D04FF0000A119B002B3CD03E
:100AE0009DF84330DAB218EA020F36D10EB1164241
:100AF00033D05B0612D50DF145020023591C1C2989
:100B00004AD012F8010B002844D118AA134413F854
:100B10001C2C012A21D10EB103F81CAC11AD0FCD54
:100B200001AC0FC495E8070084E807000DF1040C40
:100B3000BCE80F0008AD8DF83CA00FC594E8070095
:100B400085E8070008A81CF043FA0546B9F1000F34
:100B500024D1294638461CF062FD012210A96846BE
:100B60001EF0B0FB0028B8D1384619B0BDE8F08FB0
:100B70000022154920461CF03FFE002894D01DF0AD
:100B8000B1FB002815BF4FF000084FF04008402689
:100B900000268CE70B46B1E71B23B6E74946FFF773
:100BA000D7FE834668B11AF033FB80F00100C4B26F
:100BB00058461BF0BBFA002CCBD128461BF0B6FAE6
:100BC000CBE70446F4E700BF8D6105000149002032
:100BD00014F02CBA7F5F050038B50546FFF7F6FF25
:100BE000044610B12946FDF739FE204638BD000005
:100BF0002DE9FF418046FFF7E9FF0446002839D080
:100C000048F208011D481BF05BF948F20801029008
:100C10001B481BF055F90390029818B12246194958
:100C20001CF0A6FD039818B1224616491CF0A0FD41
:100C3000154D2E8A02AFB6B2B8F1000F0AD00223CA
:100C400000930023224619460197404618F0EEFC17
:100C50001BF06CFA394602202E821CF098FA14F030
:100C600001FE054630B101462046FDF7F7FD284656
:100C70001BF05CFA204604B0BDE8F081CDE502002F
:100C80005DE80200144D0500602D002070B505469A
:100C9000FBF7C8FC044640B1B5F80B3003F5007310
:100CA000A5F80B302C46204670BD28461AF0EFFA06
:100CB00040B9FFF78BFF04460028F4D02946FDF722
:100CC00085FCF0E72246094928461CF095FD0646BA
:100CD0001AF0F8FA10B13046FFF78AFF04463046A2
:100CE0001BF024FA002CDED1E3E700BF875F05008C
:100CF0002DE9F04385B0012301920746884610464E
:100D0000594901AA11F062FA0022584901981CF0D1
:100D100073FD00220546564901981CF06DFD0446FE
:100D2000002D37D0B0B30022524928461CF064FD94
:100D3000039060B31BF061FE48B34E4928461DF096
:100D40004FF900224C49204616F06AFB06461AF07D
:100D5000B9FA38B103AB01222146304612F026FE23
:100D60001BF0E4F930461BF0E1F9002243490198F9
:100D70001CF042FD81461CF0E5FA064603981BF084
:100D80003CFE3044C9F8000048461BF0CFF90398F8
:100D90001BF0CCF900223A4901981CF02DFD1DF002
:100DA000A1FA002849D07CB336492046FEF788FDD9
:100DB00035492046FEF784FD00223149204616F0D1
:100DC0002FFB06461AF07EFA38B100231A46214658
:100DD000304612F0EBFD1BF0A9F930461BF0A6F9E6
:100DE00000222949204616F01BFB06461AF06AFA33
:100DF00038B100231A462146304612F0D7FD1BF0C9
:100E000095F930461BF092F9BDB11F492846FEF70F
:100E100057FD00221C49284616F002FB06461AF030
:100E200051FA38B100231A462946304612F0BEFD69
:100E30001BF07CF930461BF079F9214628461CF05E
:100E4000D0F9D8F800402CB1B4F80B3003F500739A
:100E5000A4F80B30214638461DF012F820461BF04E
:100E600065F905B0BDE8F08379560500B75F050068
:100E7000855605009F3C05009156050097560500D4
:100E8000525F0500676F0500A0560500044B054939
:100E9000002814BF0322002258681CF0ADBC00BF1C
:100EA000602D0020626205002DE9F3410746002015
:100EB0008846FFF7EBFF044640B1014601A815F054
:100EC0001FF9019828B920461BF030F902B0BDE89F
:100ED000F0811CF021FA0022414606461CF08CFCF1
